:020000040800F2
:1000000000500020FDCB0008A9CC00080DB7000867
:10001000A9CC0008A9CC0008A9CC00080000000069
:10002000000000000000000000000000A9CC000853
:10003000A9CC000800000000A9CC0008FDB600080B
:10004000A9CC0008A9CC0008A9CC0008A9CC0008BC
:10005000A9CC0008A9CC0008A9CC0008A9CC0008AC
:10006000A9CC0008A9CC0008A9CC0008A9CC00089C
:10007000A9CC0008A9CC000899B50008A9CC0008B3
:10008000D5B50008A9CC0008A9CC0008A9CC000867
:10009000A9CC0008A9CC0008A9CC0008A9CC00086C
:1000A000A9CC0008ADB40008A9CC0008BDB4000874
:1000B0009DB400088DB400087DB40008A9CC0008E8
:1000C000A9CC0008A9CC0008A9CC0008A9CC00083C
:1000D000A9CC000855B50008A9CC0008CDB400088B
:1000E000A9CC0008A9CC0008A9CC00080000000099
:1000F0000000000000000000000000000000000000
:0C01000000000000000000005FF808F1A3
:100110002DE9F04F684B694C9FB02360002363606A
:100120000AF058F918B906F023FF0AF075F90AF039
:1001300087FE00230893624D09930A934FF4E0135E
:100140000B932B685F4A43F48033917B2B60AB6940
:10015000924643F01003AB612B6803F4003309931C
:10016000089B01330893099B1BB9089BB3F5A06F4B
:10017000F2D12A68524B12F4003201D0022315E06A
:10018000186840F00100186008922B6803F0020321
:100190000993089B01330893099B1BB9089BB3F58E
:1001A000A06FF2D12B689F073BD501230A93464BE2
:1001B00046481A6842F010021A601A6822F00302D8
:1001C0001A601A6842F002021A606B686B606B6812
:1001D0006B606B6843F480636B603D4B1A68043B53
:1001E00022F070425A603B4A10606868904620F4E2
:1001F0007C106860586840F000405860D86820F46F
:100200000040D8609B6813F4004F17BF324B4FF487
:10021000E01313604FF480130B930A9B012B01D161
:1002200017E0FEE7022B18D169B10B9BB3F5801FD5
:1002300002D14FF4A01305E00B9BB3F5E01F02D1F0
:100240004FF400130B936A680B9B134343F4803302
:1002500002E06B6843F460136B602B6843F08073BB
:100260002B602A68164B9601FBD55A6822F00302D0
:100270005A605A6842F002025A606B68104A03F0F2
:100280000C03082B0593F8D15168144B01F00C01B5
:10029000042903D0082905D00C4A01E0D8F8002031
:1002A0001A6028E051685068C1F38341C00301F12E
:1002B000020117D40A4A1CE089680008A40500203E
:1002C00000100240C81900200020024000127A00ED
:1002D0000410014014000020001BB700840000201F
:1002E00000093D00526812F4003FD8F8002018BF02
:1002F0005208514319606A68DFF844B3C2F303122D
:10030000424411791A681EAFCA401A60BB4B0026DE
:10031000CBF80830BA4BBB48CBF80C30AB69DFF8F0
:10032000249343F00103AB616B6A43F080736B620B
:10033000AB6943F01C03AB614FF6FF7327F82C3D0C
:10034000394603928DF84E6009F09AFCAE48394662
:1003500009F096FC3946AD4809F092FCD9F8043012
:10036000384643F00073C9F8043004F079F9139B60
:10037000A749039AB3FBF1F3A3604FF47A73B2FB7E
:10038000F3F2A44B013A5A60F0228BF823200722A3
:100390009E6064201A6006F056F99F48314690220C
:1003A0000EF08FFBD9F8043023F4406343F0706300
:1003B00043F40063C9F80430EB6943F00703EB61D1
:1003C000AB6943F4006343F00C03AB613346934ED7
:1003D0004FF0000906F10C0203F8029001330C2BD8
:1003E000F5D1FF2333767376B376F376AB69DFF816
:1003F00058B243F008039BE8030087E80300AB61B1
:10040000814B08221A61139814A909F039FCAA69D2
:100410004FF40043ADF84C3014238DF84E3042F0C9
:10042000040202238DF84F307648AA6139460293C0
:1004300009F026FC7A497B4A48460BF1080B11600B
:1004400006F00BF99BE80300AA6987E8030042F075
:100450000802AA61139814A909F012FC07F0D6FB50
:10046000DAF808B049460BF400600490102206F157
:100470001C000EF026FB029B012207211BF4004FFB
:100480008DF83B908DF83A30ADF83820B277F1779F
:1004900006F11C090CD0032086F8202086F82120C4
:1004A00086F8222086F82310ADF838001E4600E0BA
:1004B000164654480EA904F01DF9049B9BB1022373
:1004C00051480EA9ADF8383004F014F9092301227F
:1004D00084F8283084F82A20731C072284F82960C5
:1004E00084F82B20DEB26B694F4843F001036B6147
:1004F000AB69DFF834B143F40073AB6105F0C6FDBE
:100500004A4B002513934A4B012E14930CBF2B46E4
:10051000802318934FF4807319934FF480631A93D8
:10052000202339461B9358464FF4005316961C93CC
:10053000159517951D9505F08BFDDBF800303D4AAC
:1005400043F00103CBF800305368012E23F47023ED
:1005500094BF0021012123F4807343EA01235360F7
:100560009168354B013E0B4043F4602343F0020396
:100570009360D16AF6B221F4700141EA0656D66260
:100580002846012309EB00018A78002A7AD02B4AF9
:100590005D1C825CCF78092AEDB2264910D9A2F100
:1005A0000A0606EB46064FF0070E0EFA06FEB740A7
:1005B000D1F80CC02CEA0E0E4EEA0706CE600DE014
:1005C00002EB42064FF0070E0EFA06FEB740D1F8D6
:1005D00010C02CEA0E0E4EEA07060E61062B1549D6
:1005E00034D8013B03EB83031F269E409A404F6B98
:1005F00027EA060646EA02034B6344E000000008CF
:100600000005FA0500080140000C014000100140FF
:1006100040420F0010E000E088180020A4050020F0
:10062000F55E000870210020080002404C240140C3
:10063000D005002000240140FDF7F1FFC005002097
:1006400000ED00E0000001408C0601080C2B0CD8E6
:10065000073B03EB83031F269E409A400F6B27EA5C
:10066000060646EA02030B630DE00D3B03EB830332
:100670001F269E409A40CF6A27EA060646EA0203F2
:10068000CB6200E01D460430102801D02B4679E7EC
:10069000A74B9A6842F480729A609A6842F001020D
:1006A0009A609A6842F008029A609968A04A09071D
:1006B000FBD4936843F0040393609D4A936813F05E
:1006C0000403FAD19168BAF8E60041F4A001916000
:1006D000984A50B9B2F9E83033B9B2F9EA30D3F1F7
:1006E000010338BF002300E0034613F0010340F08C
:1006F000818088F8143000B20BF03AFD8E490BF07F
:100700008BFD8C4F0646B7F9E8000BF031FD8A49A6
:100710000BF082FD0546B7F9EA000BF029FD86498A
:100720000BF07AFD814630460EF0FAFB0746304664
:100730000EF06AFC804628460EF0F2FB064628467C
:100740000EF062FC054648460EF0EAFB824648463B
:100750000EF05AFC3946814650460BF05DFD394695
:10076000834648460BF058FD5146049040460BF036
:1007700053FD4946069040460BF04EFD314607902A
:1007800050460BF049FD4946606306F100400BF00E
:1007900043FD2946A063E56306980BF03DFD014645
:1007A00004980BF031FC2946206407980BF034FDC7
:1007B000014658460BF026FC3146606408F10040C3
:1007C0000BF02AFD2946A06458460BF025FD014692
:1007D00007980BF017FC2946E06404980BF01CFD09
:1007E000014606980BF010FC3946206530460BF0A8
:1007F00013FD6065514E524A33684E4D43F002037B
:100800003360136894F858A0B3F852B04D4B0021F0
:10081000B5F8EE8095F8ED7019709946BAF1000FB1
:1008200008D00023A4F85A30BAF1000F08D109F01B
:10083000FBFE05E008F0A0FD002800F0FA80F0E7DC
:10084000B8F1140F19D009D8B8F1050F19D0B8F1C3
:100850000A0F14D0B8F1000F0DD114E0B8F1BC0F9D
:1008600013D0B8F5807F04D0B8F1620F03D1022114
:100870000CE000210AE0032108E0042106E0052144
:1008800004E0062102E0072100E001212E4B1A209E
:100890001A8822F040021204120C1A801A8822F0E0
:1008A00038021204120C42F030021A801A8892B2F6
:1008B00042F040021A8009F0A9FE012005F0B8FEBE
:1008C00013A806F021FA9DF94E30013303D19DF9AA
:1008D0004C30013303D0B4F85A309BB21BB1002323
:1008E000A4F85A30A5E0194C194B64202360194B29
:1008F000A0466360184BE36005F0A5FE042389F869
:10090000003033680120034304903360134C00230C
:10091000062F2370DFF848A024D0092F02D0002F23
:1009200040D11FE0336823F0020333603AE000BF98
:1009300000240140C819002035FA8E3C88020020AE
:100940001802002032020020003001401C0200206A
:100950003D960008096D000890C1793D9E02002077
:100960006D210020A14A92F8583033B10021A2F83D
:100970005A1053B909F058FE07E00392029308F0A9
:10098000FBFC039A029B68B1F0E7994B994A6420FB
:100990001A60994A5A6005F056FE06238AF800301C
:1009A000042323709AF8003033B90FB11F46ADE726
:1009B000336823F002033360336823F004023260AB
:1009C00095F8E2200AB189F8002095F8E3200AB1F1
:1009D0008A490A7095F8E4200AB189490A709A0791
:1009E00002D5834B1B689847D8F800309847336886
:1009F0007E4C13F0080F19D00FFA8BF9642799FB7E
:100A0000F7F630460BF0B4FB824607FB169000B2B7
:100A10000BF0AEFB7B490BF0FFFB014650460BF0A1
:100A2000F3FA79490BF0F8FBE06505E00023E36594
:100A300002E0032005F03EFE744B08221A610A27EB
:100A4000724E1920F368013F83F00803F36005F04C
:100A5000FAFD012005F001FE192005F0F4FD00204B
:100A600005F0FBFD17F0FF07EAD108233361684B5F
:100A7000684E1B6893F90C000BF07AFB66490BF08B
:100A8000CBFB0EF04DFA074630880BF071FB394670
:100A90000BF0C2FB0EF07AFA604B614F1880308881
:100AA0000BF066FB01465F480BF06AFC5E490BF0F9
:100AB00067FC59492066D8F80C000BF0ADFB5B4988
:100AC0000BF0AAFB5A4B5B4A18606B795A4E1370B5
:100AD00007EBC3035B7C594A3360AB6862669B06D5
:100AE00044BF0123336009F095F90EA800211422B8
:100AF0000DF0E7FF6B790E2B01D0082B02D10123FB
:100B00008DF84230AB683168C3F340028DF83D2068
:100B1000C3F380128DF83E20C3F340328DF83820A5
:100B2000C3F3C03200318DF83A204548C3F3C022E8
:100B300018BF01218DF83B20C3F300428DF83F2000
:100B40008DF8401003F0010201688DF8392091F80A
:100B5000B011B5F8E000C1F380018DF84110ADF897
:100B60004600B5F8DE104FF47A70ADF84800D804AE
:100B7000ADF8441004D5334BB3F8DA30ADF8483053
:100B8000B1F5FA7F84BF0023ADF84830B5F81A31CB
:100B90002D49ADF84A3095F8223184F868300023A9
:100BA00084F869304B709DF84230002B14BF02234B
:100BB000002302B1013307EB8303D3F8C8304FF0B1
:100BC00000090693CA4606994FF6FF7231F809707C
:100BD0009742FBB23AD194F8693084F86B30154BE8
:100BE0001F78162F40F09181002681E1A405002096
:100BF0008C0200202D960008A56C00089E020020A3
:100C0000742100208988883C00002041000C0140AC
:100C1000D80200200000002035FA8E3CFC020020A3
:100C20008C0601080AE81C4100401C46BD37863589
:100C3000D4020020E8030020E4030020D81900209B
:100C400018020020C81900200D060020DFF838C364
:100C50009DF83C204FEA03180CEB08061AB19A1EC7
:100C6000012A40F22F819DF83E202AB15CF808202D
:100C7000B5498A4200F026819DF83F202AB15CF8F0
:100C80000820B1498A4200F01D819DF83A2012B136
:100C9000012B00F017819DF83D1011B1042B00F0DD
:100CA00011819DF83B1011B1032B00F00B8112B1A3
:100CB000052B00F007813F0A022F9DF8382003D151
:100CC000002A08BF002703E0012F08BF9DF83970F4
:100CD0009DF8401039B19DF8421021B9A3F10801E7
:100CE000012998BF04279DF8411031B19DF84210A9
:100CF00019B9043B032B98BF0427AAB1FB1EDBB232
:100D0000012B09D85CF80830B3F1804F00F0DA808D
:100D10008D4A93424DD1D5E0022F05D15CF80830C1
:100D20008A4A934247D1CDE0012F42D1FF2384F874
:100D3000B03084F8B130B3684FF0000BF27B7068CC
:100D400084F8B4B0C4F8C060ADF84C3013A90223E5
:100D50008DF84F3084F86CB0C4F870B0C4F874B03B
:100D6000C4F878B0C4F8ACB084F8B2B084F8B3B0CA
:100D70008DF84E20CDF80CC008F082FFDDF80CC0D5
:100D8000317B5CF808005A4603F020FC3046594697
:100D90003A4604F00FFA6E4B6E49C4F8C4306E4BFD
:100DA000C4F8CCB0C4F8C83030460A1D04F03AF894
:100DB00088E0022F3ED15FFA8AF31C225A4367492A
:100DC0004FF0000B8F18012387F801A087F802B0BD
:100DD00087F80AB08B54F17BB2687068FE60ADF89A
:100DE0004C208DF84E10022213A902938DF84F204B
:100DF000CDF80CC008F044FFDDF80CC0317B5CF886
:100E000008005A4603F0E2FB029B30461A46594658
:100E100004F0D0F9524BC7F818B03B61514B304643
:100E20007B6107F1100107F1140203F0FBFF0AF1E7
:100E3000010A47E0032F2CD1BDF8443094F86A70C2
:100E4000B3F5FA7F0FD9484A3046B2FBF3F20821D6
:100E5000BDF8483092B204F063FA04EB8707C7F894
:100E60009401424B0EE0424A3046B2FBF3F20121BC
:100E7000BDF8483092B204F053FA04EB87073D4BBB
:100E8000C7F89401836094F86A30013384F86A30BB
:100E900018E0042F16D1BDF84630354A304692FB93
:100EA000F3F20121BDF84A3092B294F8697004F06F
:100EB00037FA94F8693004EB87070133C7F8C401A7
:100EC00084F8693009F10209B9F1180F7FF47BAE9B
:100ED00081E6294B06EB030E98E80F008EE80F0021
:100EE000264B10361A78C02E02F101021A7008D073
:100EF000636E0021985903EB06080BF021FB0028D4
:100F0000E7D0AB68DB0441D419E01D4B1B4A03EB6F
:100F1000C70393F810C0D3F8148082F800C0B8F16A
:100F2000000FEED000266645EBDA134A330103EBDF
:100F3000020E43440FCB01368EE80F00F3E7082F73
:100F4000104B4BD14CE000BF0004004000080040B3
:100F50000D95000868060020E99500085806002055
:100F600009460008E194000800127A00099600087A
:100F700040420F00F995000888070020402100201A
:100F80008C060108FE0200204C1D01089B4B93F8C3
:100F90000090B9F1010FD2D9994E4FF00008C84521
:100FA00006F11006CBDA56F8100C4FF07C510BF01E
:100FB00033F94FF07C5146F8100C56F8140C0BF036
:100FC0002BF94FF07C5146F8140C56F80C0C0BF032
:100FD00023F908F1010846F80C0CE0E70E2F03D1C5
:100FE0001A7842F0100202E01A7822F010021A7009
:100FF00004F0BAFB8349844B8448854AC4F8A8327C
:1010000001600023B5F81A01C4F8A412A4F8AE32A6
:1010100084F8B032C4F8B422C4F8B8227D495852DA
:101020000233242BFAD17C4B1A60AB681E0740F1C7
:1010300081807A4B002293F81831042B74D8DFE8B2
:1010400003F003032A505F00012B4FF0030208D185
:1010500084F8BC22072284F8BE3284F8BD220C2317
:1010600008E0022384F8BC32002384F8BE3284F8FE
:10107000BD22072384F8BF320023009310200123F0
:1010800067494FF4E13206F00DFD664BC4F8C40227
:10109000C4F8C83244E00123634A64490093102035
:1010A000052306F0FFFCC4F8CC020646B5F81A0189
:1010B0000BF05EF85E490BF0AFF85E490AF0A2FF54
:1010C0000BF096FA00235C4A98500433402BFAD177
:1010D0005A4B301CC4F8C8324FF0100384F8BF32AA
:1010E0001FE000920123102055494FF4E13206F031
:1010F000D9FC544BC4F8D002C4F8C83210230DE018
:1011000000920123102050494FF4E13206F0CAFC4E
:101110004E4BC4F8D402C4F8C832082384F8BF3256
:10112000003018BF012028B9082008F0B4FB0023C4
:10113000C4F8C832AB68580405D5082284F8BF2229
:10114000434AC4F8C82242F201021A4003F00101E6
:1011500003F400505AB13F4AC4F8C82218B13E4ABD
:10116000082082F8BF0211B10C2284F8BF2294F843
:10117000BF2213F0800FA2F1040284F8C022274D91
:101180007ED0354B05F59672D5F83811C3F8D822C4
:101190000023324A02EB0310D0F8040116468842BD
:1011A00004D00133DBB2042BF3D9002384F8DD3201
:1011B0002B4B0020C4F8F83209F0F2FD294B94F8CB
:1011C000DD221B680021C4F8E43295F8283106EBD3
:1011D00002128B42C4F8E0124FF020000091D2F8C6
:1011E00004210CBF0123032306F05CFCC4F8FC02BD
:1011F000D0BB802008F04FFB39E000BF4021002029
:1012000090070020D81A002064070108040100207C
:101210004C0800206205002008020020C8190020A8
:10122000C9640008E95D0008A0860100D5650008D2
:10123000CDCCCC3F0000B044240100209D5E0008CE
:10124000616500088D5E000815650008795E00087C
:10125000C95E0008D55E0008A40500208C060108C0
:10126000F01A0020C4190020012009F099FD864BD6
:101270001868864B00F5D97204301A6008F034FC07
:10128000834B8449D4F8B4220B608033C4F8003314
:10129000814B824F1A60AB680026D9033E7040F143
:1012A000B4804FF00108DFF828B208F059FB40F293
:1012B0002A3A08F091FB08F06BFB87F80080784F22
:1012C0005246314658460DF0FCFBBB694FF0100901
:1012D00043F00803BB6118238DF8333071480323B2
:1012E0000CA98DF83230ADF8309003F003FAFB69A9
:1012F0006D4D43F00203FB616C4BA7F694771A68BF
:101300006B4BB2FBF3F22B88013A23F45C7303FAC4
:1013100009F323FA09F392B22B801D23AB852A85AA
:10132000A5F814802B8C23F0010303FA09F323FAA8
:1013300009F32B842B8CA9882A8B23F0020322F03B
:10134000730202FA09F203FA09F322FA09F223FA04
:1013500009F389B242F0600243EA0803A9802A83B4
:10136000AE862B842B8B23F0080303FA09F323FAB0
:1013700009F343F008032B83B5F844306FEA434385
:101380006FEA53439BB2A5F84430D7F8A83F43EA2D
:101390000803C7F8A83F384604F078FE454B3846A6
:1013A0001393802318934FF48073199313A94FF468
:1013B00000531C93CDF850B0CDF85490CDF858A000
:1013C00017961A961B961D9604F042FEAB890DA83F
:1013D0009BB243F40073AB813B6843F002033B6074
:1013E0008DF834908DF835808DF836608DF8378023
:1013F00003F06EFE304B1A68304BF2500436802EEC
:10140000F8D103F08EFD03F08CFD2D4FBB685A051B
:1014100040F1908008F09AFA08B1082000E004201A
:10142000012106F05FF8BB6884F82E0613F4806F84
:10143000244D02D1002104911DE02B681B78032B61
:101440000FD12B681B78032B15D1082008F050FF13
:101450000146082005F0ACFF003018BF01200490C1
:1014600009E0042008F044FF0146042005F0A0FF35
:101470000028E6D1DEE7144B049A2D681A702B7809
:1014800043BB124B1D6049E018020020D40300202A
:101490001C1B0020DC04002088050020CE04002056
:1014A00000100240000C01400004004084000020B5
:1014B00000366E01340400404C060108E0040020B0
:1014C000C8190020F4030020F00300201C040020B1
:1014D000A8080020012B21D1354E002130462C22B6
:1014E000C4F830560DF0EDFA8E2373704FF07C097E
:1014F000E0234FF07D08F37086F8009086F82B808B
:101500002C4E002130462C220DF0DBFA8A2373701A
:10151000A02386F80090F37086F82B802B78022B9E
:1015200008BFC4F8345608F011FA08B1C4F83856A8
:1015300008F022FD04F0AEFF1F4B18607B79052BED
:1015400003D11E4B4FF4C8721A801D4B4FF47A72B0
:101550001A801C4B1A7842F008021A701A4B1A783B
:1015600022F002021A70BB689B071ED5174B184A5F
:101570001D461A6003F09EFB282005F064F8059BC9
:10158000013B0593F6D12968124B48781E78024634
:101590000123964203D30133082B0244F9D10E4AAA
:1015A00013708A785343A4F83C361FB0BDE8F08F1F
:1015B000300400205C04002048030020A00200202A
:1015C00068210020FE0200206C210020040400207D
:1015D000CC1A00200804002080000020A14A2DE938
:1015E000F04F1368A04903F59C43A04D20330B60D6
:1015F000AB6885B013F4807F174604D09C4B1B6802
:101600001B681B699847AB6842F201041C405CB937
:10161000984E337873B1964B1B681B681B689847CC
:1016200003F0C4FF347005E0934B1A7801321A704E
:1016300003F0BCFFAB68DA0405D5904B1B68DB07F1
:1016400001D409F0DFFF8E4B3C681868037CCBB1F6
:101650008C4A013B32F91300A0F57A70B0F57A7F1D
:10166000A8BF4FF47A7020EAE0700AF081FD864945
:101670000AF086FE85490AF0CFFD0AF0B9FF7E4BDD
:10168000588039E0AA68160436D57B4A5168611A39
:10169000002931DB04F59C41203151607C494E79B1
:1016A0007C4931F81660417CB6B296FBF1F0117AB4
:1016B000013101F00F0111720A44507218466E4E4A
:1016C00006F109029A5C01331044102B80B2F6D166
:1016D00000B290FBF3F000B26428A8BF642020EAB7
:1016E000E0700AF045FD6C490AF04AFE67490AF0CD
:1016F00093FD0AF07DFF7080AB68D80510D5674B6D
:101700009C42674C08D923681B681B6A984718B924
:1017100023681B685B6A984723681B685B69984766
:10172000AA68DFF860A112F4805F504BB5F8DC10B6
:10173000BAF9062007D0B3F81A31581A824207DDE9
:1017400019448A4202E0B3F81C319A42C0F228845C
:101750000122002195F8238195F82401B5F81C6138
:10176000B5F81E710B463AF901409B08B442C4BF5C
:1017700063F07F03DBB20231BC42B8BF43F04003E9
:101780000829F0D13C4C617E994204D1A17EF9290F
:1017900003D8013100E00021A1766376414B374F39
:1017A0001978A1B93B68D90707D582B93E4B1B7898
:1017B000DB070CD505F03EFE09E03B4B1B785E07CE
:1017C00005D510B109F01EFF01E0002AFAD0A37E72
:1017D000294A142B354E40F09980334B18F10008FC
:1017E0001B7818BF4FF0010803F0040303F0FF005B
:1017F00093B12C490B78002B00F08880537E5F2B2F
:1018000001D109F0FFFEB8F1000F7FD0637E7D2B80
:101810007CD109F0F7FE79E0537E572B0BD1244B96
:101820004FF47A721A80234B1B6813F008036DD1B2
:10183000214A13806AE0A968490745D55A2B43D14C
:101840001E4B197819B1187001221D4B4DE0D17E45
:101850001C4B81F00101D17609B1042245E006223A
:1018600043E000BF5C2100200C020020C8190020CA
:101870000802002000010020E40B00204C0300209F
:10188000040100206205002000007A4400C07F446B
:10189000C0050020D00500200000C842404B4C008D
:1018A000580800202C0000206C2100201802002085
:1018B000682100208802002018030020CD020020AB
:1018C000CF020020CE0200205D2B00F0EF825B2BC8
:1018D00000F0EE825E2B0AD10322EAE2A72B40F051
:1018E0000783AA4B1A7842F004021A700EE0562BB6
:1018F00001D106F0DDF9A64A1378002B00F0EF8243
:10190000637E6F2B40F0E58205F094FDAB685907CC
:1019100031D5E37E9BB19F4B1B785A070FD59E4B69
:10192000BAF90620B3F81C319A4208DD3B6813F07F
:10193000010304D1994A32211180994AD3763B6838
:10194000DB030AD5974B1A782AB9974A127812B94D
:10195000924A3221118001220CE0934B1A7852B145
:101960008C4A127802F0040202F0FF011AB91970D1
:101970008E4B01221A70D6F80090002309F1750BE6
:101980003B6009F1770698460BF1020303EB08016F
:1019900013F808204B7816F8010C9A420AD2314607
:1019A00009F00CFA30B116F8023C01229A403B686B
:1019B00013433B6008F10408B8F1A00F06F10406D8
:1019C000E2D17B4B1B7843B13B68DFF8FC8113F01D
:1019D000020F784E40F09A818FE109F215120192C0
:1019E00009F58B769846019A16F8010C531C03EB07
:1019F000080113F808204B789A4228D2314609F0A2
:101A0000DDF920B3B0786C4B013800EB400096F85C
:101A100004B018444FF00C0CF3780CFB0BFC009353
:101A20005F4B03F11C0909EB0C014A6882420ED09E
:101A3000009A09F80C2000228A60012202FA0BFBAE
:101A400093F84C20486022EA0B0B83F84CB008F165
:101A50000608B8F1480F06F10606C4D1574BDFF867
:101A60006C811E68564B4FF00009D3F800B0D8F8CF
:101A70000030002B00F038811978002900F0348103
:101A8000D8F80420C2EB0B02002A0CDB0BF5FA722B
:101A9000C8F80420012202FA09F294F84C0020EA66
:101AA000020284F84C2018F8040C5A780430C0B2B2
:101AB000002A40F0E1803AF91020B5F81A0100F14F
:101AC000C80C624501DD9B7813E0C838824202DA17
:101AD0009B785B420DE0012303FA09F394F84C2054
:101AE00022EA030384F84C300BF5FA73C8F804308B
:101AF000FAE094F84C2042FA09F2D00700F1F480A1
:101B0000002B304ACCBF02200120013910700A2975
:101B100000F2E280DFE801F0060F1B28315C6E80E6
:101B2000929CA60032781344FA2BA8BFFA2323EA2A
:101B3000E373337007E072781344642BA8BF642307
:101B400023EAE3737370304604F07CFCC4E0F2785F
:101B500030461344642BA8BF642323EAE373F37075
:101B6000216D04F02BFCB7E032791344642BA8BF3D
:101B7000642323EAE3733371AEE072791344642B78
:101B8000A8BF642323EAE3737371A5E0FE0200207B
:101B90002C0000206C210020C8190020B402002075
:101BA000E40B0020CC020020CD020020CF02002058
:101BB0006B21002050030020B40C0108E00300203A
:101BC000C4190020CE02002088020020040C00204E
:101BD000616D4A781A44C82AA8BFC82222EAE27274
:101BE0004A700A781344C82BA8BFC82323EAE373BA
:101BF0000B7071E0616DCA7A1A44C82AA8BFC82266
:101C000022EAE272CA728A7A1344C82BA8BFC82398
:101C100023EAE3738B725FE0616D4A7D1A44C82A40
:101C2000A8BFC82222EAE2724A750A7D1344C82B73
:101C3000A8BFC82323EAE3730B754DE0626D91786A
:101C40000B44C82BA8BFC82323EAE373937043E077
:101C5000626D117B0B44C82BA8BFC82323EAE37332
:101C6000137339E0626D917D0B44C82BA8BFC82364
:101C700023EAE37393752FE0012A2DD13AF910007E
:101C80009B784FF49662B0F5617F92FBF3F305DB2E
:101C900040F633029042B8BF024601E04FF4617251
:101CA000A2F5617292FBF3F3DBB2AB4A581C0C292C
:101CB000107011D194F858209A420DD0A74A042BE5
:101CC00028BF02230A2184F8583001FB0323A44AC9
:101CD0000633136004F0D0FB012303FA09F394F8F0
:101CE0004C20134384F84C3009F10109B9F1040F79
:101CF00008F10C087FF4BBAE66E6AB68DB0514D5D3
:101D0000984B1B681B689B68984770B1D8F80030E7
:101D10009A070AD5338813F001020CD1924943F097
:101D20000103E26522660B8006E03388012223F07E
:101D30000103338000E000223B68580710D57AB1D8
:101D4000328822F0010102F0020289B292B231809F
:101D500052B9E2652266844A41F00201118003E033
:101D6000328822F002023280D8F80020910640F139
:101D700088807E4A127892077CD57D4A1278042AA0
:101D800078D913F4007C328812D002F010039BB291
:101D9000002B76D1744922F0200242F010027548DF
:101DA0000A80754A011D537005F0BCFA022366E0F3
:101DB00022F0100189B2580531802ED56F4B1B6877
:101DC00058896F4BB3F90080B8F1000FB8BFC8F164
:101DD0000008804509DAB3F90230002BB8BF5B4236
:101DE0008342ACBF0023012300E06346DB0714D528
:101DF00002F0200292B2002A43D15F4B61485A7030
:101E0000614B41F020011A685B683180011D6367F6
:101E1000226705F087FA012331E022F03002328098
:101E2000554A53786BBB012151701A46574900201F
:101E300050525749574C5052574904EB030C5052DB
:101E4000002119510232CCF80400CCF8081004F13A
:101E5000280C503443F80C1019519C441C44042A9B
:101E6000CCF80400CCF808106060A16003F1140302
:101E7000DCD106E0338823F030033380002384F87C
:101E80006C303B6813F4006F338814BF43F48073E5
:101E900023F4807333806B79082B02D00E2B40F033
:101EA0009280338823F0400333808CE0012200E0ED
:101EB00002225FFA82F808F1FF3385F8543708F000
:101EC000ABFA08F0BDFF02202821424604F0CCFB0B
:101ED0001CE5B8F1000F02D07E2B3FF415AD637EF8
:101EE000972B7FF4FBAC2D4B4FF4C8721A800DE595
:101EF0000022BB2B039201D1022303E0B72B04D1B4
:101F00004FF6FE73ADF80E300AE0BE2B01D102236E
:101F100004E0BD2B7FF4FAAC4FF6FE73ADF80C3045
:101F20003368BDF80C10B3F854200A44A3F85420C9
:101F3000BDF80E10B3F856200A44A3F8562008F056
:101F40006BFA08F07DFF0F201421012204F08CFBB6
:101F50000023A376DAE400BFCE020020182100207F
:101F6000E00300205808002050030020FE0200205B
:101F700018040020480C00202C000020D40300206E
:101F8000C6030020540C00202404002060210020FF
:101F9000D80300205C0C0020DC030020A0020020FD
:101FA0000A4B00220021DA651A66C3F8F020C3F854
:101FB000F420C3F8F820C3F8FC10C3F80011C3F8EC
:101FC0000411FFF7C6BB05B0BDE8F08FE40B00209D
:101FD000664B2DE9F04FB3F90600654B87B01D68DD
:101FE0002B8998420EDBB0F5FA6FAF7907DAC21A87
:101FF0005743A3F5FA6397FBF3F7643703E0C7F1A0
:10200000640700E064275B4B5B4AB3F81A1193F94D
:10201000EC3016685B4204919BB200210593344674
:102020000A46524BDDF810C0CB5E40F2E63E039309
:10203000CCEB030303F2F31CF44503D8002BB8BF29
:102040005B4201E04FF4FA73022ADFF8388131D0A5
:1020500096F85DE1BEF1000F04D07345CCBFCEEB26
:10206000030300234FF0640EDFF814A193FBFEFC82
:102070006FF0630B3AF81C900BFB0C3B0CF1010C5E
:102080003AF91CA00FFA89FCCCEB0A0C0CFB0BFCF8
:102090009CFBFEFCCC4428F801C095F804C003FB6F
:1020A0000CFC364B9CFBF3F373449BB27B4393FBDA
:1020B000FEFE1BE096F85EE1BEF1000F04D0734512
:1020C000CCBFCEEB03030023DDF814C003FB0CFEF2
:1020D000A8F804E095F805E0002BB8BF5B4203FBCD
:1020E0000EFE264B9EFBF3FE0EF1640EB31893F822
:1020F0000480DFF894C00EFB08F8642398FBF3F823
:1021000002F80C8094F80E900CF103080EFB09F90C
:1021100099FBF3F902F8089094F818800CF1060C7A
:102120000EFB08FE9EFBF3F302F80C30DDF80CE02A
:10213000049B9E45DFF84CE004DA3EF801305B4238
:102140002EF801300132032A01F1020104F10104E9
:102150007FF467AF074EB6F81C31984216DBB0F536
:10216000FA6FA8BF4FF4FA6011E000BF62050020CB
:10217000E0030020C8190020180200200CFEFFFF19
:10218000F00C0020C6030020FE0C00201846C01AE8
:102190004FF47A725043C3F5FA63B0FBF3F364274C
:1021A000A24C93FBF7F204EB42016FF0630000FBDB
:1021B0000233098B04EB4202B2F91A000AB2821A06
:1021C000534393FBF7F73944994F9A4D3B88AEF848
:1021D00006105A063CD5984B1888238EC01A00B2B8
:1021E00009F0C6FF95490AF017F880460CF098FEF2
:1021F000814640460CF008FF8046B5F9020009F020
:10220000B7FF8246B5F9000009F0B2FF49468346A0
:102210000AF002F8414603465046029309F0FCFFDB
:10222000029B0146184609F0EDFE0AF0BBF949464B
:102230002880504609F0F0FF41468146584609F093
:10224000EBFF0146484609F0DFFE0AF0ABF9688073
:10225000B26840F602031340002B53D0784B06219E
:102260001D88636B1D4494F8383065630133DBB21D
:10227000B3FBF1F084F8383001FB103313F0FF0F9B
:1022800040D1930706D502F015FD04F02FF8674BF7
:1022900083F83900B368180532D56A4BE16B5A7B75
:1022A000694B33F81200082391FBF3F280B28A1ACB
:1022B0000244E26392FBF3F292B240F6E4435A43E3
:1022C000624B40F6FF71B2FBF1F219684FF47A737A
:1022D000C8888988121A5A4392FBF1F255435C4927
:1022E00095FBF3F30A60D4E91001C01841EBE371E8
:1022F000C4E910010023574A0AF09AF9564B1860B6
:10230000002363635549494A0B6894F8398013F4F4
:10231000805318BF012382F84830B3688A4613F40B
:10232000807F4F4D2CD0DFF84C912878D9F80030C1
:10233000C0F380001B685B68984760B1012384F894
:102340004930D9F800301B68DB68984718B1374B23
:10235000022283F84920D9F800301B689B6898470F
:1023600028B12B7859075CBF022384F84930D9F88B
:1023700000301B689B69984710B1002384F84930EE
:10238000384B1A6892060DD5DAF8003013F4C06F96
:1023900005D0354B1B789B0701D4012300E00023B7
:1023A00084F84A3094F84920204B022A02D14C206C
:1023B0004E211EE0012A06D153204D214C220B460E
:1023C00008F062FC2BE093F84A20012A03D1532045
:1023D00001464E2206E093F84820012A04D15320FA
:1023E000014602464D23EBE7B8F1000F04D053201D
:1023F0004D210A464423E3E73A88170603D55320C4
:102400004D210246DBE7194A12781AB1192008F06B
:102410000FFC04E0404683F84B8004F01EF92A7854
:10242000500729D5124B08225A617BE0F00C00209E
:1024300050030020C60300201803002035FA8E3C0C
:1024400044030020C0050020D00500200404002023
:102450000C040020407E0500100400204C030020E6
:102460006C21002088020020FE020020CE02002005
:10247000000C01405C080020DAF80030D90703D4D2
:10248000BB4942F001020A70BA4A12881AB1BA492D
:102490000A68920705D4B94A1288003218BF01228F
:1024A00000E0012242B1B64AD16881F00801D16052
:1024B0002A7822F001022A70B24A1278170703D450
:1024C0002A7822F001022A70D80203D52B7823F053
:1024D00001032B702B78AC4A13F0010F05D00023B9
:1024E000E364A74B082119610BE0E16C136841B963
:1024F000A64903F5F42303F59073CB64A04B0821A0
:102500005961E36C12686BB1D21A002A0ADB9C4A4B
:1025100003F5F423D16803F5907381F00801D160CD
:102520009A4AD36407F028FD994B1B7813B106F043
:1025300023FEFAE3012004F0E6FF002800F0F58313
:10254000DFF86C9299F84A30012B40F0E883914A09
:10255000914BD9F80010C2F80090196092468E4A4B
:10256000106804F0D7F8002800F0D3838A4B18686D
:1025700004F0CBF8DAF8003093F84820DAB9B0F17B
:1025800024014A424A4183F84820002AE7D12B78A7
:102590005B07E4D4232802D106F0EEFDDFE7D4F890
:1025A000E8301B7D8342DAD17C4A7D4B1A607D4A3C
:1025B0007D4BDA60D3E7012A04D14D2814BF0022F5
:1025C0000222A3E3022A04D13C2814BF00220322E2
:1025D0009CE3032A0AD140284FF0000200F29683C0
:1025E0001A71DA715871987104228FE3042A06D1A6
:1025F0009A7983F8490050409871052286E3052AAC
:10260000ADD159791A799142997906D94140997198
:10261000511C197113441872A1E7814240F0738371
:1026200093F8490005F050FB002840F06783DAF882
:10263000003093F84930C82B00F0DB8043D82D2BB5
:1026400000F0F18224D8252B00F0CE8206D8212B71
:1026500000F02182232B00F0668182E3292B00F019
:10266000CE822B2B00F0D782272B40F07A830020DC
:1026700004F096F803F05AFE4C4FA7F8E60003F07A
:1026800055FEA7F8E80003F051FEA7F8EA0032E390
:10269000332B00F0DC820CD82F2B00F0EE82312B94
:1026A00040F05F83414FC02004F07AF807F18008C2
:1026B000F9E2412B00F0D382442B00F01683352B36
:1026C00040F04F8351E1D02B00F0F38142D8CC2B66
:1026D00000F0798106D8C92B00F00D82CA2B00F0DA
:1026E000A0803EE3CE2B00F0F88140F2ED8103F0B4
:1026F0001DFE03F01BFE2D4FDFF8B880A7F8D000B9
:1027000003F014FEA7F8D20003F010FED8F800B0D2
:10271000A7F8D40003F00AFEABF8A80103F006FE08
:1027200003F00EFED8F8008003F000FE00EB8000FE
:102730004000A8F8520003F0EFFD87F8040103F011
:10274000EBFD87F8060103F0E7FD87F8050103F0CC
:10275000E3FDD0E2D42B00F068812DD8D22B35D008
:1027600040F2078203F0E2FDA4F8EC00C3E200BFF0
:102770006C210020A0020020880200206821002097
:10278000000C0140FE0200205C210020F00C002023
:102790006B210020A8040020AC040020EFBEADDEB9
:1027A000F04F00200400FA0500ED00E0C8190020F9
:1027B000400D002018020020EF2B25D0FA2B00F04E
:1027C0009681D62B40F0CD82002726E12B7803F0AE
:1027D000040303F0FF07002B40F08D8203F09CFD03
:1027E000C94B022883F8540740F2698183F8547773
:1027F00065E1002703F09AFDC44BD8530237102F30
:10280000F8D10122C24B70E1C24FD7F8008003F02B
:102810008DFDA8F856003F6803F088FDA7F8540026
:1028200069E2BC4B00271A6898461278022A61D1E7
:10283000D8F800B003F070FD07F108020BEB820B33
:1028400009F092FCB44909F09BFDCBF80400D8F8DC
:1028500000B003F061FD07F10A020BEB820B09F0F7
:1028600083FCAE4909F08CFDCBF80800D8F800B025
:1028700003F052FD07F10E020BEB820B09F074FC22
:10288000A74909F07DFD0137032FCBF80400CFD114
:10289000072FD8F800B016D103F03EFD09F064FC14
:1028A0009D4909F06DFDCBF84800D8F800B003F061
:1028B00033FD09F059FC984909F062FDCBF84C0052
:1028C00003F02AFD12E003F027FD0BEB070318715C
:1028D000D8F800B003F020FD0BEB07039873D8F88D
:1028E00000B003F019FD0BEB0703187601370A2F30
:1028F000CED100E2D8F800B003F00EFD0BEB0703D9
:102900001871D8F800B003F007FD0BEB07039873BC
:10291000D8F800B003F000FD0BEB070301370A2FD6
:102920001876E7D1E7E103F0F7FC272821D8794BA7
:1029300000F11C081B6803EB880803F0EDFC794BE1
:1029400008F1050703F58A72197A814203D00C3326
:102950009342F9D10DE01B7888F8053003F0DCFCD8
:10296000787003F0D9FCB87053E003F0D5FC0B2865
:1029700004D90120002103F0F5FEBCE14FF0060868
:1029800008FB00F0634B00F588701B6803EB000840
:1029900003F0C2FC0328ECD888F80A0003F0BCFC62
:1029A00088F8050003F0B8FC88F8060003F0B4FCD2
:1029B00088F8070003F0B0FC88F8080003F0ACFCCE
:1029C00088F8090097E1584FD7F8008003F0A4FC7D
:1029D00088F80000D7F8008003F09EFC88F801001A
:1029E000D7F8008003F098FC88F80400D7F800803E
:1029F00003F092FC88F80500D7F8008003F08CFC07
:102A000088F80600D7F8008003F086FC88F80200FA
:102A10003F6803F081FCF8706DE103F087FC434BE5
:102A2000D8530237102FF8D165E14FF00008394F25
:102A300008F12C0B3968029103F078FC02994FEAF7
:102A4000CB021144C88039680192029103F06EFCF8
:102A5000019A029911440881019203F067FC07284A
:102A6000019A02D839680A445073A0F57A7292B27A
:102A7000B2F57A7F03D83A6802EBCB0250813F6807
:102A800003F04AFC08F1010807EBCB03B8F1080F8B
:102A90001873CCD12FE100271E4BD3F8008003F030
:102AA0003BFC08EBC7030137082F83F86D01F3D116
:102AB00021E12B785F0700F11E8104F059FA07F03D
:102AC000ABFC08F0BDF916E12B78580700F1138133
:102AD000174B4FF4C8721A800DE12B78590700F19B
:102AE0000A81144B1A7842F004021A7003E12B7821
:102AF0005A07E4D535E103F00FFC0E4B1A78D8B134
:102B000042F002021AE000BFC8190020620500204E
:102B10000402002018020020000020410000C842EA
:102B200000007A44D80C0108E0030020DE0D0020EC
:102B3000A0020020FE02002022F002021A7003F020
:102B4000EBFB8C4B8C4F187003F0FAFB386003F0F2
:102B5000F7FB786003F0EAFB884B188003F0E6FB94
:102B6000874B188094F8063143F0020384F806314D
:102B7000C1E003F0D1FB019003F0E2FB029003F00F
:102B8000DFFB804603F0DCFB074603F0CFFB03F0DE
:102B9000CDFB03F0C1FB019A029B9AB9794A82E806
:102BA0000801794B1A8822F010021A80774B1A78A4
:102BB00042F001021A70002F00F09D80744BC3F8A0
:102BC000087198E0102A40F09680724A82E8080165
:102BD00017B16F4BC3F808716E486F4B0222011D8D
:102BE0001A7004F09FFB86E0002003F0D9FD00235B
:102BF000B36003F0A5FBB3681843B0607BE000202E
:102C000003F0CEFD03F092FBA6F8080103F08EFB63
:102C1000A6F80A016FE0002003F0C2FD03F07CFB80
:102C20005E4B587167E0002003F0BAFD03F074FBBF
:102C300086F8180103F07AFBA6F81E0103F076FB74
:102C4000A6F81A0103F072FBA6F81C0153E000205D
:102C500003F0A6FD03F060FB86F820014BE00020A6
:102C600003F09EFD002703F057FB4C4B3B4401371C
:102C7000082F83F81001F6D13DE0002003F090FD0D
:102C8000464F07F1400803F051FBA7F8D40103F0C9
:102C900043FB87F8D60103F03FFB043787F8D301E5
:102CA0004745F0D127E003F041FB00F03F00A7F8D3
:102CB000560103F03BFBB7F85621800100F4F8639E
:102CC0001343A7F8563103F027FB000187F854019E
:102CD00003F022FB97F8543100F00F00184387F8F7
:102CE000540104374745DED105E0002003F058FDCC
:102CF000012384F80C31002003F052FDDAF8003093
:102D0000987903F01EFDDAF80030002283F848209D
:102D100025E494F80C3113B1214A224BDA60224B9E
:102D200009F14C0999457FF40DAC20490B689B06CD
:102D300011D51F4BD4F810211B689A1A002A0ADB00
:102D40000C4A1278042A06D903F51233104A03F507
:102D5000F873C2F81031174B9B683BB1164898477F
:102D600004E00120002103F0FDFCC7E707B0BDE847
:102D7000F08F00BF18040020240400201604002057
:102D800014040020480C002050030020FE02002004
:102D9000F00C0020540C0020500C0020C81900201A
:102DA0000400FA0500ED00E0D80D002088020020A4
:102DB0005C2100201C020020020400202DE9F04FBD
:102DC000974B91B01B68BBB9964C2378013B042B01
:102DD00000F2F086DFE813F00B060B060B06DE06AA
:102DE000C406206803F091FC8F4B04461B681B78D7
:102DF0004BB1012B00F0ED80894C206803F08AFC78
:102E00000028EED1E0E72428884D0CD006D80A2807
:102E100000F08E800D2800F08B80C6E02A2806D0B6
:102E20002C2804D0C1E02B706B70AB70CEE06A78B8
:102E30002E782A4400217D4BD170EEB9DA789E7449
:102E4000472A19D11A79502A16D15A79472A07D117
:102E50009A79472A04D1DA79412A01D101229A7458
:102E60006A79724B522A07D19A794D2A04D1DA79BC
:102E7000432A04BF02229A74AB7C6C4F012B02D010
:102E8000022B36D049E0B31E072B46D8DFE803F00B
:102E9000040810141C27452C02F0A7F968613CE0D7
:102EA000EA78624B532A38D15A6952425A6134E067
:102EB00002F09BF9A86130E0EA785C4B572A2CD1EC
:102EC0009A6952429A6128E0EB78302B584B1A7875
:102ED0008CBF42F0020222F002021A701DE00020B4
:102EE00002F0DEF9287718E0002002F0D9F9E88333
:102EF00013E0072E06D0082E0FD1012002F0D0F9E2
:102F000078840AE0012002F0CBF941F218435843DB
:102F10004FF47A72B0FBF2F33B84013600232A2C83
:102F2000424A2E706B704CD1012182F824104DE082
:102F300095F82430002B34D03C4BDB78402B04D95F
:102F4000A3F137021201D2B202E01B0103F0F0023A
:102F50002B79A978402B8CBF373B303BDBB2134435
:102F6000DBB29942314A1BD1937C012B08D0022B52
:102F700016D1118C2F4B528C19802F4B1A800FE0D9
:102F80002B4909788E070CD52C4950690860906947
:102F90004860107F2A490870D18B2A4A118000E0CE
:102FA0000023002285F8242010E06B781F4A0E2BA6
:102FB00003D8591C13445170DC7095F824301B4A17
:102FC0001BB991784C40947000E0002303F001039A
:102FD00061E1164B002193F82520082A00F25A815E
:102FE000DFE802F00B0514324353718D9A0062281A
:102FF00001D1022207E083F82510B52C40F04A8168
:1030000093F82520013283F8252043E1032283F839
:10301000252083F8260083F8270083F8280039E16B
:10302000A0080020800800209C080020080E002036
:10303000FE02002014040020FC16002024040020BE
:103040001804002016040020042283F8252093F899
:10305000272093F828100244D2B283F827200A448C
:1030600083F8282083F8290014E1052283F825201D
:1030700093F8272093F828100244D2B283F827202F
:103080000A4483F82820588504E1062183F8251096
:1030900093F8271093F828002144C9B283F8271029
:1030A000014483F82810598D6C4A01EB0424A4B222
:1030B000B4F5007F89BF00215485518582F8251021
:1030C00000229A85E6E093F8272093F8281002441E
:1030D000D2B283F827200A4483F828209A8DC72A81
:1030E00003D85E49114481F83000013292B29A85CA
:1030F0005B8D934240F0CE800722584B83E7082235
:1031000083F8252093F82730834200F0C380534A88
:10311000002382F82530BEE083F8251093F82810AC
:103120004E4A814240F0B68092F82910062947D0D5
:1031300004D8022912D003292CD0ABE012295CD08C
:10314000302940F0A78092F83410454A102988BFF2
:10315000102111701078434900225CE04249506B05
:103160004860906B0860116C4FF47A7091FBF0F13D
:103170003E48018092F8F8103D4A19B1117841F0AB
:10318000020102E0117821F002011170012283F89E
:10319000F92055E092F8351011F0010105D092F8B0
:1031A0003420D41E6242624100E00A4683F8F820CF
:1031B000002A45D12E4A117821F0020111703FE01A
:1031C00092F83B1011F0010105D092F83A20D01E80
:1031D0004242424100E00A4683F8F82022B9244ADC
:1031E000117821F00201117093F85F10214A1170DB
:1031F000B3F85C10204A118022E0516C1F48018016
:10320000916C42F2107091FBF0F11D480180012198
:1032100082F8FA1014E0824201F10C0110DA11F880
:10322000045C184C155511F8035C174C155511F832
:10323000015C164C15550D78154C15550132EAE711
:1032400093F8F930054A2BB392F8FA3013B3002300
:1032500082F8F93082F8FA3001231CE0080E0020D1
:10326000FE160020380E0020240400201604002042
:10327000FE02002018040020820000201404002018
:10328000FC160020FF1600200F1700201F1700203B
:103290002F1700200023002B3FF4AEADA54BA64E08
:1032A0009A68DA6032689A60A44B1A6842F0200289
:1032B0001A60A34B1A78012A0CBF002201221A704F
:1032C000A04B1A7891077FF597AD9F49097804299B
:1032D0007FF692AD9D49097801F0040101F0FF00ED
:1032E00011B922F001021A701B78964F13F0010FEA
:1032F000974C984D11D180B19B070ED5964B2868FD
:103300006A6818605A6006F0D1FB944B1B88A4F8D9
:10331000FC303B7843F001033B7094F8FE304FF0F3
:103320000509013393FBF9F909EB8909C9EB030995
:103330008B4B8C481B7884F8FE900593831D03EB20
:10334000890907900023DFF80CE2874A53F80E0042
:10335000864F985090FBF7FC02F1080743F807C02E
:10336000834F03EB0E0107FB0C0742F2107097FB33
:10337000F0F00691079980B221F8020F02F1100ACD
:1033800003EB830B0490079153F80A0059F80B10D4
:1033900049F80B70C1EB000808EB0700734F4FF0C2
:1033A000050843F80A0090FBF8F007FB0C000599AC
:1033B000183201299850774608D1DDF810E0AEF1B7
:1033C0000202B2F5797F9CBF069908600433082B8E
:1033D000B9D1DFF87C813068D8F84C31C01A08F0D8
:1033E000C3FE644908F0CCFF33684FF07E51C8F843
:1033F0004C31814609F0AEF810B94FF07E5000E034
:1034000048460CAAC4F85001534B00920DAA0192F1
:1034100097E803000CCB06F007FB0C9B564964228F
:10342000B3FBF2F30D980B80544B90FBF2F21A8031
:10343000444A474E127812F0010208BF1A8098F8E9
:10344000543108BF0A80002B3AD0D6F850114FF003
:103450007E5008F095FFD6F8583181462868C01A8A
:1034600008F086FE494608F0D7FE09F09BF8D6F82A
:103470005C211FFA80FA68680FFA8AFA801A08F04D
:1034800077FE3F4B196808F0C7FE494608F0C4FEB6
:1034900009F088F8B6F9623100B2C218B6F96031A5
:1034A0000221534492FBF1F293FBF1F392B29BB2EF
:1034B000A6F86621A6F86431A6F86221A6F8603164
:1034C000012388F854312F4B79681B88386803F042
:1034D00030031F4E1F4DC8F85C11C8F85801002B6F
:1034E0003FF48AAC06F5B873009306F5BA730193FE
:1034F000D6F86821D6F86C3106F096FA6B68D6F8E3
:103500006C01C01A08F034FE1D4B196808F084FEE7
:1035100009F048F8D6F868312A68C6F87C019B1A89
:10352000C6F878310E4B1B78012B2DD0022B00F002
:10353000F58061E480080020C41900208802002082
:10354000F60D0020FE020020180400206C2100204F
:10355000080E002024040020480C0020180300203E
:10356000500C0020060F0020340F00208096980099
:10357000806967FF00007A44880400208A040020E4
:103580003000002050030020D6F89C41D6F890313E
:10359000D6F88021D6F8947104F100400593049286
:1035A000079708F0FFFF0746204608F0FBFF8C4B0B
:1035B000D6F850511B68D6F898618A4C0890069648
:1035C00009934FF0000ADFF83C9259F81A60A9F10C
:1035D000140230463AF8028008F0CAFD049908F057
:1035E0001BFE08F0DFFFC8EB000080B209F12809DC
:1035F0002AF809000FFA80F9484608F0B9FD059944
:1036000008F00AFE08F0CEFF1FFA80FB09EB060067
:1036100008F0AEFD079908F0FFFD294608F0FCFD13
:10362000216808F0F1FC08F0BDFFB84204DB089AFD
:103630009042A8BF104600E0384608F099FD20608F
:1036400008F0B0FF58441FFA80FB606808F13108A9
:10365000301A08F08DFD294608F092FE099B206182
:1036600002469878D4F80890039208F07DFD5E49F0
:1036700008F0D2FD01464FF07E5008F081FE294649
:1036800008F0C2FC0146284608F07AFE039A8446F8
:1036900049461046CDF80CC008F0B4FCDDF80CC06B
:1036A0000146604608F0B8FD0146484608F0ACFC0B
:1036B0001FFA88F8B8F1620F014620616660A060C9
:1036C0000ED9069808F0A8FD08F06CFF474AB0F53F
:1036D000FA6FA8BF4FF4FA609042B8BF104600E0FE
:1036E0000020834440F6B8320FFA8BFB9345A8BF05
:1036F00093463F4A0A219345B8BF934601FB0AF11E
:103700003C4A54F8140B2AF802B03B4A0AF1020A68
:10371000BAF1040F88503FF46FAB54E7304BD6F842
:1037200070911F68B6F8A451B7F808A04FEA590382
:103730009A4528BF9A462BB29A4502DC1FFA8AFAAC
:103740000BE02E49D6F8500108F066FD08F02AFF7C
:1037500028441FFA80FAA6F8A4A1D8F87451D8F822
:10376000A861AE1B304606F00FFA0028D8BF4042D1
:1037700041F293139842CCBF00200120002843D08F
:10378000304608F0F5FC1E4908F046FD0BF03CFC05
:103790000646484608F0E8FC0146304608F03CFD85
:1037A00008F000FF80B240F6B83203B29342A8BFDF
:1037B00013460F4AA8F8AC019342ACBFEB18AB1804
:1037C00048F6A042934203DDA3F50C43A03B04E07E
:1037D000002BBCBF03F50C43A033C8F8B03115E093
:1037E000D4030020840C0020DB0FC94030F8FFFF19
:1037F00048F4FFFFDC030020AC0C00200000C842AE
:10380000D3023739800F0020C8F8B051D4F8B02166
:10381000C2F50C502830049208F0AAFCAA4908F01E
:10382000FBFC05460BF07CFB0F9028460BF0ECFBF5
:10383000D4F8C051D4F8B431D4F8B8210E9005F1C1
:10384000004007930A9208F0ADFE0590284608F064
:10385000A9FED4F85081D4F8BC410B9009949B4C3C
:103860000025504608F084FC0EAB53F8151008F004
:10387000D3FCDFF894B206463BF9050008F078FC6B
:103880000146304608F0BEFB08F08CFE904B06B2B5
:10389000B6F57A7FA8BF4FF47A769E42B8BF1E462F
:1038A000B0B20BF13C0B25F80B0000B208F060FC45
:1038B0000799834608F0B0FC08F074FE80B20890C7
:1038C0000A99584608F0A8FC414608F0A5FC216872
:1038D00008F09AFB08F066FE059B984204DB0B9A01
:1038E0009042A8BF104600E0059808F041FC8346CE
:1038F000206060681434301A08F03AFC414608F041
:103900003FFD54F80C3C44F8040C0246B87806938A
:10391000039208F029FC6F4908F07EFC01464FF045
:103920007E5008F02DFD414608F06EFB01464046F2
:1039300008F026FD039A844606991046CDF80CC07F
:1039400008F060FBDDF80CC00146604608F064FC3E
:103950000146069808F058FB44F8106C014644F8FC
:10396000040C44F80C0C099808F056FC08F01AFEF8
:10397000089E0644584608F015FE304440F6B8321A
:1039800000B29042A8BF1046534A0A219042B8BFE5
:1039900010466943514AA852514A0235042D41F854
:1039A00002B07FF45EAF3B792BB1049B642293FBA2
:1039B000F2F24C4B1A803B884B4C99450ED9D4F807
:1039C000A831D4F87401C01A06F0DEF842F2107380
:1039D0000028B8BF404298427FF70EAA434B01220D
:1039E0001A70B4F8FC203F4B1A80FFF705BA404A22
:1039F000116890460F7817B1012F0DD0ADE0012B63
:103A000000F2AB8062783B4B03EB02133A4A5968F1
:103A1000106802F075FE9DE0374E306802F06BFED4
:103A2000B146002800F099802378344D022B29D02C
:103A3000032B31D0012B40F09080314B1F686B6914
:103A4000FB1A632B40F289802B69042B18D8DFF80E
:103A5000A480306808EB0313596802F051FE6B78BC
:103A6000366808EB03139D6815F8011B19B1304641
:103A700002F062FEF8E723696761013323616CE0BD
:103A8000022068E06A781B4B306803EB0213596828
:103A900002F036FE03205EE02B7E03B92F76227EF5
:103AA000164B012A36D11A697B2A2FD8D8F8003054
:103AB0009B782BB9134BD9F80000995C02F03CFEBF
:103AC00023690133236125E0D3023739AC0C002090
:103AD00018FCFFFFDB0FC94048F4FFFFDC030020A8
:103AE000840C0020DC0D0020080E0020500C00206B
:103AF0009C0800208C070108A008002080080020F6
:103B0000C4190020EC0D01086C0F002000221A617E
:103B100002221A76227E294B022A18D11A690F2A0C
:103B200013D8D8F80030997859B95B78244903EB59
:103B300003130B441A44D9F8000092F87D1002F0E8
:103B4000FBFD23690133236101E003221A76237E02
:103B5000022B02D9042007F023F90023636029E037
:103B60006368052201336360637801200133DBB2AF
:103B7000B3FBF2F202EB82029B1A6370114B00223C
:103B80001B68A360104B1A70104B1A7822F00202C7
:103B90001A700DE00B4B1A68A368D21A40F6C413D2
:103BA0009A4207D90A4B05201A6822F020021A60AF
:103BB00007F0F6F811B0BDE8F08F00BF80080020D4
:103BC000EC0D0108C419002018040020FE0200209A
:103BD000880200202DE9F04F064689B00F461546B1
:103BE0009B462978002900F0B880252902D00135AC
:103BF0003046B0E06C78302C03D002354FF000092D
:103C000003E0AC784FF001090335A4F13003092B30
:103C10004FF000081AD8A4F13003DAB2092A07D805
:103C20000A2B13DC0A2202FB083815F8014BF2E7D5
:103C3000A4F16103052B02D8A4F15703F0E7A4F126
:103C40004103052B02D8A4F13703E9E76C2C03BF2D
:103C50002C78012201350022632C66D006D8252C51
:103C600077D0582C3FD0002C77D0BAE7732C63D094
:103C700002D8642C11D0B4E7752C02D0782C32D045
:103C8000AFE70BF1040A05ACDBF800000A2112B122
:103C90000022234613E0234620E00BF1040A05AC82
:103CA000DBF8000072B1002806DA2D238DF81430FD
:103CB00040420DF1150300E023460A21002205F0E1
:103CC0007BFD0DE0002806DA2D238DF814304042EC
:103CD0000DF1150300E023460A21002205F044FD02
:103CE000D34600941AE00BF1040303930DF1140A78
:103CF000DBF80000102132B1583C62426241534669
:103D000005F05AFD06E0B4F158035A425A415346B1
:103D100005F02AFDDDF80CB0CDF800A0304639469C
:103D200042464B4605F084FD5BE730469BF80010A9
:103D30000BF10404B8470AE0DBF80030304600938A
:103D40003946424600230BF1040405F071FDA346F9
:103D500047E730462146B84743E709B0BDE8F08F52
:103D60000FB407B50A4904AB08680A4953F8042B95
:103D700009680193FFF72EFF074B186802F0BBFCA0
:103D80000028F9D003B05DF804EB04B0704700BF21
:103D9000A8050020A4050020F0170020F8B507466C
:103DA0000AF0D0FE044638B9194B1A485A791A4B12
:103DB000013A53F8221028E03846184922460AF002
:103DC000C9FE60B9164802F051FD164C54F8041FA4
:103DD00019B11548FFF7C4FFF8E7144805E00025BE
:103DE0000D4B53F8256026B91148BDE8F84002F0A4
:103DF0003DBD3846314622460AF0ACFE013500286A
:103E0000EED1034B0B485D713146BDE8F840A7E7A2
:103E1000C81900209F1F0108DC1101083226010883
:103E2000B31F0108D8110108C61F0108B8270108EF
:103E3000CA1F0108DF1F010870B504460AF082FEA0
:103E400008B91E482EE020461D490AF0F5FE002460
:103E50002646254678B12CB1012C06D10AF0C7FEC2
:103E6000064602E00AF0C3FE05461549002001346B
:103E70000AF0E2FEEEE70B2D04D9BDE870401148D0
:103E80000C216DE7012C07DC0F4B294633F9152077
:103E90000E48BDE8704063E7A6F57A73B3F57A7F04
:103EA00003D90B48BDE870405AE70A482946324614
:103EB000FFF756FF044B23F8156070BDF11F010892
:103EC000462401082B200108DE0D002051200108A6
:103ED000692001088B2001082DE9F74304460AF008
:103EE00031FEC0B290B9304C054694F8D711B4F801
:103EF000D42194F8D6312D48009129460135FFF799
:103F00002FFF102D04F10404EFD14AE020460AF0FF
:103F10006EFE0F28054636DC204620210AF005FEFD
:103F2000234FEDB2D7F80090441CAD000026204688
:103F30000AF05DFE5FFA86F8B8F1010F83B208D08F
:103F4000B8F1020F0BD0B3F5B47F1ED23A685353C9
:103F50000AE0FF2B19D83B682B44987004E0FF2B34
:103F600013D83B682B44D87020462C210AF0DDFD85
:103F7000044608B1441C02E0B8F1020F05D1013635
:103F8000032ED4D10DE00B4806E009EB050000211B
:103F900004220AF096FD0848102103B0BDE8F04362
:103FA000DEE603B0BDE8F083C8190020A4200108B4
:103FB000A4080020B8200108DC200108124870B5D0
:103FC000002304781A46D1B28C4209D0057B8D4279
:103FD00008D00D4D2D7E8D4208BF02210ED102E08A
:103FE000002100E001210C2505FB0101074D084ED1
:103FF0001D4495F82C510133755D0D720132032A71
:1040000001D0022BDFD970BD48000020C819002064
:104010008722010870B50546441E14F8011F61B1DE
:10402000064E30460AF081FD0028F6D0861B044873
:10403000631B304480F81031EFE770BD0D2A010892
:10404000C819002030B587B005460C4603A80021EA
:104050000C220AF036FD2846002108F099FA20B11A
:1040600028462A4907F0D0FF03E02846274907F0F1
:10407000C9FF274908F0D0F808F094FA054685EA08
:10408000E570A0EBE57069460A2205F0BDFB002350
:104090009D420370ACBF20232D2368468DF80C3061
:1040A0000AF050FD012807D130238DF80D308DF82E
:1040B0000E308DF80F300CE0022805D130238DF83A
:1040C0000D308DF80E3004E0032804BF30238DF846
:1040D0000D30694603A80AF01BFD03A80AF032FD63
:1040E0000338C5B22A4603A920460AF055FD00232D
:1040F0006355204607490AF00BFD03A920462944D1
:104100000AF006FD204607B030BD00BF6F12033A2B
:1041100000007A44EA2001082DE9F04389B0044602
:104120000AF010FDC6B2002E6CD18B4802F09EFB47
:104130008A4C2069002108F003FA40BB0136884808
:104140003146FFF70DFE206904A9FFF77BFF01460A
:104150008448FFF705FE606904A9FFF773FF014675
:104160008048FFF7FDFDA06904A9FFF76BFF01463A
:104170007C48FFF7F5FDE06904A9FFF763FF0146FE
:104180007948FFF7EDFD0C2E04F11004D1D1002584
:10419000764C2F462B464FF00008B04504F1100432
:1041A00015DA184654F8101C07F02EFF54F80C1CB2
:1041B0008146284607F028FF54F8081C0546384673
:1041C00007F022FF08F101084B460746E5E768487B
:1041D00001930295039702F049FB002401ABE058DC
:1041E000644920F0004008F0D3F9634B634A04347B
:1041F000002814BF1046184602F038FB0C2CEDD1F5
:104200005F4891E020465F4905220AF0A3FC38B9D7
:10421000524B002203441030C0281A61F8D197E0B5
:104220002046594904220AF095FC06462046002EF5
:1042300040D120210AF079FC002800F08980451C3B
:1042400028460AF07FFC34468046504B53F82460E1
:104250000EB94F4868E0284631465FFA88F20AF006
:1042600079FC671C20BB3D4B0021C2181030C028D0
:1042700011619C46F7D1474B002403EBC702D2F8EB
:1042800004E09846BEF1000F04D143483146FFF7E1
:1042900067FD55E018F837309C42F6DA23010CEB45
:1042A0000305103573440FCB013485E80F00F1E7A7
:1042B0003C46CAE70AF09BFC461E0B2E074643DC31
:1042C000204620210AF031FC054640B1451C284615
:1042D00005F0B5F9214B3F01D851012400E0044617
:1042E000284620210AF021FC054640B1451C2846FD
:1042F00005F0A5F9194B013403EB06135861284664
:1043000020210AF012FC054640B1451C284605F064
:1043100096F9124B013403EB0613986128462021CD
:104320000AF003FC18B91D4802F0A0FA10E00130B1
:1043300005F085F9094B032C03EB0616F061F2D169
:104340001748FFF7E9FE03E016480C21FFF708FDC8
:1043500009B0BDE8F08300BFF4200108C8190020AF
:104360001F2101082521010841220108DC19002034
:10437000292101080AD7233CF0200108EC2001087C
:10438000B8270108382101083E210108DC11010885
:10439000CA1F01089C060108432101085321010896
:1043A000772401088D2101080A88F0B54B888F8891
:1043B0000E89CD88002A3AD1048C834A24F0010466
:1043C0002404240C0484018B048C89B221F0F301B1
:1043D00041EA0616B6B29042A4B246EA070743F095
:1043E000010315D002F50062904211D0B0F1804F68
:1043F0000ED0A2F5983290420AD002F58062904227
:1044000006D002F58062904218BF24F00A0401D160
:1044100024F00204234307830384038B23F00C035B
:104420001B041B0C0383038B9BB21D4344E0042A33
:1044300044D1048C644A24F010042404240C048421
:10444000018B048C21F440710905090D41EA063104
:1044500089B241EA07279042A4B2BFB212D002F556
:10446000006290420ED0B0F1804F0BD0A2F598328E
:10447000904207D002F58062904203D002F580623C
:10448000904207D124F0200444EA03139BB243F086
:10449000100304E024F0A00443F010032343078337
:1044A0000384038B23F440631B041B0C0383038BE3
:1044B0009BB243EA0525ADB20583F0BD082A018C05
:1044C0003ED121F480710904090C0184818B3E4A9C
:1044D00089B221F0F301048C41EA0616B6B290428B
:1044E000A4B246EA070712D002F5006290420ED04D
:1044F000B0F1804F0BD0A2F59832904207D002F570
:104500008062904203D002F58062904207D124F489
:10451000007444EA03239BB243F4807304E024F460
:10452000206443F48073234387830384838B23F0C5
:104530000C031B041B0C8383838B9BB21D4341E044
:1045400021F480510904090C0184828B048C22F42B
:1045500040721205120D42EA072242EA06361A4A52
:10456000A4B29042B6B212D002F5006290420ED0D0
:10457000B0F1804F0BD0A2F59832904207D002F5EF
:104580008062904203D002F58062904207D124F409
:10459000005242EA033292B242F4805205E047F6FA
:1045A000FF52224043F480531A4386830284838B54
:1045B00023F440631B041B0C8383838B9BB243EA6D
:1045C0000525ADB28583F0BD002C01401FB5012348
:1045D000ADF808300023ADF80C30ADF80A30094BC7
:1045E000ADF804101B7801A9012B08BF0323ADF817
:1045F000062008BFADF80C30FFF7D6FE05B05DF819
:1046000004FB00BF0C06002038B510F80E2C044641
:1046100050F8043C52B9012200F80E2C20F80C1C72
:10462000197B18680222BDE83840CFE730F80C2C1F
:1046300020F80A1C891A89B220F8081C074A10F8C9
:104640000F0C002522F8101004F80E5C1868197B76
:104650002A46FFF7BBFF04F8065C38BDCC0F0020EC
:104660001F4B10B55A6802F00C02042A03D0082A26
:1046700004D01C4A14E01C4A126811E05A685968B8
:10468000C2F38342C90302F1020201D4174906E0D2
:10469000596811F4003F1449096818BF49084A4392
:1046A00002605968124AC1F30311545C0168E14089
:1046B00041605C68C4F30224145D21FA04F4846050
:1046C0005C68C4F3C224145DE140C1605B68C3F35D
:1046D00081331A44137CB1FBF3F1016110BD00BFBB
:1046E0000010024000127A001400002000093D0072
:1046F00034000020CB78F0B5DA0648BF8A78098804
:1047000003F00F0548BF154311F0FF0F1DD00468DB
:1047100000220127974007EA0106BE4211D1970007
:104720004FF00F0C0CFA07FC05FA07F724EA0C040B
:10473000282B44EA070401D1466102E0482B08BF58
:1047400006610132082AE4D10460FF291FD94468B8
:10475000002202F108060127B74007EA0106BE421F
:1047600011D197004FF00F0C0CFA07FC05FA07F770
:1047700024EA0C04282B44EA070401D1466102E034
:10478000482B08BF06610132082AE2D14460F0BD1F
:1047900010B5044601F047FC012806D11CB101F018
:1047A00042FC013CF8E7052010BD002C08BF0520A5
:1047B00010BD00BF07B5064B06480093064B074ADD
:1047C0001968074BFFF7CCFA03B05DF804FB00BF94
:1047D000E6210108B521010888000020D121010847
:1047E000DD2101080EB40FB5074906AB0190074A59
:1047F00001A80393FFF7EEF9019B00221A7004B0A1
:104800005DF804EB03B07047FD930008EE2101084A
:104810002DE9F0438DB005460AF094F9C0B20028A6
:1048200058D104467F4B00211E68142207A80AF0C5
:1048300048F9A500002303A905A803930593771958
:104840000B7183801A46DFF8F0E1B7F802C03EF83A
:10485000138018EA0C0F0CD00EF10A0E0DF130087F
:1048600013F80EE002F1010C424402F824EC5FFA66
:104870008CF20133052BE6D100231A46DFF8C0E1A4
:10488000B7F802C013F80E8018EA0C0F0CD00EF126
:10489000060E0DF1300813F80EE002F1010C42444F
:1048A00002F81CEC5FFA8CF20133062BE6D1735D43
:1048B0008DE803001A0907A85B4903F00F03FFF70F
:1048C00091FF2146594807AA0134FFF749FA202CE5
:1048D000A8D1A3E028460AF08AF91F28044600F36D
:1048E000918028462021E4B20AF01FF91F2C01D93B
:1048F0004F4888E04B4B471C1B68002103EB8404A6
:10490000204604220AF0DDF800254A4B07AE304667
:1049100000210A2215F803905FFA85F80AF0D1F811
:104920000023FA5CF91832B10A2B04D04A4502D0B0
:10493000F2540133F5E74A4501F1010767D1B8F1B7
:10494000020F0DD0B8F1030F0CD0B8F1010F0BD04E
:1049500030460AF04CF92378C0B243EA00100AE06E
:10496000002219E0002226E030460AF040F92378C0
:1049700000F00F001843207038E00133062B0AD0F6
:104980002D4800F115069E5D8E42F6D10344D97B79
:1049900063880B43638001320CA9D3B20B4413F834
:1049A000141C19B30023EBE7412B1DD0542B08BF77
:1049B00004230ED00132D3B20DF13008434413F872
:1049C000143C9BB1492B01D1002302E0572B07D1A6
:1049D0000123194931F8131063880B436380E9E719
:1049E000462BE1D10223F4E70323F2E70135042D3E
:1049F0008BD1012404F0B4FF04F0EEFF04F0C8FFF3
:104A000064B975E70D482021FFF7AAF906E02046B2
:104A1000002104220AF055F80024EBE70DB0BDE8B0
:104A2000F08300BFDC040020EE210108FA21010818
:104A3000DC200108D90E0108BE0E0108062201087B
:104A4000CD0E010810B5074801F010FF0024064BF9
:104A50000648E218E15852680C34FFF781F9FC2C43
:104A6000F5D110BD28220108041001083E220108DA
:104A70007FB504460AF066F8082824D100231F49B0
:104A8000E25C09681144497801F00301022908BF7A
:104A9000203AE2540133082BF1D10025665D184815
:104AA00031460AF042F828B10135601931460AF062
:104AB0003CF818B1134801F0D9FE1CE0082DEDD1E7
:104AC0002046FFF7A7FA104801F0D0FE00230F4A56
:104AD00004A91A4492F810210A440949595C013387
:104AE000082B02F80C1CF2D10023094801A98DF80B
:104AF0000C30FFF735F904B070BD00BF9000002006
:104B00000D2A01084622010866220108C819002062
:104B10004122010837B582880446836810060D4695
:104B200006D529494FF4E07091F8541700FB013382
:104B3000D10504D525490A20097800FB013302F08C
:104B40003F02042A12D006D8012A0DD0022A2FD102
:104B500093F900102DE0102A0AD0202A0AD0082A42
:104B600026D1B3F9001024E0197822E0198820E05A
:104B700019681EE069461868FFF764FA0146144890
:104B8000FFF7EEF8F5B1E06807F0F2FA6946FFF7D3
:104B900059FA01460F48FFF7E3F8206907F0E8FAF1
:104BA0006946FFF74FFA01460A48FFF7D9F809E0CE
:104BB00000210948FFF7D4F825B10848E1682269C7
:104BC000FFF7CEF803B030BDC81900203C0C002020
:104BD000202701081F2701087F2201087B220108E6
:104BE0004B8810B5DC0607D52C4B14791B6853F89D
:104BF00024402B4B43F820404B889B0607D5274B7E
:104C000054791B6853F82440254B43F820404B88C7
:104C10001C070DD5234B0C781B78B3EB141F07DB57
:104C20001E4BD4781B6853F824401D4B43F820409A
:104C30004B889B070DD51C4B0C781B78B3EB141FCE
:104C400007DC164B54781B6853F82440144B43F888
:104C500020404B88DC070ED5144B0C781B7804F0F1
:104C60000F049C4207DC0D4B14781B6853F824405A
:104C70000B4B43F820404B885B070ED50C4B097853
:104C80001B7801F00F01994207DB044B92781B68F7
:104C900053F82220024B43F8202010BDA408002026
:104CA000E0040020970500209505002094050020D1
:104CB0009605002010B5174B1A78511C197016492B
:104CC00002F007024878154903EB420331F810104F
:104CD000598000231846124A9A5A02331044102B66
:104CE00080B2F8D1C00807F043FA0E4907F094FAF1
:104CF0000D4907F045FB0D4B04461B68187807F07B
:104D000037FA0146204607F087FA07F071FC084B96
:104D1000187010BDE40F0020C0050020D005002051
:104D2000E60F00203333534000F07F450404002099
:104D30000804002070B5046D4279A38902F00401D3
:104D400023F400531B041B0C0546866886B0A38120
:104D500001F0FF0021B14FF480604FF4005100E0FA
:104D6000014612F0010F14BF0423002312F0020FBA
:104D70001CBF43F008039BB212F0080F228A18BF31
:104D80000C2392B222F4405211432182A28992B2A2
:104D900022F4B05222F00C02104303439BB2A381D1
:104DA000A38A01A823F440731B041B0CA382FFF702
:104DB00057FC1949049A039B8C4208BF1346A289E9
:104DC0001921594312B2002AB4BF7600B600B1FBD4
:104DD000F6F16423B1FBF3F21201100903FB101189
:104DE000A08900B2002806DAC9003231B1FBF3F322
:104DF00003F0070305E009013231B1FBF3F303F0DF
:104E00000F031A4392B22B6D22819A8992B242F417
:104E100000529A8106B070BD00380140417189E7A7
:104E2000816087E70368F0B52E4D9C0AAC4257D0ED
:104E300003D8B4F5801F51D0F0BD2B4DAC4203D048
:104E40004935AC4202D0F0BD032400E00024057BCC
:104E5000AD08AEB241B94FF0020C0CFA05F59F89CE
:104E6000BFB227EA05059D81204D04EBC4073E44EF
:104E700045F82610043645F8262041B1027B022071
:104E8000920800FA02F299890A4392B29A81242286
:104E900002FB045404F12001EFF31286502282F346
:104EA00012880022A018056915B10D60016904314E
:104EB0000432102AF6D100220A60F2B282F311887D
:104EC000226A22B19A8992B242F0010204E09A89E0
:104ED00022F001021204120C9A81F0BD0124B6E7FF
:104EE0000224B4E70100100002001000881800201E
:104EF000826A8169436B1144D960416A914203D946
:104F00008A1A5A60816204E001698A1A5A60002292
:104F10008262002280F844201A6842F001021A607E
:104F200070472DE9F04F634C63696349581C0A7858
:104F3000894602F0FF0C0AB10346F6E7277F667F39
:104F4000A57F216A6361E0461FFA88F213B21F2B26
:104F500000F39380594901EB8300C278807831F8DF
:104F60002310C0F1FF0080B2002861D0C0F1FF0023
:104F700050433C23B1FBF3FA0012BAF1050F5AD8A3
:104F8000DFE80AF0030B1A283846161A4E43C5B25A
:104F9000B6FBF3F62E44F6B248E0B1FBF3F703FBA1
:104FA0001717BFB2C5B2C7F13C07101A4743B7FB8A
:104FB000F3F72F44164629E0B1FBF3F503FB151573
:104FC000C7B2ADB2101A4543B5FBF3F53D44EDB29F
:104FD000164630E0B1FBF3F603FB1616B6B2C7B2C5
:104FE000C6F13C06101A4643B6FBF3F63E4415469E
:104FF000F6B220E0B1FBF3F703FB1717C6B2BFB25E
:10500000101A4743B7FBF3F737441546FFB212E0D7
:10501000B1FBF3F503FB1515ADB2C6B2C5F13C0506
:10502000101A4543B5FBF3F53544EDB2174602E0DF
:105030001546164617464FEA072A4AEA064A4AEA3A
:10504000050A1723012199400CF1170211EA0A0FF2
:10505000C3EB02021A490CBF0920112092B213F1CE
:10506000FF338854EED20CF1180C08F101081FFA36
:105070008CFC1FFA88F8134966E7012389F8003091
:10508000114B628340F22A3227776677A577216237
:10509000A4F818C05A600D4A00219184118889B281
:1050A00041F0010111801A6842F001021A60BDE866
:1050B000F08F00BFE40F00206A210020E0040020F0
:1050C000A8080020001000206C00024000040040EE
:1050D0000D4B10B5DC680122E443C4F30224C4F193
:1050E000040402FA04F40178A3F54063240119448E
:1050F000E4B281F800430178480901F01F018A40B9
:1051000043F8202010BD00BF00ED00E0254B10B596
:105110005343254A254C12680139B2FBF3F2038848
:10512000013AA04289B292B29BB212D004F5006457
:10513000A0420ED0B0F1804F0BD0A4F59834A0421D
:1051400007D004F58064A04203D004F58064A04237
:1051500002D123F070039BB2154CA04206D004F597
:105160008064A0421CBF23F440739BB203800F4BAA
:105170008185984202850FD003F5006398420BD0D9
:1051800003F54063984207D003F58063984203D04B
:1051900003F58063984201D10023038601238382B3
:1051A00010BD00BF40420F0084000020002C0140D1
:1051B0000010004013B504460068FFF7A7FF2368FE
:1051C00001A81A8892B242F001021A80637B002281
:1051D0008DF8043001238DF805308DF806208DF808
:1051E0000730FFF775FF02B010BD294BF0B51D6801
:1051F00000222848165C1418AB19597801F00401F4
:1052000001F0FF0371B10132102AF2D10020F0BD8C
:105210001BB103EB83035B00DBB210F8012B303AC8
:105220001344DBB2221A022AF2DC002184420AD99A
:1052300019B101EB81014900C9B210F8012B303AD4
:105240001144C9B2F2E72E2E14D1601C00220424AE
:10525000067802EB8202AF197F7852007F0792B284
:1052600003D5303A3244013092B2013C14F0FF04CD
:10527000EED100E00022084806244143642000FBF0
:1052800002120648B2FBF4F200FB0320F0BD00BF9F
:10529000900000200B0E002040420F0080969800E6
:1052A00030B5002213460D495C5C9CB12E2C04D114
:1052B000013378B11C1800250D550A246243C95CDE
:1052C000A1F13004092C9CBF303A52180E2B03D8A0
:1052D0000133E8E7104630BD002030BD0B0E002042
:1052E00008B540F2E9330D4A1189890709D5908143
:1052F00040F2E933094A1189C9070AD59089C0B239
:1053000008BD013B9BB2002BEDD104F0F2FCFF2065
:1053100008BD013B9BB2002BECD1F6E70030014009
:105320002DE9F74F9F4E9B4633780C4691465A1C09
:10533000054606F8042B0068224649460C275F43C1
:10534000FFF7E4FEAB686868ADF8043018238DF809
:10535000063001A902238DF8073004F091FC2B7B65
:1053600006EB070A2C680C2B00F2F280DFE813F042
:105370000D00F000F000F0004D00F000F000F00033
:105380008200F000F000F000B600238C864823F085
:1053900001031B041B0C2384218CA288238B8442D1
:1053A00023F073034FEA03434FEA134389B292B2E7
:1053B00043F0700314D000F50060844210D000F573
:1053C000406084420CD000F58060844208D000F533
:1053D0008060844204D021F0020141F0030107E023
:1053E00021F00E0122F4407241F0030142F4807278
:1053F000A2802383A4F834B02184238B23F00803F4
:105400001B041B0C43F0080332E0238C664823F096
:1054100010031B041B0C2384218CA288238B844241
:1054200023F4E6434FEA03434FEA134389B292B2AF
:1054300043F4E04308D000F50060844204D021F03A
:10544000200141F0300107E021F0E00122F4406248
:1054500041F0300142F48062A2802383A4F838B086
:105460002184238B23F400631B041B0C43F400638F
:1054700023836DE0238C4C4823F480731B041B0CA6
:105480002384218CA288A38B844223F073034FEAE8
:1054900003434FEA134389B292B243F0700308D03A
:1054A00000F50060844204D021F4007141F44071A1
:1054B00007E021F4606122F4405241F4407142F46B
:1054C0008052A280A383A4F83CB02184A38B23F054
:1054D00008031B041B0C43F0080338E0B4F820C099
:1054E000314A2CF4805C4FEA0C4C4FEA1C4CA4F877
:1054F00020C0B4F820C0A388B4F81C802CF4005C51
:1055000028F4E6484FEA08484FEA0C4C4FEA18489E
:105510004FEA1C4C94429BB248F4E0484CF4405C87
:1055200003D002F50062944203D123F4804343F494
:105530008043A380A4F81C80A4F840B0A4F820C045
:10554000A38B23F400631B041B0C43F40063A383AD
:10555000AB7B43B1B4F844306FEA43436FEA534343
:105560009BB2A4F8443023889BB243F0010323800C
:105570002B7B0C2B10D8DFE803F0070F0F0F090F60
:105580000F0F0B0F0F0F0D00343404E0383402E01E
:105590003C3400E04034F4515046AAF8049003B083
:1055A000BDE8F08F08100020002C0140434A2DE98F
:1055B000F84F916840F201130B4040F201118B4209
:1055C00093460CD13E4B93F8942093F8959083F832
:1055D0009520B9EB020918BF4FF0010901E04FF027
:1055E00001094FF00008374B5FFA88F41B78A3429B
:1055F00061D9354B354E1B68354F23B93B685B8904
:1056000026F8143054E03A68072C94BF12F804A02E
:10561000A2462C4851469847DBF808300546DB0582
:1056200009D5B9F1000F06D02A4B50461B68294610
:105630001B68DB699847A5F2EE2240F2DC5392B278
:105640009A4288BF3B68DBF8082088BF5D8942F238
:105650000103134053B3204B1978194B01F0030297
:1056600002EB840293F8F60003EB4202A2F8965094
:105670001A4620B9032919D9012183F8F61002EB43
:10568000C403B3F89810B3F8965002EB44020D44EB
:10569000B3F89A10B3F89C300D441D44ADB2A2F893
:1056A000F85004232DB295FBF3F5ADB226F8145053
:1056B00008F1010897E7BDE8F88F00BFC81900207E
:1056C00008100020630800206C08002062050020FC
:1056D0000401002008020020E40B00202DE9F04125
:1056E0001E4C137CA46804F0400C022B32D80C260C
:1056F0005E431B4C03F1010835192F7A384226D03E
:10570000335D2BB1012B03D0022B14BF03230223E3
:10571000144F1E01BC19BCF1000F02D1BE5D022E58
:1057200015D04E7B277B3740B74210D14F68666853
:10573000B7420CD38F68A668B74208D8137094603C
:105740005560D16082F810801046BDE8F0815FFAA4
:1057500088F3CAE70020BDE8F08100BFC819002027
:1057600048000020E00E0108094B30B59D68094B48
:1057700005F480551868084B1C6800230DB1828819
:1057800000E0A28805495A520233182BF6D130BDE9
:10579000C81900205418002058180020DE0D0020E1
:1057A0002DE9F04FAF4E85B03778032F14D9AE4BAB
:1057B000AE48B3F90410B0F904200029B8BF49423B
:1057C0006FF063035B1A9A4204DB01F164039342B6
:1057D000A8BF134683801FE0012F1DD8A44BA54C02
:1057E0001B78013B142B00F2E381DFE813F09100FA
:1057F000E101E10168009F00E101E1013101E10106
:10580000E101E101E101E101BD00E101E101E101AD
:10581000E101E101A301BA01934B9749B3F806A056
:10582000924B0968B3F80280B3F80090B3F904B062
:10583000924C02910025BD4204F11004CED20FFA21
:105840008AF006F095FC54F8101C06F0E5FC0346BF
:105850000FFA88F0019306F08BFC54F8081C06F050
:10586000DBFC019B0146184606F0CEFB03460FFA0F
:1058700089F0019306F07CFC54F80C1C06F0CCFC7B
:10588000019B0146184606F0BFFB029A034692F9B7
:105890000000019340420BFB00F006F069FC54F855
:1058A000041C06F0B9FC019B0146184606F0ACFB4F
:1058B00006F078FE724B23F815000135BBE7022194
:1058C000042001F057F8694D0121AF8878431FFA91
:1058D00080F8042001F04EF86D8800FB05801FFA67
:1058E00080F8042001F054F8404420810221052072
:1058F00001F040F87843012187B2052001F03AF821
:1059000000FB057087B2052001F042F838440BE037
:105910000520012101F02EF8544B9D88684385B283
:10592000052001F035F82844608141E1554B002005
:105930001D6801F02DF8DFF8688195F90630B8F997
:1059400002203227534393FBF7F3184420800120B1
:1059500001F01EF895F90E30B8F90020534393FB7F
:10596000F7F73844608023E1474B1B7813F0040FAE
:10597000464B02D11B689B880BE019683A4A0B889A
:10598000B2F9062049889A4203DB9142B4BF0B4624
:105990001346E381E2893A4B3A4F1A803C4B1B682D
:1059A0001D7855B3022000F0F3FF3A68B2F91030C9
:1059B000518A984203DB0BB29842B8BF034635497F
:1059C00009684889C3EB000E334B0FFA8EFEB3F81B
:1059D00010110FFA81FCF44501DA0D4401E002DDFB
:1059E0004D1BA3F8105192F91620B3F9103153430F
:1059F000642293FBF2F31844A080284B1B88DB053C
:105A00000CD5194B1A88D7F80090E28022819A8829
:105A1000184F62815B880325A38101E0134BF1E7F6
:105A200009EBC50393F90630B7F90680284608FB51
:105A300003F8642398FBF3F8A7F8068000F0A8FFAA
:105A400001354044072DF88007F10207E8D1AFE0A7
:105A50000D4B1B7813F0040F0C4B23D11B689B8854
:105A60002CE000BF40210020C6030020A817002022
:105A7000E80300206C000020EC03002088070020D1
:105A800042210020501800206C21002058180020CE
:105A90005C1800206018002008100020500300202F
:105AA000080300201968AD4A0B88B2F9062049881E
:105AB0009A4203DB9142B4BF0B461346E381E2896D
:105AC000A74BA84D1A80A84B03201B880121DF0596
:105AD00003D500F04FFFA14F02E000F04BFFA34FB2
:105AE000B7F80280022100FB08F01FFA80F90320BA
:105AF00000F040FF3F88012100FB0790E880042070
:105B000000F038FF00FB08F002211FFA80F80420A3
:105B100000F030FF00FB07802881032000F038FFF1
:105B2000E3881844E080042000F032FF2389184401
:105B300020813DE00121042000F01CFF8B4D6F8887
:105B4000784387B20420278100F022FF3844208167
:105B50000121052000F00EFF2D88684385B2658184
:105B6000DEE6824B0325B3F80490984628460221CE
:105B700000F000FF00FB09F0012187B2284600F089
:105B8000F9FEC5F106035B0838F8133000FB03701B
:105B900087B224F81570284600F0FAFE384424F83D
:105BA00015000135072DE1D16C4BDA886C4B1A805A
:105BB0006F4DDFF8E491AB6813F0200F34D0002074
:105BC00000F0E6FE20808046012000F0E1FE694BF7
:105BD000644F1B6860801A0626D5674B1B681B78CC
:105BE00013F0020F654B23D0D9F800C0B3F90010B1
:105BF0009CF90E209CF906C0B3F902304A43CCF15F
:105C0000000C03FB0CF3322192FBF1F26FF0310C2C
:105C100092B293FBFCFC9444E04493FBF1F1A7F8AF
:105C200000800A4410447880D9F80010002319E05D
:105C3000D9F80010B3F902C091F90620B3F9003089
:105C40000CFB02FC32229CFBF2FCE044A7F8008033
:105C500091F90E104B4393FBF2F2E3E7E252023369
:105C6000102B0CD0E05E31F9232001EB830790422A
:105C70007F88F3DB3AB28242A8BF0246EEE73E4B92
:105C80001B681B785B0704D43549347808880123E6
:105C90001BE03B4B00241F780423043FFFB25FFA54
:105CA00087F84FFA88F2D4420BD4364A03F101093F
:105CB000381932F813105FFA89F9C0B203F0D5FF32
:105CC0004B460134042CECD1DEE7A34208D231F973
:105CD000132000B28242A8BF104680B20133F4E71D
:105CE000294B4FEA44081A68AB6803F480550395C2
:105CF000244D03F01009254BB5F90660244D1B789F
:105D00002F68244D03F00403DBB2D5F800C00293E2
:105D10000023434562D0B2F802A004B2544505DD29
:105D20000F4CC0EB0A0A1D5B55441D53039D0C4CE0
:105D3000002D33D07D8931F903A0AE42CBBFBCF832
:105D400002509588B2F802B0BCF800B0AA4503DB57
:105D5000DA45B4BF55465D46E55238E0C60300203B
:105D6000422100206C00002050030020A8170020D2
:105D7000C81900204C0300206418002008030020EC
:105D80000F06002062050020581800206C2100201A
:105D900060180020541800205018002031F903A08A
:105DA0001588B2F802B0AA4503DBDA45B4BF554600
:105DB0005D46E55204EB030ABC89A64207DAB9F155
:105DC000000F01D1148800E09488AAF80040029CDA
:105DD00014B9044C1C5BCC5202339AE705B0BDE801
:105DE000F08F00BFDE0D00201E4B2DE9F0431A7826
:105DF0001D460AB31C4B07781E781C4B93F800C055
:105E000002231B4A03F10108D45C344104F00F045F
:105E1000BC420CD20B2C0AD812F8039012F808805E
:105E200002EB840209EA0C0408EB04241461023337
:105E3000102BE6D100232B7003788B420FD90C4B2B
:105E400093F8400060B10B4A890012780B4418693E
:105E500002B1400800F5777080B2BDE8F083002001
:105E6000BDE8F083080100206008002061080020E0
:105E70001C1100206208002007299ABF024B33F84A
:105E800021000020704700BFE4010020024B53F8BE
:105E90002100C0F3CF0070478C01002008B5074BEC
:105EA00053F8210006F060F9054906F0B5F90549F7
:105EB00006F0AAF806F09CFB80B208BD2401002081
:105EC0000000203F00005C44014B33F81100704794
:105ED00062050020014B33F811007047CC0F002001
:105EE000034B4FF4004208B11A6170475A61704782
:105EF00000080140034B4FF4004208B15A6170475B
:105F00001A61704700080140032810B5114B0FD8E3
:105F1000114A126894888C420AD2D2888A4207D9E0
:105F2000012202FA00F093F84120104383F8410067
:105F300093F841300F2B0CD1064B002283F84120FF
:105F4000064B998808B2142802DD1439998010BDD7
:105F50009A8010BD1C110020C01900204C080020A0
:105F6000024B9A8801329A80704700BF4C0800208B
:105F7000074B1A68074B1178B3F9040053780B44A8
:105F800003EB83039842D4BF00200120704700BF79
:105F9000C01900204C080020064BB3F90400064B42
:105FA0001B681B7803EB83039842D4BF00200120B9
:105FB000704700BF4C080020C019002010B50446EF
:105FC000FFF7EAFF002814BF2046002000F0010080
:105FD00010BD024B01221A72704700BF4C0800200E
:105FE000014B187A704700BF4C080020034BB3F9EF
:105FF0000400D0F1010038BF002070474C08002099
:10600000014B00229A8070474C08002038B50C687C
:106010000546204608F096FD214602462868BDE860
:10602000384008F097BD094BDA68D10709D4DA681F
:10603000520708D4DB6813F0100F0CBF04200320B4
:106040007047012070470220704700BF00200240C7
:106050008A6810B50C6A036814430A6923F4FF4385
:1060600014434A6923F0700314438A691443CA69CC
:1060700014434A6A14438A6A224313430360CB6879
:1060800043600B6883604B68C36010BD02684FF6C5
:10609000FE73134003600023036043608360C360AA
:1060A0002A4B984222D02A4B984229D0294B984219
:1060B00030D0294B984237D0284B98423ED0284BBD
:1060C000984206D153F8682C42F4700243F8682CC9
:1060D0007047244B984206D153F87C2C42F07062F2
:1060E00043F87C2C7047204B984206D153F8042C7F
:1060F00042F00F0243F8042C70471C4B984206D123
:1061000053F8182C42F0F00243F8182C7047184B43
:10611000984206D153F82C2C42F4706243F82C2C90
:106120007047144B984206D153F8402C42F4704209
:1061300043F8402C7047104B984205D153F8542C2B
:1061400042F4702243F8542C704700BF080002400C
:106150001C0002403000024044000240580002404F
:106160006C00024080000240080402401C0402400F
:106170003004024044040240580402402DE9F84330
:10618000574B0C460168013AC3F842108188A3F8C6
:106190004610072A42D8DFE802F0040A1018222924
:1061A0002F35B3F842202280B3F8442013E0B3F82F
:1061B00044202280B3F8422005E0B3F84220524246
:1061C0002280B3F84420524205E0B3F84420524202
:1061D0002280B3F842206280B3F846301DE0B3F865
:1061E000422052422280B3F8442012E0B3F8442007
:1061F0002280B3F842200CE0B3F842202280B3F8AA
:10620000442005E0B3F8442052422280B3F84220F3
:1062100052426280B3F846305B42A380314B1B7818
:10622000002B5AD1B4F9000005F0A2FF8046B4F962
:10623000020005F09DFF0746B4F9040005F098FF41
:10624000294D06462968404605F0E6FFE968814683
:10625000384605F0E1FF0146484605F0D5FEA9693C
:106260008146304605F0D8FF0146484605F0CCFE91
:1062700008F08CFE69682080404605F0CDFF296952
:106280008146384605F0C8FF0146484605F0BCFE89
:10629000E9698146304605F0BFFF0146484605F0F2
:1062A000B3FE08F073FEA9686080404605F0B4FFB5
:1062B00069698046384605F0AFFF0146404605F063
:1062C000A3FE296A0746304605F0A6FF0146384678
:1062D00005F09AFE08F05AFEA080BDE8F88300BFE2
:1062E0001C11002028000020D8050020074B084A78
:1062F0001B7812889A4207D3064A1268907898420F
:106300008CBF002001207047002070470804002047
:10631000E00B002004040020034B1B68DA79511CB9
:10632000D9711344187A7047A804002010B5FFF7FC
:10633000F3FF0446FFF7F0FF04EB002080B210BD2E
:1063400010B5FFF7F3FF0446FFF7F0FF04EB004042
:1063500010BD094B5A6882420AD01A69824206D09F
:10636000DA69824208BF183302D0002300E00C3300
:1063700000225A725A607047480000200E4B1A7A69
:10638000824215D01A7D82420FD093F8202082429B
:106390000DD003F124011A7A024001D043B909E07B
:1063A0000C338B42F7D1104670470C3300E01833A2
:1063B0005868704718467047480000202DE9F0479C
:1063C0008278C6781E4BC2F1640802EB820C5442FC
:1063D0005FFA88F84FEA4C0CC6F16409A4B203F1E5
:1063E0001807A5B228B2002804DC002D14BF1546FA
:1063F000012500E0454600FB00FA6D430AFB06FA62
:106400009AFBF5F54D4468434FF00A0A90FBFAF009
:10641000604480B258800D88B1F802A000B2C5EB8C
:106420000A0A00FB0AF04FF47A7A90FBFAF005446E
:1064300023F8025F0A34BB42A4B2D2D1BDE8F08790
:10644000060D002010B544780078002303FB03F10B
:106450001939614301F6C4115943414340F6C4124E
:1064600091FBF2F1034A22F813100133072BEDD10F
:1064700010BD00BFF00C002010B5044C2068FFF7E1
:10648000E1FF20680249BDE8104097E7E0030020E3
:10649000981A002010B5094A094913688C681268D7
:1064A0009342F8D1074A106811684FF47A7250434A
:1064B000001BB0FBF1F002FB030010BDC41900206B
:1064C00010E000E0AC05002038B5104C0123054673
:1064D00084F84030FFF7DEFFA36C41F28832C31A24
:1064E0009342E36484BF002384F8503094F8503022
:1064F000EDB20F2BA064E55403D1054B01221A70B5
:1065000038BD024A013382F8503038BD1C110020DA
:106510000801002010B50446FFF7BCFF0D4B41F207
:1065200088315A6D5865821A8A429A6584BF002262
:1065300083F85C2093F85C30074A142BD45403D1C1
:10654000064B01221A7010BD024A013382F85C30FA
:1065500010BD00BF1C110020CD010020CC01002087
:1065600010B50446FFF796FF164A136E1066C31A5D
:10657000B3F57A6F84BF002382F8643092F86430F8
:1065800023B9A82C1CD110490B7006E0022B02D1B4
:106590000E490C7001E0242B01D80D49CC54013375
:1065A000DBB282F86430094A127852000532934215
:1065B00006D1044B002283F86420034B01221A7099
:1065C00010BD00BF1C110020640100208A010020C2
:1065D0006501002038B50446FFF75CFF114B40F61B
:1065E000C4119A6E9866821A8A4284BF002283F888
:1065F0006C2093F86C200AB90F2C11D10A480021A5
:10660000017052B1094D182A154405F8014C04D106
:10661000012283F86C10027038BD013283F86C20BF
:1066200038BD00BF1C110020090100200A01002014
:1066300038B50446FFF72EFF0546FFF72BFF401B3A
:10664000A042FAD338BD10B504462CB14FF47A708D
:10665000FFF7EEFF013CF8E710BD08B5014B1B68E2
:10666000984708BD702100202DE9F04106460F46ED
:1066700090460025EBB2434518D20024E3B2B34262
:106680000FD20B4B0120DA68013482F00802DA6085
:10669000FFF7E3FF3846FFF7D6FF0020FFF7DDFFE7
:1066A000ECE73C20FFF7CFFF0135E3E7BDE8F081E1
:1066B000000C014040F2DB14604308B50A4B08228D
:1066C0001A61841E084B2046DA6882F00802DA60FC
:1066D000FFF7B9FF0120FFF7C0FF1920FFF7B3FF55
:1066E0000020FFF7BAFFEDE7000C014008B5036892
:1066F0005B69984708BD08B503681B69984708BDE2
:1067000008B50368DB68984708BD08B503689B684F
:10671000984708BD08B503685B68984708BD10B581
:10672000044C2068FFF7F6FF18B12068FFF7EDFF73
:10673000F6E710BD9004002008B503681B68984771
:1067400008BD064B10B5044621461868FFF7F4FF54
:10675000034B1B689A7954409C7110BDAC04002017
:10676000A804002038B5044624200D46FFF7E9FFB1
:106770004D20FFF7E6FF002C084C0CBF3E202120E7
:10678000FFF7DFFF2368002228469A71FFF7D9FF41
:10679000236893F84900BDE83840D2E7A8040020F8
:1067A00001460020DEE7F8B50E4E0F4C0F4DC1B28A
:1067B0000746306884F86D10FFF7BEFF2B6894F829
:1067C0006D109A7930684A409A71C7F3072184F8AE
:1067D0006D10FFF7B1FF2B6894F86D109A794A405D
:1067E0009A71F8BDAC0400201C110020A804002000
:1067F000F8B51B4D1B4C1C4F0646C1B2286884F8E7
:106800006E10FFF799FF3B6894F86E109A7928682C
:106810004A409A71C6F3072184F86E10FFF78CFF87
:106820003B6894F86E109A7928684A409A71C6F3CA
:10683000074184F86E10FFF77FFF3B6894F86E10F5
:106840009A7928684A409A71310E84F86E10FFF7E1
:1068500073FF3B6894F86E109A794A409A71F8BDBC
:10686000AC0400201C110020A804002010B5441E18
:1068700014F8011F21B1034B1868FFF75DFFF7E71C
:1068800010BD00BF10180020014B186854E700BF6E
:10689000F0170020A0F17D03012B70B504460D46D2
:1068A0000A4E05D830687D21FFF746FF84F02004AA
:1068B00030682146FFF740FF35B12B881C4404EBBC
:1068C000142404F0FF042C8070BD00BFB804002025
:1068D00038B5054C05465E212068FFF72DFF20687E
:1068E0002946BDE8384027E7F8030020014B5E2128
:1068F000186821E7F803002010B50A4C5E2801460D
:10690000206805D15D21FFF717FF20683E2105E0D3
:106910005D2903D1FFF710FF20683D21BDE810403D
:106920000AE700BFF803002010B50446C0B2FFF725
:10693000E3FFC4F30720BDE81040FFF7DDBF10B54B
:106940000024094BE0B21B7883420CD9074B33F883
:106950001010074B53F820301BB10B2801D89B684F
:1069600098470134EDE710BD40210020422100206E
:1069700038070020054B1B6803EBC00090F9063078
:1069800019420CBF01204FF0FF3070475018002013
:106990000A4B1A6802EBC002D379FF2B07D00849D3
:1069A0000978994203D9074A32F8130004E007280E
:1069B000D4BF908840F2DC5000B2704750180020DD
:1069C000630800206205002010B5054C00202188D6
:1069D00003F04BF961880120BDE8104003F045B990
:1069E0006C0000202DE9F04F0C68836889B0D0F866
:1069F00000A0D0F804800646204603938B4608F09A
:106A00008FFA0746204608F0FFFADBF8044081467B
:106A1000204608F085FA0546204608F0F5FADBF82E
:106A2000082004461046019208F07AFA019A83463B
:106A3000104608F0E9FA39460290584605F0ECFB9A
:106A400039460490029805F0E7FB59460590484600
:106A500005F0E2FB02990690484605F0DDFB294669
:106A60000790584605F0D8FB0146504605F0D4FB88
:106A700021468346069805F0CFFB0146059805F0B0
:106A8000C3FA0146404605F0C7FB0146584605F0EB
:106A9000BBFA21468346049805F0BEFB01460798E1
:106AA00005F0B0FA0146039805F0B6FB01465846DA
:106AB00005F0AAFA3060029905F1004005F0ACFB40
:106AC0000146504605F0A8FB21468346079805F08D
:106AD000A3FB0146049805F095FA0146404605F0EF
:106AE0009BFB0146584605F08FFA214683460598E0
:106AF00005F092FB0146069805F086FA01460398D8
:106B000005F08AFB0146584605F07EFA2146706082
:106B1000504605F081FB2946044609F1004005F086
:106B20007BFB0146404605F077FB0146204605F019
:106B30006BFA39460446284605F06EFB0146039879
:106B400005F06AFB0146204605F05EFAB06009B028
:106B5000BDE8F08F2DE9F84F2E4E044637683846D1
:106B600008F0DEF90546384608F04EFA76688046A9
:106B7000304608F0D5F98346304608F045FAD4F897
:106B8000049006462946484605F046FBA76882461B
:106B90004146384605F040FB0146504605F032FAC2
:106BA00021688246584605F037FB41460446484670
:106BB00005F032FB314605F02FFB0146204605F07B
:106BC00023FA31460446384605F026FB294605F0EF
:106BD00023FB0146204605F017FA0146504608F00F
:106BE000A1FA0D4905F018FB0C4905F0C9FB0C4B47
:106BF000196805F009FA0B4905F0C2FB08F0C6F95F
:106C000083B21A0444BF00F5B4739BB218B2BDE856
:106C1000F88F00BF000300200000E144DB0F494073
:106C20000006002000002041064B1B7803F00403FF
:106C300003F0FF001BB1044B1888C0F3C01000F034
:106C4000010070476C2100205003002010B504465D
:106C5000204607F077FF10F0FF0F06D10C4B0D48D0
:106C60001978BDE81040FDF77BB8204607F0BFFF5C
:106C700002280CD8064B0A221870074B074C02FB5F
:106C80000030074B06301860FFF7F6FBE0E710BD59
:106C90003C0C0020912201081821002077240108D3
:106CA000E0030020174B13B51A88044622F0400277
:106CB0001204120C1A801A883B2022F038021204A7
:106CC000120C1A801A88694692B242F040021A8069
:106CD000062203F065FC9DF800209DF8013043EA90
:106CE000022323809DF802209DF8033043EA02230B
:106CF00063809DF804209DF8053043EA0223A380B9
:106D000002B010BD00300140174B13B51A8804467D
:106D100022F040021204120C1A801A88432022F03A
:106D200038021204120C1A801A88694692B242F094
:106D300040021A80062203F033FC9DF800209DF8E3
:106D4000013043EA022323809DF802209DF803309E
:106D500043EA022363809DF804209DF8053043EA4E
:106D60000223A38002B010BD0030014010B5A0F591
:106D700013746379DB074CD594F8383213B3236B63
:106D80001868828DC2F34E02828494F83C2222B1AC
:106D9000B4F842220132A4F84222A279197B012AD6
:106DA0000CBF0222002203F090FA012384F83B3248
:106DB000002384F8393284F83A3284F83832A4F85F
:106DC000403210BD94F83B322046012B04BF94F8AA
:106DD000393284F83A3202F023FF94F83B12236BE5
:106DE000A27949B9012184F83B128A421868197BBB
:106DF0000CBF0222002208E0002184F83B12012A85
:106E00001868197B14BF02220022BDE8104003F06D
:106E10005CBA10BD10B5A0F5127494F83C22C2B94A
:106E2000A36A616A994229D0591CA069A162C05C19
:106E30002369C0B299424FEA400343F40073A4F8B7
:106E40003E324FF00A0384F83D3228BFA26201238C
:106E500012E094F93D327BB1B4F83E1220464B0863
:106E6000A4F83E3201F0010102F0EFFE94F83D3249
:106E7000013B84F83D3201E084F83C3294F838322A
:106E8000002B4FD194F839320133DBB2092B84F84F
:106E9000393204D12046BDE8104002F0C1BE0A2BB1
:106EA00040D194F83B322BB9B4F8403243F001039F
:106EB000A4F840326379D9071CD5B4F840028205A2
:106EC00001D4C30705D4B4F844320133A4F84432E2
:106ED00010E0E36AC0F347000BB198470AE0E369AA
:106EE0006269D054E269E3680132B2FBF3F103FB5B
:106EF0001123E361012284F8382294F83B22002315
:106F0000012A84F839320DD1A27984F83B32236BFF
:106F1000012A1868197B14BF02220022BDE8104024
:106F200003F0D3B910BD00230F49DAB2595C4F29E1
:106F300003D001330A2BF7D11A460C4B83F82C21CE
:106F4000002283F82D2183F82E214FF4E132C3F87B
:106F50003021C3F83421C3F83821C3F83C21522230
:106F600083F84021704700BF87220108C81900201C
:106F70002DE9F04FD84AD94C85B01068516802AB62
:106F800003C3DFF8908300214FF4EF62204607F03F
:106F900098FD04F50573C8F80030D14B0025DFF8E3
:106FA00078A31D7004F25673CAF80030032363718E
:106FB0000223A36040F24C404FF41673A4F8F03063
:106FC000A4F81C01FA2340F26C70A4F8F230A4F883
:106FD0001E012A231920A4F8EE3084F825014FF46D
:106FE000FA7340F27E40A4F8F630A4F8D0002023D3
:106FF00040F23A7084F8F430A4F8D2006E234FF4D3
:107000007A7084F80431A4F8D4002B2340F27E5027
:1070100084F80531A4F8D600212340F2EA50012675
:10702000552240F2DC514FF01E0B4FF0320984F82C
:107030000631A4F8D8004FF4C87340F2B45022705F
:10704000A4F80831A4F81A11A4F8DA00A4F8DE3084
:1070500084F8EC6084F821B184F8246184F8276115
:10706000A4F8DC90A4F8E0908DE80600FFF75BFF41
:1070700040F6AC53A381D8F8003028271720A57319
:1070800018761F7183F80EB05F7183F80FB05876D1
:107090001D700B20019A1872142058721875502018
:1070A00098776420D8774FF0080E782083F813E0A3
:1070B0005873DFF868C28B484FF00E0E9A7183F850
:1070C0000AE02D224FF05A0E4FF00A0B1A745A772D
:1070D00083F80BE01F73DA7583F821609D7683F8DF
:1070E00007905D74DD769D741D7783F815B0C3F845
:1070F00024C0D86318644FF08240D8624FF07C50AF
:1071000098637948C3F828C05864784A7848DFF80B
:1071100010C200991A635A639864C3F84CC084F88B
:1071200056E74FF0410EA4F85E1784F857E784F84D
:107130005A5784F85B5784F8589784F8595784F85D
:107140005C579A666B4A0421DA666B4A83F85810DA
:107150001521D86583F8607083F861701A6783F829
:107160007460A3F85450A3F85650A3F8525083F813
:1071700064106248FCF74EFFD8F800304FF44872B4
:10718000A3F86221C82283F8A7214FF49662A3F8DE
:10719000A82140F2D932A3F8AA2140F6430283F88D
:1071A0005F7183F86061A3F8AC2183F85D5183F8C7
:1071B0005E5183F8645183F8A6B11A464746564695
:1071C0004FF47F71A2F866114FF4FA61A2F86811CA
:1071D00002A840F2DC51A2F86A11415D013582F843
:1071E0006C11082D4FF0FF0182F86D1102F10802B9
:1071F000E6D1012283F8AE2183F8AF2183F8B021D4
:10720000C82183F8B6216422A3F8B211A3F8B821EB
:1072100014214FF4967283F8B411A3F8BA211E21F9
:10722000282283F8B511A3F8BC210023E2181033FB
:107230000021C02B1161F9D131480021402207F013
:1072400040FC00232F49E218595804330868382BB2
:10725000C2F8D401F6D12C480021802207F031FC7D
:107260002A4B294D03F1300E186859682A4603C28B
:10727000083373451546F7D1254D02F071FB02F036
:10728000ABFB02F085FB3F68284639464FF4E072BD
:1072900007F00EFC394605F5E0704FF4E07207F098
:1072A00007FC336805F563725968186803C21989C9
:1072B00011801A68C5F896235A68C5F89A231B8965
:1072C000A5F89E33012384F82434022384F8E4359E
:1072D00005B0BDE8F08F00BF100F0108C8190020ED
:1072E0003C0C00208FC2753DCDCC4C3D9A99193F86
:1072F0000000A040F6287C3F3D0A773FA22201080B
:107300009C1B0020500601081C1B0020180F0108C0
:107310009C1D002018020020E003002000002040F7
:1073200000004040F7B50368174C184D23600B6808
:10733000174E6360006802F0B9FB95E80300154B37
:107340000196009394E80C0002F06EFB3668124B35
:1073500060681E606B68114FC01A04F009FF104B83
:10736000196804F059FF05F01DF922682B68786050
:10737000D31A3B600B4B1E600B4B1B68DA880B4B20
:107380001A8003B0F0BD00BF700F0020240400205D
:107390007C0F0020780F0020B80F0020800F002005
:1073A00030000020B00F0020D4030020AC0F0020DC
:1073B0002DE9F043142285B0814688461B48002100
:1073C00007F07FFB02261A4B0027B74224DA13F896
:1073D000042C0021C8B2013112B1501E0240F9E75D
:1073E0001C7AD1B2013214B1611E0C40F9E7421A85
:1073F000002A0EDD01ACA3F10C0595E8070084E836
:10740000070093E8070085E8070094E8070083E891
:10741000070001370C33D8E7013ED4D1034A484670
:10742000414605B0BDE8F043FEF758B98C11002085
:107430005400002070B52548037813F0010F03F0C5
:1074400004023AD0002A40D103F0020101F0FF0605
:10745000002932D143F0040303701D4B1A881D4BE1
:107460001A801D4B9B6859052FD5042002F040FF60
:1074700001460420FFF79CFF43681A7AD20724D5FF
:107480005C6814B3154D2B68A34208D12046012136
:10749000FEF75FFF284631464C2207F012FBEB6CEB
:1074A000A34212D120460121FEF753FFBDE87040F0
:1074B0000B4800214C2207F004BB32B90220FF2107
:1074C0000122BDE87040FFF7CFB870BD6C210020ED
:1074D00018030020200D0020C8190020400D0020B6
:1074E0008C0D002038B505460C4602F001FF014620
:1074F0002846FFF75DFF28B143681B7A1C420CBF8A
:107500000020012038BD38B50B4B05469B685A0555
:107510000ED502F01BFA044650B10820E9B2FFF77D
:10752000E1FF30B1054B1C78231F5C425C4100E059
:107530000124204638BD00BFC8190020B404002033
:10754000084B5A6882420AD01A69824206D0DA6928
:10755000824208BF183302D0002300E00C33597276
:10756000704700BF480000202DE9F34706461F463C
:107570004FF41473734345489246C418804626B9A5
:10758000434A2263103AC4F83421424A0025C250CB
:10759000032363714FF480734FF00109E3602361AB
:1075A000D4F8343184F83C5284F8389284F8395253
:1075B00084F84662586804F134029B68626104F5FD
:1075C0009C72A261E1622562E561A5626562A4F830
:1075D0004252A4F84452ADF804300225102301A908
:1075E000C4F808A0A7718DF806308DF8075002F096
:1075F00047FB236B01A958689B688DF80750ADF8CD
:10760000043048238DF8063002F03AFB4946204604
:1076100002F01BFB3220FFF716F81F4BD4F8349111
:107620001B681D46B5FBFAF1B1F5803F03D3012D70
:10763000F8D96D08F6E7194A4846B3FBF2F289B269
:10764000D2B2FDF7B7FD4FF414735E43144B06F549
:10765000127608EB060548F806304846294600220F
:10766000FDF7E0FB266B012F14BF022200223068D9
:10767000317B02F02AFE0B4B30466B60291D002245
:10768000FDF7D0FB204602B0BDE8F087A011002036
:107690006C1D0108480F01088400002040420F00C3
:1076A000156E00086D6D000803460A4690F8460204
:1076B000D96A9B7958E700BF044B1A6942F48042AB
:1076C0001A611A6922F480421A6170470010024060
:1076D0002DE9F0418CB01D469DF848308846012BBD
:1076E0001746A54B06D1984265D10422A3F5305325
:1076F0001A6101E098425ED1A048A14B8760036007
:10770000A04BA907436103F1C00383614FF0C0039D
:10771000C3600361984B036503F104038364C3648E
:1077200003F5484303F154030363A3F11403D3F8AF
:10773000D42F436342F48042C3F8D42FD3F8D02F20
:1077400042F00102C3F8D02F4FF002038DF803304E
:107750004FF40073ADF800304FF018038DF802308D
:1077600003D58948694602F08BFA1C232A078DF855
:10777000023003D58448694602F082FA4FF48063F0
:10778000ADF8003048238DF80230EB0703D57E4872
:10779000694602F075FA0E238DF8043000220123A9
:1077A00001A88DF805308DF806208DF80730734C50
:1077B000FDF78EFC53E0754B984240F0D980744B36
:1077C0006F4A9F601A60734A18655A61C0329A61A5
:1077D000C022DA601A61704AAE079A64DA646F4BAD
:1077E000DA6942F48022DA619A6942F008029A6109
:1077F0004FF002038DF803304FF48063ADF8003092
:107800004FF018038DF8023003D56548694602F041
:1078100037FA1C232C078DF8023003D560486946DF
:1078200002F02EFA4FF40063ADF80030E8074FF095
:1078300048038DF8023003D55948694602F020FA12
:1078400027238DF804300022012301A88DF805308C
:107850008DF806208DF80730FDF73AFC4C4C0026D9
:10786000012384F844302662E661A6626662C4F8A9
:107870002C806571A760A6712046FDF75BFA15F0B4
:10788000090F31D0206B002826D0E36C03960193BA
:107890004FF480530A9380230693E368059604937C
:1078A0002023099363690796029308960B96FEF7C7
:1078B000EDFB01A9206BFEF7CBFB236B1A6842F0AE
:1078C00001021A60226D918A89B241F040019182D1
:1078D0005B689BB2236407E0236D4FF6DF721A806A
:1078E000DA6842F02002DA6015F00A0F2CD0606BE3
:1078F00028B3A36C002601934FF480530A9380238E
:107900000693236902960493102303930596079622
:10791000089609960B96FEF7B9FB606B01A9FEF776
:1079200097FB636B1A6842F002021A605E605E6049
:10793000236D9A8A92B242F080029A8204E0236D0B
:10794000DA6842F08002DA60236D29079A8992B2E0
:1079500042F400529A819A8A03D592B242F0080208
:1079600003E022F008021204120C9A82204600E082
:1079700000200CB0BDE8F081003801406C190020F7
:10798000600F0108F013002000080140004800408B
:107990001819002070150020044800400010024013
:1079A000000C01402DE9F047054607F0CBF8304BBD
:1079B0000446D3F808809A4690B92E48FEF756FF41
:1079C0002D4B53F8241049B10123A34013EA080FAB
:1079D00002D02A48FCF7C4F90134F1E7284821E035
:1079E00028462849224607F0B5F858B92648FEF738
:1079F0003DFF264C54F8041F0029EFD01F48FCF728
:107A0000AFF9F7E72B7800262D2B03BF013504F1E2
:107A1000FF344FF001094FF00009174B53F826705F
:107A200027B91B48BDE8F047FEF720BF2846394676
:107A3000224607F08FF8C8B90120B040830501D570
:107A40001448EFE7B9F1000F03D001F024FF12480A
:107A500004E040EA0800CAF808001048FEF706FFF4
:107A600039460F48BDE8F047FCF77AB90136D4E74C
:107A7000C8190020AB220108780F0108C61F0108B1
:107A8000B827010832260108BE220108740F010838
:107A9000D3220108EA220108FE2201080823010876
:107AA000412201082DE9F04F87B09A468046894669
:107AB00016469DF8404002F01BFC02AF0546034607
:107AC00000F1100E186859683A4603C2083373452E
:107AD0001746F7D12B7B0BB903960496404602A9B3
:107AE000FFF766FC054640B14368586830B1404630
:107AF00002A92A46FDF7F2FDF4E72CE0AB6895F801
:107B000000B01F78012F22D1144800944946324614
:107B10005346FFF7DDFD04460AE0022F1BD149461C
:107B200023463246FFF720FD51460446FEF7DEFDB0
:107B30005CB10B4B277103EB8B03C3F800436B68FD
:107B400020465C604146FFF7FBFC204603E0E4D2A0
:107B500000940448DAE707B0BDE8F08F0048004021
:107B6000F013002000380140254B37B5DA69254C69
:107B700042F48042DA611A69204642F480421A6176
:107B800018238DF806304FF42043ADF8043001A9D6
:107B900003238DF8073002F073F84FF48043ADF8FB
:107BA000043004230DEB030120468DF806304FF41A
:107BB000805502F065F81023204601A98DF80630A3
:107BC000ADF8045002F05CF82561FFF775FD0E4B2F
:107BD0001A8802F4415242F4457242F003021A80BC
:107BE0009A8B22F400621204120C9A8307221A82E2
:107BF0001A8892B242F040021A8003B030BD00BF32
:107C000000100240000C01400038004037B5254C00
:107C1000254DA369284643F48053A361E36801A975
:107C200043F48053E36018238DF80630A023ADF8A9
:107C3000043003238DF8073002F022F84023ADF81A
:107C4000043004230DEB030128468DF8063002F0C2
:107C500017F81023284601A9ADF804308DF8063036
:107C600002F00EF8E36843F48053E360E36823F422
:107C70008053E3600D4B1A8802F4415242F445727E
:107C800042F003021A809A8B22F400621204120C52
:107C90009A8307221A821A8892B242F040021A800E
:107CA00003B030BD00100240000801400030014028
:107CB00008B502F0B1FB03F0C3F8BDE808400F209F
:107CC00014210122FEF7D0BC2DE9F04F692887B0BE
:107CD000044600F0A38200F296802E2800F037853B
:107CE00062D8242800F007852BD8202800F07E8257
:107CF000222800F0B383012840F05A852C20FEF79B
:107D00004FFD0020FEF71DFD2046FEF71AFD002066
:107D1000FEF717FD4320FEF714FD4C20FEF711FD82
:107D20004620FEF70EFD4C20FEF70BFD2046FEF729
:107D300008FD0020FEF705FD0020FEF702FD0024EF
:107D4000F0E0282800F0DF8412D8262840F03085A3
:107D5000924C0320FEF724FDB4F9E600FEF723FD64
:107D6000B4F9E800FEF71FFDB4F9EA0000F029BC01
:107D70002A2800F0D3842C2840F01A85874C07204D
:107D8000FEF70EFD94F81801FEF7DBFCB4F91E01B6
:107D9000FEF709FDB4F91A01FEF705FDB4F91C015F
:107DA000FEF701FD00F0C0BC642800F0E2801AD8A4
:107DB000322800F0B9840AD8302840F0F984774C92
:107DC0008020FEF7EDFC04F1800500F0D6BC3428DD
:107DD00000F06483402840F0EB840820FEF7E0FCCC
:107DE000002400F0AABC662800F09881C0F0EE8064
:107DF000672800F0CC81682840F0DA841020FEF774
:107E0000CFFC002402E2732800F0AF8355D86D2820
:107E100000F0178212D86B2800F0D78340F2B083AD
:107E20005F4C0620FEF7BCFCB4F90000FEF7BBFC7B
:107E3000B4F90200FEF7B7FC5A4BC0E36F2800F01C
:107E40003082C0F00682702800F07682722840F0FE
:107E5000AF84524C1620FEF7A3FC0020FEF7A3FCD3
:107E6000B4F9D000FEF79FFC4F4DB4F9D200FEF7F5
:107E70009AFCB4F9D400FEF796FC2B68B3F9A8017C
:107E8000FEF791FC0020FEF78EFC0020FEF7B0FC10
:107E90002B68B3F952000A2390FBF3F0FEF783FC42
:107EA00094F80401FEF74DFC94F80601FEF749FC36
:107EB00094F80501FEF745FCE3E3782800F07381B0
:107EC00010D8752800F0BE82C0F00983762800F033
:107ED0008E83772840F06C84344D00242878FEF798
:107EE0005FFC37E3A42800F0CE8310D8A02840F030
:107EF0005F840C20FEF754FC2D4B1868FEF778FCCD
:107F00002C4B1868FEF774FC2B4B1868F8E3F0282C
:107F100000F0E483FE2840F04B840820FEF740FC8C
:107F20000024D3E3254B1B68185D0134FEF709FCE0
:107F3000042CF7D10020FEF736FC0024204B185DFE
:107F40000134FEF7FEFB0B2CF8D100241D4B185D0D
:107F50000134FEF7F6FB082CF8D10720FEF7F1FB01
:107F60000024194B185D0134FEF7EBFB072CF8D108
:107F700087E30720094CFEF713FCE620FEF7E1FB40
:107F80006079FEF7DEFB0020FEF7DBFB94F826317C
:107F9000002B0CBF04200C20B2E300BFC819002046
:107FA0000803002018030020180200200E180020EB
:107FB000E8F7FF1FECF7FF1FF0F7FF1F8C00002012
:107FC000D1210108DD210108E62101080B20FEF77F
:107FD000E7FBC34BB3F90000FEF7E5FB0020FEF71B
:107FE000E2FBC04B1B68C3F3C000C3F380028000F8
:107FF00040EA4200C3F340021043C3F3401240EA98
:10800000C20003F010031843FEF7CDFBB64B1A88ED
:1080100012F0010F0CBF0020022012F0020F0CBF63
:108020000021042112F0040F0CBF0023102312F0D2
:10803000400F0CBF00242024019312F0100FAB4B13
:1080400002940CBF00244FF4007412F0200F1B6840
:1080500003940CBF00244FF4806412F4807F0494D6
:108060000CBF00244FF4006402F0080B03F4807A84
:10807000059403F4805903F4005803F4004C03F40E
:10808000803E03F4003703F4802603F4002503F454
:10809000801403F0C00343EA0B0343EA0A0343EAF4
:1080A000090343EA080343EA0C0343EA0E0E904B2C
:1080B0004EEA07073E431B7835432C43C3F3800346
:1080C000234303430B430199029C0B43039923432E
:1080D000049C0B430599234312F4007F43EA0103F8
:1080E0000CBF00224FF400121A43824B00201C7870
:1080F0000346A3420CD280495D5C012101FA05F5DB
:10810000154218BF994003F1010318BF0843F0E777
:10811000FEF76EFB794B93F854070BE31220FEF742
:108120003FFB774B774C1B88B3F5806F22D9002536
:10813000605F082390FBF3F00235FEF734FB062D59
:10814000F6D1714CB4F90000FEF72DFBB4F9020032
:10815000FEF729FBB4F904006C4CFEF724FBB4F9DC
:108160000000FEF720FBB4F90200FEF71CFBB4F997
:10817000040026E2B4F90000FEF715FBB4F9020092
:10818000FEF711FBB4F90400FEF70DFBD9E7102050
:10819000FEF706FB00245E4B185D0134FEF7D1FAB2
:1081A000102CF8D10FE23820FEF7FAFA0025594ECC
:1081B00005F12C043368E4002344B3F90600FEF70C
:1081C000F2FA336801352344B3F90800FEF7EBFAFD
:1081D00033682344B3F90A00FEF7E5FA33681C4418
:1081E000207BFEF7AEFA082DE1D1ECE10820FEF786
:1081F000D7FA0024474B1B6803EBC40393F86D01C7
:108200000134FEF79EFA082CF4D1DCE1424B185DF4
:108210000134FEF796FA102CF8D1D4E13F4D00243A
:108220002878400000F0FE00FEF7BAFA2B789C4256
:1082300080F0C9813A4B33F91400FEF7B4FA0134E7
:10824000F4E70620FEF7ACFA0020FEF7D1FA002092
:10825000B7E10720FEF7A4FA324B4FF6FF74187807
:10826000FEF76FFA304B1868A042A8BF204620EAFC
:10827000E07000B2FEF797FA2C4BB3F90000FEF75E
:1082800092FA1E4B93F80C21294B18680028B8BFAE
:1082900040420AB10A235843A042A8BF204600B278
:1082A0008FE1244C0720FEF77BFA23681878FEF74D
:1082B00048FA23685878FEF744FA23681879FEF7DD
:1082C00040FA23685879FEF73CFA23689879FEF75C
:1082D00038FA23689878FEF734FA2368D87829E2C8
:1082E0004403002088020020500300204C0300209B
:1082F0006C2100200E180020F8170020C81900205B
:1083000000000020E80200203C0300209E05002021
:108310006C00002018020020422100206308002089
:10832000620500200804002010040020E60B002055
:108330000C040020E0030020B44D1E20FEF730FAAC
:108340002B6800241B78022B69D12B68B04903EB02
:108350008403586A03F060FF06F018FEFA28A8BFED
:10836000FA2020EAE070C0B2FEF7EBF92B68A949C9
:1083700003EB8403186B03F04FFF06F007FEFA28A7
:10838000A8BFFA2020EAE070C0B2FEF7DAF92B6845
:10839000A14903EB8403D86B03F03EFF06F0F6FD22
:1083A0006428A8BF642020EAE070C0B20134FEF760
:1083B000C8F9032CC9D1072C2B681ED1986C94499D
:1083C00003F02AFF06F0E2FDFA28A8BFFA2020EA0F
:1083D000E070C0B2FEF7B5F92B688D49D86C03F098
:1083E0001BFF06F0D3FDFA28A8BFFA2020EAE070B0
:1083F000C0B2FEF7A6F900200BE023441879FEF77F
:10840000A0F92B682344987BFEF79BF92B68234443
:10841000187E0134FEF795F90A2CCCD1D3E02B68F5
:1084200023441879FEF78DF92B682344987BFEF7D7
:1084300088F92B682344187E0134FEF782F90A2C50
:10844000EDD1C0E02F20FEF7ABF9744C14F8010F0A
:10845000002800F0B880FEF774F9F7E7A020FEF7D7
:108460009FF90024694B04F11C021B680C2103EBEB
:1084700082035D1D6A4A5B79013401FB0323187A8C
:10848000FEF75FF96878FEF75CF9A878FEF759F90E
:10849000E878FEF756F9282CE4D194E04820FEF75E
:1084A0007FF9002506266E43584B06F588761B6833
:1084B00001351E44B07AFEF744F97079FEF741F9B0
:1084C000B079FEF73EF9F079FEF73BF9307AFEF726
:1084D00038F9707AFEF735F90C2DE3D173E00027F7
:1084E000012400254F4B1B789D4222DA4E4BE95C5C
:1084F00000234B4A03EB02089A5C8A4204D00C33F7
:10850000B3F58A7FF5D112E0D8F8040006F01AFB23
:1085100081460CB9264601E0074408E04E4506DADC
:10852000D8F80430985DFEF70CF90136F6E701350E
:10853000D8E7002C47D0F8B2FEF732F90024D0E794
:10854000374A99189A5C82420BD00C33B3F58A7F74
:10855000F6D101342B789C4235D2334BE05C0023BA
:10856000EEE7087AFEF7EDF8F3E70820FEF718F9D2
:108570000124E0B20134FEF7E4F8092CF9D122E03D
:108580001020FEF70DF9294B294C187800F0020055
:10859000FEF7D7F8274B1878FEF7D3F82068FEF7D8
:1085A00027F96068FEF724F9234BB3F90000FEF7C2
:1085B000FAF8224BB3F90000FEF7F5F8204BB3F9B7
:1085C0000000FEF7F0F80120F3E00520FEF7E8F8E0
:1085D0001C4BB3F90000FEF7E6F81B4BB3F90000A3
:1085E000FEF7E1F8194B187800F00100A2E0FDF762
:1085F00093FE06461220FEF7D3F80EB9144B02E0A4
:10860000102E29D1134B1D685C6827E0180200204A
:10861000000020410000C84200007A44C30F010856
:10862000D80C01080E180020F8170020FE020020C8
:108630002404002018040020160400201404002044
:10864000FC160020880400208A040020F60D00207B
:10865000480C0020540C0020002425463046FEF72C
:1086600070F82846FEF7C4F82046FEF7C1F8524BD2
:108670001868FEF7BDF80020FEF795F80020FEF719
:1086800092F8002056E04D4D0024A8782E46800038
:108690000130C0B2FEF784F8A878FEF752F8B3783C
:1086A0009C4290D2464D285DFEF74BF805F1100331
:1086B000185DFEF746F805F12003185D3035FEF72A
:1086C00040F8285DFEF73DF80134E8E73D4B185FC0
:1086D0000234FEF768F8082CF8D174E73A4C04200D
:1086E000FEF75EF82368B3F95600FEF75CF82368DE
:1086F000B3F9540065E70420FEF752F8334B98684D
:10870000FEF776F85FE7314C0420FEF749F8B4F93C
:108710000801FEF748F8B4F90A0152E70120FEF714
:108720003FF82A4B587905E00120FEF739F8274B2E
:1087300093F82001FEF705F845E7244B234493F80E
:1087400010010134FDF7FDFF082CF6D13BE7402076
:10875000FEF726F81D4C04F14005B4F9D401FEF7EC
:1087600022F894F8D601FDF7ECFF043494F8D30115
:10877000FDF7E7FFAC42F0D125E7B4F85601043429
:1087800000F03F00FEF70FF8B4F85201C0F3841078
:10879000FEF709F894F850010009FDF7D2FF94F8AC
:1087A000500100F00F00FDF7CCFFAC42E5D10AE725
:1087B000002007B0BDE8F08FF80D0020FC16002067
:1087C000FF1600204017002018020020C8190020C2
:1087D000954B2DE9F74F1B78013B012B00F22081CF
:1087E000924B1E78864240F01B81914B1B78022BE6
:1087F00000F016818F4B904D13F806808F4B83F855
:1088000000808F4B1A7801921AB18E4B33F9160003
:1088100007E08C4A2B6832F9160003F100432B6005
:10882000404203F0A5FC884903F0AAFDDFF838A216
:108830000446DAF800B00021584603F081FE002714
:10884000DFF82C92002859D0D9F800B020465946BC
:1088500003F09EFE68B17D4B2A687B491A60C9F817
:108860000040204603F0D8FC03F09CFE784BD880F3
:10887000BDE05846394603F08BFE002800F0B78073
:10888000744B1A78002A31D12046296803F0BAFBCC
:108890004FF07E5103F05EFE6F4C28B160686F4967
:1088A00003F0BAFC60600FE06D49606803F0B4FC4F
:1088B000DFF8CCA18346514603F04CFE10B9C4F852
:1088C00004B001E0C4F804A0624A01231370654BB0
:1088D00000221B68C9F8007043449A72019A82F022
:1088E0000103574A1370604B1F6080E05F4BCAF86A
:1088F00000401A68554BFA325A6078E020465946D3
:1089000003F028FE48B1584A4F491460204603F04E
:1089100083FC03F047FE4E4BD880534BD9F80090B0
:10892000D3F800A04846514603F06CFB4F4B8346FA
:108930001968464B5A688A1A002A0BDA4FF07E51A2
:1089400003F026FE002852D02046514603F020FEB8
:1089500000284CD03D4A4846116803F019FE3E4CB1
:1089600038B120683E4903F057FC3C492060A068BC
:1089700007E058464FF0804103F00AFE28B1A06896
:10898000374903F049FCA06004E02068334903F054
:1089900043FC2060334B2C492068D3F8009003F04F
:1089A0003BFC03F025FE09F80800A06803F020FE58
:1089B000019AC84482F00103214A88F81400137018
:1089C000294B1F602A4B1F60224B1A780132D2B20A
:1089D000032A01D01A700AE000221A701E4B2549A2
:1089E000586803F019FC03F003FE88F80A001EB96A
:1089F000174B1A8864321A80114A13780BB11E4B38
:108A000000E01E4B2B600F4B33F9160003F0B0FB58
:108A10000D4903F0B5FC0146286803F0F3FA00E0C5
:108A2000084603B0BDE8F08F52030020A4030020E5
:108A3000B40300200806010854030020B5030020F9
:108A4000A503002008030020000020414817002053
:108A500040170020A6030020B80300200AD7833F58
:108A6000EC51783FB0030020A8030020C419002077
:108A7000AC03002000007A440000A0410000A0C127
:108A80006F12833A10B50848FDF7F0FE074B1C68DB
:108A90002046FDF730FE18B90A20FDF7D4FDF7E7B0
:108AA000034A044BDA6010BDB623010810180020F9
:108AB0000400FA0500ED00E008B50548FDF7D6FE14
:108AC000FEF756FA01F0A8FCBDE80840FFF7DABF50
:108AD000C223010808B50748FDF7C8FE064A00236F
:108AE00013729363054A1370FCF73EFEBDE808401D
:108AF000FFF7C8BFD8230108481700206B210020CA
:108B000008B50448FDF7B2FE01F086FCBDE8084058
:108B1000FFF7B8BF042401082DE9F04F002487B007
:108B2000074603919146049382462546022DDFF8BD
:108B300078814FEA450607D103984379B8F90400D4
:108B40001B3343435B1148E04D4B38F9151033F9A3
:108B5000153003EB4101C9F10003994203DB49459C
:108B6000B4BF0B464B464749049A31F906B0915FB2
:108B7000CBEB030303EB010BFEF756F898B1424B26
:108B800058465B5D029303F0F3FA404903F0F8FBAB
:108B9000029B01461846FFF71BFE3C4903F03CFBD5
:108BA00003F000FD83463A4B1988C80711D4039897
:108BB0008A07037938F9060003F11B0300FB03F36E
:108BC0004FEA231309D57A7C02FB0BFB03EB2B2323
:108BD00003E0FB7903FB0BF31B112E4A2E49905F38
:108BE000042290FBF2F0181A7B5D9AF80AC0434306
:108BF00005932A4B6258B3F800B001350BFB00F324
:108C0000DB120CFB0323264AB3F5001FA8BF4FF469
:108C100000139342B8BF1346635022494FEA1B1B0F
:108C200062584FF6FF7C821ABCFBFBFC0CFB02FC7B
:108C3000605001F1180B01F10C0054F8008054F859
:108C40000B204FEAAC1C44F800C042449AF81400D0
:108C50006244019242430598121202EBE012243161
:108C600002EB6333032D44F80B808B530AF1010AA6
:108C700004F104047FF45AAF07B0BDE8F08F00BFE1
:108C8000602100200803002000100108000020419E
:108C9000500300203C030020D40C0020440300209B
:108CA0000000E0FF84170020C60300202DE9F04FEC
:108CB00089B00793914B0692B3F90220B3F90030C3
:108CC000002AB8BF5242002BB8BF5B4200249A4230
:108CD000B8BF1A46039005922646A146274604943B
:108CE000A0462546DFF844A2BAF8003099075AD0CA
:108CF000022D58D0814BDDF818B0F25E804BF35E48
:108D000003EB4202CBF100039A4203DB5B469A423B
:108D1000B8BF13467B4ADDF81CC036F902B03CF9F7
:108D20000620CBEB030303EB020BFDF77DFF90B1B5
:108D3000754B584615F8038003F01AFA734903F08F
:108D40001FFB01464046FFF743FD704903F064FAFC
:108D500003F028FC834603996423CA7902FB0BF2D3
:108D600092FBF3F2CB7E6FF0040101FB03F8424566
:108D700005DB03EB83039A42B4BF90469846644AEE
:108D800042F21071A3585B448B42A8BF0B46614965
:108D90008B42B8BF0B46A350039A92F811B00BFB5D
:108DA00003F31B130493BAF8003003F00302012A03
:108DB00001D1022D3ED15849504A895FB75EDDF896
:108DC0000CB0564A81EAE170A0EBE170B0F5206F7B
:108DD0001BF805C054F802901DDC022D15D0502060
:108DE000784390FBFCFC042091FBF0F1C1EB0C0CF0
:108DF000E1444B48B9F57A5FA8BF4FF47A598145F1
:108E0000ACBF42F80490105107E087EAE770A0EB8E
:108E1000E7706428E3DD00211151404AA1587D220A
:108E200091FBF2F9039A2A44927A02FB09F9402253
:108E300099FBF2F99A0716D5022D14D0DDF814C06B
:108E4000DDF810B00CFB07F30CFB09F0CCF5FA7160
:108E500001FB083301FB0B014FF4FA7293FBF2F3B1
:108E600091FBF2F108E0DB0701D5022D02D1494662
:108E70003B4601E004994346274ADFF8B4B0B25AB2
:108E800004200FFA82FC15F80BB09CFBF0FA0BFBE8
:108E90000AFB6FF04F0A9BFBFAFA9A44214BCDF87C
:108EA00004A036F903A0F252CAEB0C0C9CFBF0FCB8
:108EB00003F1120A981D225854F80AB044F800C071
:108EC00019489344285CCDF808B0E34444F80A20DC
:108ED00000FB0BF2202092FBF0F2DDF804C08A1AAE
:108EE0000135063B6244032DF25204F1040406F1FD
:108EF00002067FF4F7AE09B0BDE8F08FC60300208C
:108F0000602100200803002000100108000020411B
:108F1000400C0020F0D8FFFF3C030020D40C0020C0
:108F200080C1FFFFAE170020040D00205003002079
:108F3000FE0C00202DE9F04F89B007937A4B814653
:108F400018880491059203F00FF9784903F064F949
:108F5000002403904F4625462646022EDFF80CA239
:108F60000BD10499BAF904004B790A33584303F042
:108F7000FFF86F4903F004FA44E06E4B3AF905201C
:108F8000EB5E05991A444B429A4203DB0B469A4228
:108F9000B8BF1346684AAA5E9B1A079A505F1844E6
:108FA00003F0E6F8654903F0EBF98046FDF73CFE77
:108FB00028B1634B4146985DFFF70AFC8046614B40
:108FC0001A88D10705D54046D9F8441003F024F992
:108FD00018E004993AF905000B79019214335843CB
:108FE00003F0C6F8524903F0CBF9019A8346930780
:108FF00009D5D9F84810404603F00EF90146584605
:1090000003F002F88346504A505F03F0B1F84F4A2C
:10901000D16803F001F982465146584602F0F2FF4A
:10902000396A804603F0F8F8DFF844B106900399F6
:10903000404603F0F1F8F96A03F0EEF854F80B102B
:1090400002F0E2FF4249804603F084FA38B9404614
:10905000404903F09DFA20B1DFF8F88001E0DFF825
:10906000F0804BF80480DFF80CB1504654F80B1038
:1090700002F0C8FF44F80BA0034603994FF07E505E
:10908000029303F07DF9029B0146184603F0C4F8F1
:109090000BF10C03E2580BF1180B54F80B1082463D
:1090A00010460192029302F0AFFF514602F0ACFF6E
:1090B000019A029B44F80B2044F803A0264903F0D0
:1090C0005FF9B96B03F0A8F82449824603F042FA2D
:1090D00038B95046224903F05BFA20B1DFF880A08E
:1090E00001E0DFF878A00698414602F08DFF514676
:1090F00002F088FF05F04AFF1A4BB0F57A7FA8BF4F
:109100004FF47A709842B8BF18460136164B032EBA
:10911000E85204F1040405F1020507F104077FF4A5
:109120001CAF09B0BDE8F08F44030020BD37863581
:109130000000484260210020080300200000204178
:1091400000100108500300203C0300201C020020F6
:1091500000007AC300007A4300004040000096C33C
:109160000000964318FCFFFFA8170020C60300204C
:10917000E00C0020CC1700202DE9F047704B86B0A2
:109180001A789946DFF8C88192B90123D8F800000F
:10919000022189F80030FEF7D3F9D8F80030694A87
:1091A0006948C2F8A830FDF761FB6848FDF75EFB2F
:1091B000D8F80000FDF7AEFA002800F0BE80644B3E
:1091C000604C1868FDF7A1FA0928014601D03F2834
:1091D0004FD14FF0000AA56B5E4F56462DB15E4849
:1091E00039682A4605F0B6FC10B9BA4606B93E46BB
:1091F0005A4B0C379F42F1D3CEB13768DAF800E012
:109200002B46F85C1EF80310814201D0A3630EE0E8
:109210005A1C41B92D2B06D8A26323442020224496
:109220001872117203E04C4958541346E9E7A36BD6
:109230000BB1564512D04A48FDF718FB564509D8E0
:1092400056F80C0BFDF712FBD8F800000921FDF7CA
:1092500073FAF3E73D48FDF709FB0025A36B9D4238
:10926000A6D23D4BD8F80000595DFDF765FA0135EF
:10927000F4E7A36B33B904283BD104F10800FFF7EE
:1092800029FC5AE00C2801D136488CE70A2901D084
:109290000D2949D13448FDF7E9FAA36BE218002300
:1092A0001372227A232A17D00493304B2A4E00934C
:1092B00003A8284915220C23039605F09CFC0546BB
:1092C00038B1006805F03EFC0130AB683044984787
:1092D00002E02748FDF7CAFA1F480021302205F0B6
:1092E000F0FB0023A36399F80030002B7FF45DAFFF
:1092F00023E00C28C8D07F2903D159E72F2B3FF654
:1093000057AFA1F12002D2B25E2A3FF651AF13B996
:1093100020293FF44DAF5A1CA263D8F800001C442A
:109320002172FDF709FA43E77F29E7D1013BA363E7
:10933000002223441A720F4838E706B0BDE8F087D0
:109340006B210020481700200B240108432401084A
:109350001018002004100108501700200011010807
:10936000482401084D240108B82701080D600008B1
:1093700058240108742401081F4B13B51A886B2068
:1093800022F040021204120C1A801A88802122F066
:1093900038021204120C42F030021A801A88062495
:1093A00092B242F040021A8001F030F99620FDF7A7
:1093B0004AF975200DF10701012201F0F1F89DF83D
:1093C0000730682B04D0013C14F0FF04EED110E00C
:1093D0000C200DF10701012201F0E2F89DF80730A1
:1093E000142B06D3182B02D9543B062B01D801208D
:1093F00000E0002002B010BD0030014003685A1C9C
:10940000026019707047016B0346C26810B540696D
:1094100041B1196C541A005D013918BF0A46C0B237
:109420001A6410BD196A405C0131B1FBF2F402FB11
:109430001412C0B21A6210BD026B03691AB15168EE
:10944000013B026C02E0C169026A013B881A1840C4
:10945000C0B27047436B13B190F844007047826A02
:10946000436AD31A58425841704743799B070AD53B
:10947000436A8269D154426A03690132B2FBF3F153
:1094800003FB112343627047437913F0010307D0B4
:10949000C368C169026A013B881A1840C0B27047AC
:1094A00018467047437910B513F0010304460DD0F8
:1094B000FFF7EAFF58B1226A6369985CE3680132FA
:1094C000B2FBF3F103FB1123236210BD184610BD5C
:1094D000426A806A131A5842584170474171704776
:1094E00010F80A3C0133DBB20A2B00F80A3C0AD917
:1094F00010F8123C23B910F8131C034A22F811305B
:10950000002300F80A3C7047CC0F0020334A10B506
:10951000136C90681944081A40F68C2398429160A5
:10952000D060516013463CD9127893F945108A42B5
:109530000BD1111F082908D893F84610182901D813
:10954000013103E083F8442002E0002183F8461053
:1095500093F944108A421CD1204991F84710C1B1B7
:10956000002191421E4806DA03EB8104246920F8A9
:1095700011400131F5E7511E00EB410116308142E7
:1095800003D0002421F8024FF9E71649087801308A
:10959000087083F84520002201211A7083F84710D3
:1095A00010BD92F84710B9B1A0F2EF2440F2DA51A1
:1095B0008C4208D811780B2905D80B1D0131117088
:1095C00042F8230010BD002283F847209918043286
:1095D0000020302A0861F9D110BD00BF100600201C
:1095E000CC0F00209C100020024B1A6C0132114459
:1095F0001964704710060020024B53F820301B6896
:109600001980704738070020074BA1F57A7153F88D
:1096100020304FF47A701A689B884B4393FBF0F329
:109620009BB21380704700BF38070020024B4FF4F5
:1096300080521A80704700BF0000002070472DE95B
:10964000F04102780346202A00F10100F9D0092AEE
:10965000F7D02D2A02D10346404D04E02B2A08BF43
:1096600003464FF07E551E460024334616F8012B64
:10967000A2F13007F9B209290DD83949204602F084
:10968000CBFD0446384602F073FD0146204602F049
:10969000BBFC0446E9E72E2A17D1314F334616F8B2
:1096A000010B3038C2B2092A0FD802F061FD3946E9
:1096B00002F066FE0146204602F0A6FC2849044658
:1096C000384602F0A9FD0746E8E71A7802F0DF0203
:1096D000452A38D15A782D2A02D10233012604E0D6
:1096E0002B2A14BF013302330026013B002713F855
:1096F000012F303AD1B2092903D80A2101FB0727EB
:10970000F5E7B7F59A7F28BF4FF49A77B8464FF040
:109710007E51B8F1070F07D90846124902F07CFDC7
:10972000A8F108080146F4E707F0070737B1084633
:109730000B4902F071FD013F0146F7E72EB12046CB
:1097400002F01EFE04E04FF07E51204602F064FD60
:109750000146284602F060FDBDE8F081000080BFB0
:109760000000204120BCBE4CF0B50124B0FBF4F554
:109770008D4201D34C43F9E70026DCB1B0FBF4F590
:1097800004FB1500B4FBF1F41EB9002D01DC002C24
:10979000F3D1092D03F101075FFA85FC04DD002AEE
:1097A0000CBF5725372500E0302565441D70013674
:1097B0003B46E2E71C70F0BDF0B50124B0FBF4F5C8
:1097C0008D4201D34C43F9E70026DCB1B0FBF4F540
:1097D00004FB1500B4FBF1F41EB9002D01DC002CD4
:1097E000F3D1092D03F101075FFA85FC04DD002A9E
:1097F0000CBF5725372500E0302565441D70013624
:109800003B46E2E71C70F0BD70B50646B6FBF2F4CD
:109810000846154614B12046FFF7F6FF05FB146411
:10982000024B1B5D00F8013B70BD00BF78240108AE
:109830002DE9F041069C002B06460F460CBF4FF069
:1098400020084FF03008234613F8011B09B91546CC
:1098500003E0002AFBDD013AF6E7002D04DD304687
:109860004146B847013DF8E714F8011B11B13046F5
:10987000B847F9E7BDE8F08180EAE073A3EBE07355
:109880008B4206DB002801DD401A704702D00844F5
:10989000704700207047034B9A6822EA00009860E6
:1098A000704700BFC81900200E4B1B78BBB10E4B90
:1098B0001B681A78032A06D10C4B187802288CBF33
:1098C0000020012070475B7823B1094B1868C0F372
:1098D000C0407047074B1878C0F3800070470120E4
:1098E000704700BFD20B0020F4030020B404002016
:1098F0004C0300206C210020114A30B50028B8BF6D
:109900004042104C90FBF2F304FB03003C256843FB
:109910000D4D90FBF2F22D682D7B25B903EB8303EF
:1099200003EB830301E0C3EB031302EB830304FBAC
:1099300002020B804FF47A7392FBF3F24A8030BD3F
:1099400080969800806967FF1C040020034B1B6809
:109950001878C31E58425841704700BFF4030020D6
:10996000094A0A48002310B5116803701A46CC183A
:1099700064880CB9CC5C24B104330132802BD2B2A0
:10998000F5D1027010BD00BFDC040020600500208E
:1099900010B50B4B0B4819780B4B1A784B085C1E13
:1099A000047001F0010109480B4403700849530891
:1099B000581E087002F00102064913440B7010BDD6
:1099C0009905002094050020F4170020960500203A
:1099D0009705002095050020F0B50F4A0F4816782E
:1099E0000F4A0023176803701A4619460546D0B27D
:1099F000B0420CD217F82200013204099C4200F058
:109A00000F00A8BF631C8842A8BF411CEFE72B7062
:109A1000044B1970F0BD00BF60050020F417002052
:109A2000DC04002099050020F8B5101A0C461F46EA
:109A300002F09EFB0546381B02F09AFB174B079E6F
:109A4000196802F0E9FB29460446284602F0E4FBC7
:109A500021460746204602F0DFFB0146384602F069
:109A6000D3FA05F061FB0E4902F0D6FB02F0C0FD0F
:109A7000069B2146186005F1004005F053FB09499B
:109A800002F0CAFB084902F0BFFA02F08BFD002881
:109A9000BCBF00F50C40A0303060F8BD30000020A5
:109AA0002C7D8E3FA00CB34500A00C4610B502F0F3
:109AB0005FFB0021044602F06BFD08B1204601E087
:109AC00004F10040054902F05BFC054902F0A4FBEB
:109AD00005F026FA034B186010BD00BF8096184BA6
:109AE00035FA8E3C3000002070B50446007902F053
:109AF0003BFB1E4902F044FC1D4D1E4E2860A07B1E
:109B000002F032FB194902F03BFCEE6068606079BC
:109B100002F02AFB184902F033FC184D2860E07B64
:109B200002F022FB114902F02BFC6860607E02F01B
:109B30001BFB134902F024FCEE60A860A07902F040
:109B400013FB0D4902F01CFC0E4D2860207C02F036
:109B50000BFB064902F014FC6860A07E02F004FBD7
:109B6000074902F00DFCEE60A86070BD0000C8421D
:109B7000880F00200000FA4400002041980F0020C8
:109B800000007A44BC0F002044F25063984203DD89
:109B9000A0F50C40A0387047034B9842BCBF00F5BD
:109BA0000C40A030704700BFB0B9FFFF2DE9F04175
:109BB000038A87890446BFB20D461F40002F2DD06F
:109BC000B7FA87F34FF00042DA40D24391B21B3B21
:109BD00021821740042BF1D8DFE803F01916131087
:109BE0000300B4F82C802E6A1FFA88F8002EE5D006
:109BF00033683046414698477668F7E72868A18E73
:109C000008E06868218F05E0A868A18F02E0E86895
:109C1000B4F84010036889B29847CFE7BDE8F081F7
:109C200090F83B3210B57BB990F83A3290F839226F
:109C3000934209D201219940B0F8404201332143B7
:109C4000A0F84012DBB2F3E710BD8379012B03D1FA
:109C5000D1F1010138BF0021D0F834315A681B8995
:109C600009B11361704753617047044B53F82030BA
:109C70001BB107289CBF1B6819807047680700202C
:109C80002DE9F0410F88002347FA03F2D2072BD5C4
:109C90008A7803F0070512F0100F18BF91F803C07F
:109CA00002F00F0618BF46EA0C06AD004FF00F0C8D
:109CB0000CFA05FC06FA05F5DC0850F82480282A81
:109CC00028EA0C0C45EA0C0540F8245005D1012285
:109CD0009A40C46824EA020205E0482A04D101221D
:109CE0009A40C4682243C2600133102BCCD1BDE836
:109CF000F081034B1A88013292B21A80704700BF7C
:109D0000FE050020F7B5294B1B78042B48D14020D5
:109D1000FCF734FB044670B12046FCF7ECFC18B9A4
:109D20000A20FCF790FCF7E7214B20461B681969D5
:109D3000FCF7E6FC0AE01E4B21461B6800901A69FE
:109D400040200323FDF7AEFE044648B3194D2868B2
:109D500041798B0703D441F00201FCF7C7FC164B95
:109D600008221A612868FCF7D5FC58B1114B124E35
:109D7000082718687761FCF7C8FC01462046FCF705
:109D8000DBFC37612046FCF7C5FC0028EAD0204602
:109D90002E68FCF7BAFC01463046FCF7CDFCE1E743
:109DA000064803B0BDE8F040FCF760BD8008002025
:109DB0007C080020A0080020000C01409D24010820
:109DC0002DE9F743124C814604F1980894F84A6053
:109DD000C6B9D9F80420002500950120294603239F
:109DE000FDF760FE074620B97EB94FF49642012682
:109DF000F1E7204629464C2204F063FE0123276048
:109E000084F84A304C344445E0D103B0BDE8F083D7
:109E1000400D0020F7B5524B524C2360FAF7CEF8B4
:109E20000120FDF770FB002800F084804E4BFF21DD
:109E300018461622256804F044FE002202704B4AA0
:109E40000121126803469707817504D541700321EB
:109E5000817502218170560704D5997D481C98753B
:109E60000320585412F00A0F0CD09A7D0421995403
:109E7000511CC9B205205854D11C02329975D2B276
:109E8000062199543A4FBA68900604D5997D481C2A
:109E9000987507205854110608D5997D0920585403
:109EA000881C01319875C9B20A205854797908295B
:109EB00001D00E2904D1997D481C98750B20585467
:109EC000997D4FF00C0E481CC0B212F0040F264EC4
:109ED000987503F801E003D00231B17510213154B7
:109EE000997D97F84571481CC0B24FF0120E002FB3
:109EF0000CBF002702F001071B4E987503F801E024
:109F00001FB10231B17513213154997D1427481CBA
:109F1000C0B298755F549305134E03D502311523D3
:109F2000B175335413480021982204F0CAFD284625
:109F3000FFF746FF0220FDF7E6FA70B10220FCF7BA
:109F40001DFA2568084C0146A06130B90090AA6846
:109F500002200323FDF7A6FDA06103B0F0BD00BF02
:109F6000F41A0020D80D0020F817002088020020E5
:109F7000C8190020400D0020A94B2DE9F7431B789C
:109F8000002B00F08181FFF78FFCA64E0546337849
:109F9000834200F07981A44C23681B78002800F0EC
:109FA000EF8063BB0420FCF7E9F9A04F014638605D
:109FB000DFF8848290B143794FF4165188F81C3051
:109FC0008368C8F82030FCF79BFB38680221FCF757
:109FD0008DFB38680421FDF7B3FA10E0944B0420A0
:109FE0001B684FF416529B7800930223FDF75AFD2D
:109FF0004379386088F81C308368C8F820302368BB
:10A000001F78012F33D10420FCF7B8F9DFF8448220
:10A010000146C8F80000DFF82092A0B143794FF460
:10A02000964189F824308368C9F82830FCF768FB2A
:10A03000D8F800003946FCF759FBD8F80000042195
:10A04000FDF77EFA13E000903B4604204FF4964261
:10A05000FDF728FD4379C8F8000089F824308368AB
:10A06000C9F828300379022B04BF724B1F70236894
:10A070001F78022F41D10420FCF780F96E4C014675
:10A08000E06288B143794FF4964184F830308368B8
:10A090006363FCF735FBE06A3946FCF727FBE06AAF
:10A0A0000421FDF74DFA0CE000903B4604204FF4EC
:10A0B0009642FDF7F7FC4379E06284F8303083681C
:10A0C0006363E76A5D4C94F84A30022B09D094F838
:10A0D0009620022A00F0D6801BB14C34002A18BF0B
:10A0E0000024574B1C6044B1204600214C2204F050
:10A0F000E8FC0223276084F84A30FFF727FC002899
:10A1000000F0BE804F4F3B78002B40F0B980082014
:10A11000FCF734F94C4C0146206090B1464B427933
:10A120004FF4614183F838208268DA63FCF7E8FA7B
:10A1300020680821FCF7DAFA20680821FDF700FA08
:10A140009EE0424B08201B684FF461429B780093CD
:10A150000346FDF7A7FC206040B1012342793B7024
:10A16000354B83F838208268DA6389E0384B1B78F6
:10A17000002B00F0858004233B70FFF74BFE7FE04F
:10A1800083B92A4FDFF8B080386898F81C10FCF7C4
:10A19000ADFA3868D8F82010FCF7B2FA3868042114
:10A1A000FCF7D7F823681B78012B10D1294FDFF873
:10A1B0008880386898F82410FCF798FA3868D8F83E
:10A1C0002810FCF79DFA38680421FCF7C2F82368D0
:10A1D0001B78022B0DD1184CE06A94F83010FCF774
:10A1E00085FAE06A616BFCF78BFAE06A0421FCF700
:10A1F000B0F8FFF7ABFB002842D0124F3B7813F0CA
:10A20000FB0F3DD0124B104C1B782BB3206808215C
:10A21000FCF79FF804233B70FFF7FCFD2EE000BF26
:10A22000F0030020F1030020F4030020F8030020D5
:10A230001C0400209D050020F8170020400D002080
:10A24000A4040020B4040020B8040020DC0B00208B
:10A25000D20B002090040020DFF83480206898F8AA
:10A260003810FCF743FA2068D8F83C10FCF748FA9D
:10A2700020680821FCF76DF804233B70002323605D
:10A28000357001E04C342CE703B0BDE8F08300BF2B
:10A29000F8170020426A10B58469A154416A026926
:10A2A0000131B1FBF2F402FB14124262426B32B193
:10A2B0001368DB0708D4BDE81040FAF719BE036D38
:10A2C000DA6842F08002DA6010BD1FB50123ADF8F4
:10A2D0000830ADF80410002301A9ADF80A30ADF83C
:10A2E0000C30ADF80620FAF75FF805B05DF804FB16
:10A2F00070B50022064631491301585CB04204D0C3
:10A300000132072AF7D1002070BD2D4C0B44082ED6
:10A310000FCB254684E80F001AD009D8022E0ED0A4
:10A32000042E15D0012E46D1264B1B685B683FE0FA
:10A33000202E3AD0402E06D0102E3CD11FE0214BCB
:10A340001B689B6802E01F4B1B681B6963602FE062
:10A350001D4B1B681B7853B1013B012B0AD9FFF73A
:10A36000F5FA002814BF4FF46143002304E04FF4D2
:10A37000165301E04FF496436B60AB601BE0134B48
:10A380001B681B7A042B16D8DFE803F008080308C3
:10A3900008000F4B6360A360032304E04FF4E13334
:10A3A0006360A36001236B7305E0064B1B68DB68E9
:10A3B000A360204670BD024870BD00BF00110108B7
:10A3C00038180020D80D0020F403002004010020DC
:10A3D000A08601000E4B1A78552A16D15A88B2F57C
:10A3E000EF6F12D11A79BE2A0FD193F8742700208B
:10A3F000EF2A0CD113F8012B5040064A9342F9D1B1
:10A40000D0F1010038BF002070470020704770472E
:10A4100000F8010878FF01084A4B55222DE9F34165
:10A420001A704FF4EF625A80BE221A71EF2283F83D
:10A430007427002283F8752711461E46B35C01324B
:10A44000B2F5EF6F81EA0301F8D13E4B3E4A83F843
:10A4500075173E4B04275A6002F188325A6000207B
:10A46000013F17F0FF075DD0384B3422384CDA60DB
:10A47000C4F309037BB1331903F17843A3F5FC332B
:10A48000D3F800804FF4005000230193FAF780F9CD
:10A490000428E5D11BE04FF43020FAF779F90428BD
:10A4A000DED12A4D4FF430202B6943F002032B619B
:10A4B0006C612B6943F040032B61FAF769F92A6953
:10A4C00041F6FD73134004282B61D4D0C8E71F4D1B
:10A4D0004FF400502B6943F001032B611FFA88F3FE
:10A4E0002380FAF755F9042812D1A31C0193019B8C
:10A4F0004FEA1848A3F800804FF40050FAF748F9E3
:10A500002B6941F6FE721A4004282A6106D0A7E79B
:10A510002B6941F6FE721A402A61A1E70D4B043403
:10A520009C42A5D1094B04281A6942F080021A61A5
:10A5300002D1FFF74FFF10B90A20FCF7BBF802B0B9
:10A54000BDE8F081C81900202301674500200240C2
:10A5500000F8010878FF01088A2802D08E2809D067
:10A560007047094B1B689B060DD5084B1B7853B9E8
:10A57000074A03E0054B1B782BB9064A064B1A60C5
:10A58000064B2D221A707047880200208C04002090
:10A590005C0400203004002098040020A104002066
:10A5A00070B5184E1023736140F080000C461546BC
:10A5B000FAF796FE144B9B894FF47A737DB1124AD9
:10A5C0001189880706D5FF2191810F4A1189C90792
:10A5D00011D509E05A1E92B223B9FFF78AFB102366
:10A5E000336170BD1346EAE7928992B20CB12270D2
:10A5F0000134013DE2E75A1E92B2002BEDD0134622
:10A60000E3E700BF000801400030014070B5054C91
:10A6100010250E466561FAF763FE3046FAF760FED4
:10A62000256170BD0008014008B5284B80211A88BB
:10A630006B2022F040021204120C1A801A8822F0B9
:10A6400038021204120C42F030021A801A8892B2B8
:10A6500042F040021A80FFF7D9FF9620FBF7F3FF84
:10A6600003216820FFF7D2FF9620FBF7ECFF0321C0
:10A670006B20FFF7CBFF0120FBF7DAFF10216A20E8
:10A68000FFF7C4FF0120FBF7D3FF00216C20FFF789
:10A69000BDFF0120FBF7CCFF00211920FFF7B6FF1B
:10A6A0000120FBF7C5FF10211C20FFF7AFFF0120A1
:10A6B000FBF7BEFF1B201821FFF7A8FF0120FBF7C7
:10A6C000B7FF034B01221A7008BD00BF00300140E4
:10A6D000FC050020224B70B519684FF47A73B1FB6A
:10A6E000F3F1204B20481A78204B214D1B78F9F7C5
:10A6F00037FB204B20481968204B2E68B1FBF3F143
:10A70000F9F72EFB00241E4BE2B253F8221049B198
:10A71000012303FA02F2324202D01A48F9F720FB71
:10A720000134F0E72A6892070DD5174A17481278C6
:10A7300003EB8203196AF9F713FB154B197A11B170
:10A740001448F9F70DFB1448FCF790F8BDE8704089
:10A75000124B1348198800224FF4EF63F9F700BB3E
:10A76000C419002008040020BD2601088000002034
:10A770008802002084000020FB26010840420F00D0
:10A7800070110108C61F01086D210020192701085A
:10A790008C02002023270108B82701084403002069
:10A7A0002727010870B50E462021154604F0BDF993
:10A7B0000446B8B1441C204604F019FAB0F5617F94
:10A7C00005DB40F634039842A8BF184601E04FF479
:10A7D00061701923A0F5617090FBF3F030702B7855
:10A7E00001332B702046202104F09FF90446B8B1B4
:10A7F000441C204604F0FBF9B0F5617F05DB40F610
:10A8000034039842A8BF184601E04FF46170192341
:10A81000A0F5617090FBF3F070702B7801332B7012
:10A82000204670BD70B586B0054604F08BF9C0B205
:10A8300008BB044606236343444A03F58873126841
:10A8400019201344591D4D789A7A454305F56175D1
:10A850005B7900958D78684300F561700190C87848
:10A86000029009793A48039121460134F9F778FAC0
:10A870000C2CDFD168E0284604F0B9F90B285FDC26
:10A8800006267043314B00F588701E68202106446F
:10A890000023681C8DF8173004F047F9741D054635
:10A8A00058B1451C284604F0A2F9032805D89DF8A4
:10A8B0001730607101338DF817302846202104F0DD
:10A8C00034F9054658B1451C284604F090F90D2886
:10A8D00005D870719DF8173001338DF81730284670
:10A8E000611C0DF11702FFF75DFF202104F01DF937
:10A8F000054658B1451C284604F079F90C2805D8BE
:10A900009DF81730E07001338DF81730284620216C
:10A9100004F00BF950B1013004F069F90D2805D8A5
:10A920009DF81730207101338DF817309DF81730DE
:10A93000062B09D020460021062204F0C2F803E0CD
:10A9400004480C21F9F70CFA06B070BD180200207B
:10A950005927010812220108F0B585B0074604F016
:10A96000F1F8C0B2E0B90446324B04F11C021B6896
:10A97000192003EB8203591D8D785A79454305F55B
:10A9800061759B790095C978484300F56170019025
:10A99000214629480134F9F7E3F9282CE4D146E0AF
:10A9A000384604F024F927283DDC224B00F11C0630
:10A9B0001B68781C03EB8606202100238DF80F30DE
:10A9C00004F0B3F8751D044658B1441C204604F049
:10A9D0000EF9152805D870719DF80F3001338DF8E8
:10A9E0000F302046202104F0A0F8044658B1441C42
:10A9F000204604F0FCF80D2805D89DF80F3068704B
:10AA000001338DF80F302046A91C0DF10F02FFF71E
:10AA1000C9FE9DF80F30042B09D0284600210422DE
:10AA200004F04FF803E005482821F9F799F905B03B
:10AA3000F0BD00BF1802002079270108122201088A
:10AA40002DE9F041002407462546104B3946E658CB
:10AA500004EB0308304604F0B1F858B10C48314615
:10AA6000F9F77EF940460021FAF754F80948F9F75A
:10AA700077F901351434B4F52F6FE6D125B90648BE
:10AA8000BDE8F041FBF7F2BEBDE8F08138120108E5
:10AA9000EA270108B82701088E2701082DE9F74F9A
:10AAA000044604F04FF8054620B1012818D1237858
:10AAB0002A2B15D15548FBF7D9FE0024544B554895
:10AAC000E618E158F9F74CF930462946FAF722F82A
:10AAD00014345148FBF7CAFEB4F52F6FEED192E063
:10AAE00020463D2104F021F8002800F0878003462D
:10AAF00013F8012C202A01D1013BF9E7451C284617
:10AB0000C4EB030A04F073F883462846FEF797FD6A
:10AB10000026054614237343DFF8F49053F80970B8
:10AB200003EB0908384604F00DF803461A462046A0
:10AB30003946019304F00EF8019B002855D15FFAC5
:10AB40008AF29A4251D1D8F80C0001F011FB01466B
:10AB5000284601F013FD002845D0D8F8100001F078
:10AB600007FB0146284601F0FFFC00283BD0B8F85F
:10AB700004309B064FF0140303FB0696B28858BFBF
:10AB80005D4614062946B36806D524484FF4E074A0
:10AB900090F8540704FB0033D00504D520480A245C
:10ABA000007804FB003302F03F02042A0BD004D8E3
:10ABB000013A012A0CD819700AE0102A05D0202A7F
:10ABC00005D0082A04D1198002E0196000E01D6058
:10ABD00039461448F9F7C4F83046002103B0BDE8FF
:10ABE000F04FF9F797BF104803E001368C2E91D152
:10ABF0000E4803B0BDE8F04FFBF738BE204603B067
:10AC0000BDE8F04F1CE703B0BDE8F08FA6270108B0
:10AC100038120108EA270108B8270108C8190020DE
:10AC20003C0C0020BB270108C62701088E2701081D
:10AC300038B5114B114D1A78114C29688AB1226828
:10AC40000244914217D300201870FBF706FD2B68D1
:10AC500023600C4B1A780AB1013A1A700123237150
:10AC600038BD2268C832914205D301201870FBF725
:10AC7000F4FC2B68236038BD3B0D0020C419002074
:10AC800048180020CE02002037B5224D8DF807303D
:10AC90006B798DF8062002AA8DF804008DF8051056
:10ACA0001A4412F8042C443AD2B20F2A2BD81A496B
:10ACB000022B01EB4202B2F84C4003D814B12046FB
:10ACC000FFF7B6FF6B79134A022B09D9134B1968AA
:10ACD0001368091B8B4203D200235371104A13706F
:10ACE0002B79012B00D09CB96B79022B02D8094A31
:10ACF000013353710B4B00202871187003B0BDE86D
:10AD00003040FBF7AABC022B4FF0C804D7D9D9E7D3
:10AD100003B030BD4818002070110108C41900208C
:10AD2000CE0200203B0D002030B585B004AC0025DC
:10AD300024F8025D0091ADF8060021461020FBF7D3
:10AD4000A9FD9DF806002146FBF7A4FD9DF807002C
:10AD50002146FBF79FFD9DF800002146FBF79AFD79
:10AD60009DF801002146FBF795FD9DF80200214664
:10AD7000FBF790FD9DF803002146FBF78BFD9DF846
:10AD80000E002946C043C0B2FBF784FD024B1A688F
:10AD9000024B1A6005B030BDC4190020C804002061
:10ADA0000449054B0968002218701A6159611A7626
:10ADB000704700BFC419002080080020104B0430E9
:10ADC00033F91030B3F5617F05DB40F6330293426F
:10ADD000A8BF134601E04FF461730878192250436D
:10ADE00000F28330984208DA4878504300F283300A
:10ADF0009842B4BF0020012070470020704700BF78
:10AE00006205002070B5064600240A4BE518AA88A2
:10AE100016420AD0E1580848F8F7A2FF2846002158
:10AE2000F9F778FE0548FBF721FD1434B4F52F6FD0
:10AE3000EBD170BD38120108E6270108B8270108D8
:10AE40002DE9F041FFF7C6FA10B90A20FBF732FCF2
:10AE5000AF4C4FF4EF622046AE4903F029FE94F860
:10AE600054374FF4E072022B84BF002384F8543728
:10AE700094F85437A84E02FB034303F5057393F887
:10AE800050203360022A84BF002283F8502093F8B8
:10AE90005030A24A13700A2202FB0343A04A03F275
:10AEA00056731360A36842F201021A403AB944F2A1
:10AEB00008021A401AB9964A43F400539360A368F3
:10AEC000DA0703D54FF40050FEF7E5FCA3685B04F6
:10AED00009D50820FEF7DFFC4FF40050FEF7DBFC3D
:10AEE0000120FEF7D8FCA3681F0706D54FF40050D9
:10AEF000FEF7D1FC0120FEF7CEFCA3689D040ED521
:10AF00004FF40040FEF7C7FC4FF40060FEF7C3FCAF
:10AF10004FF48030FEF7BFFC4020FEF7BCFCA36876
:10AF2000580603D54FF48030FEF7B5FC7D4D7E4BBF
:10AF30002F461D60F9F742F87C4B05F11C020120F9
:10AF40001A60FFF7D5F901460120FCF731FA002815
:10AF500049D00220FFF7CCF901460220FCF728FA7D
:10AF6000002840D02020FFF7C3F901462020FCF73D
:10AF70001FFAA368190601D5002834D01020FFF766
:10AF8000B7F901461020FCF713FAA3681A0700D599
:10AF900048B30420FFF7ACF901460420FCF708FA97
:10AFA00030B90820FFF7A4F901460820FCF700FAA1
:10AFB000A3685B0503D400231A46194609E000285C
:10AFC000F9D110E079B90121C00708D40C33242B42
:10AFD0000BD057481844007A8507F5D5F2E70132BF
:10AFE000D2B2022AF2D9FBF79EFFFBF745FA514D88
:10AFF000514B32681D60514B101D186002F17501F4
:10B000000023A846CD5C55B901EB030E9EF802C0A3
:10B010009EF803E0F44502D2494B1D7002E0043370
:10B02000A02BEFD1474B48490B60484950330B6088
:10B030001178474B012903D0022903D0454902E08A
:10B04000454900E045491960454B02F5D9721A603F
:10B05000FEF74AFD3668434B06F5D3721A60424B41
:10B0600000229A80414B424A424D136006F5B3726A
:10B070002A60A3F122026A602E333F4A06F5D77197
:10B08000EB6006F5D87311606B61C5F808802F611D
:10B09000B4F8F00001F068F8E861B4F8F20001F0EB
:10B0A00063F896F8583005F118022B7696F874304C
:10B0B00028626B7694F82531C5F8348085F8243001
:10B0C0002E4BB6F862011A60331DAB622C4B06F1B1
:10B0D00060021A6006F16403EB6206F25D132B63F3
:10B0E00001F046F80146274801F04AF9264901F0E7
:10B0F00093F8264B26491860F06D01F08DF8014653
:10B100004FF07C5001F03CF9224B1860BDE8F08113
:10B11000C819002000F80108180200203C0C00208B
:10B12000E0030020D81A002004010020D80D0020E0
:10B1300048000020981A0020340C0020380C002011
:10B140002C000020BC1A002034020020F403002050
:10B150007C000020AD8C0008198B0008358F00089A
:10B16000D4030020C01900204C080020C01A002081
:10B17000A402002050180020EC030020D802002078
:10B1800034030020000061444C3D0F44D0030020F4
:10B19000DB0F49402403002010B50446204603F08D
:10B1A000D1FC10F0FF0F07D10B4B0C4893F854174C
:10B1B000BDE81040F8F7D4BD204603F018FD022882
:10B1C00008D8054B064C83F85407FFF725F9FFF71D
:10B1D00037FEE3E710BD00BFC81900209522010823
:10B1E000772401082DE9F04F844985B0054603F026
:10B1F00071FC8349002828460CBF0124072403F072
:10B2000069FC80490028284608BF022403F062FC3C
:10B21000002808BF0424E10740F1BE807A48F8F70F
:10B220009FFD0020F9F7C6FA784F7948F8F798FDA6
:10B230007848F8F795FD7A79774B013A774853F8D3
:10B240002210F8F78DFD3869002101F079F9002806
:10B250005CD13D460646D5F810800021404601F0FD
:10B260006FF900284ED101366D483146D5F814B03B
:10B27000D5F818A0D5F81C90F8F772FD40460021CB
:10B2800001F068F910B16748F8F76AFD6946404671
:10B29000F8F7D8FE01466448F8F762FD58460021E9
:10B2A00001F058F910B15F48F8F75AFD6946584661
:10B2B000F8F7C8FE01465C48F8F752FD50460021F9
:10B2C00001F048F910B15748F8F74AFD6946504671
:10B2D000F8F7B8FE01465448F8F742FD4846002109
:10B2E00001F038F910B14F48F8F73AFD6946484681
:10B2F000F8F7A8FE01464D48F8F732FD0C2E05F18F
:10B300001005A8D14A48711CF8F72AFD4948F8F7FA
:10B3100027FD494DD7F8088055F8041F19B1474853
:10B32000F8F71EFDF8E70D46454B53F8256056B17A
:10B330000123AB4013EA080F03D042483146F8F727
:10B340000FFD0135F0E74048F8F70AFD31467B185C
:10B3500093F8103104AA13443C4A8A5C013108294D
:10B3600003F8102CF3D10023694639488DF80830D2
:10B37000F8F7F6FC3748F8F7F3FC3748F9F748FADE
:10B380003648F8F7EDFC3448F8F7A6FD3448F8F7EE
:10B39000E7FC4020FFF736FDA2071AD53148F8F741
:10B3A000DFFC3148F8F7DCFC2B48FFF7F5FE2F48AF
:10B3B000F8F7D6FC2848FFF7CFFA2D48F8F7D0FC6D
:10B3C0002548FFF72FFA2648F8F7CAFC8020FFF738
:10B3D00019FD63070FD52748F8F7C2FC2648F8F790
:10B3E000BFFC1D48FBF732FC1D48F8F7B9FC4FF4D1
:10B3F0008070FFF707FD05B0BDE8F08F4A2801080F
:10B400003B2F01085128010857280108C8190020BE
:10B410006528010877280108DC1101088328010844
:10B420008E2801084624010820270108412201082E
:10B4300096280108A8280108740F0108B8280108F7
:10B44000780F0108C6280108D32801080D2A010831
:10B45000DF280108E828010877240108F4280108FA
:10B46000B827010802290108152901082329010824
:10B470002D2901083C2901084D29010801480249EC
:10B48000FEF794BB00080040F41800200148024970
:10B49000FEF78CBB00040040D01800204FF0804025
:10B4A0000149FEF783BB00BFAC18002001480249E8
:10B4B000FEF77CBB002C014088180020014802499F
:10B4C000FEF774BB002C01408818002038B5204CD2
:10B4D000D4F8E0301D88ADB2AA0618D5D4F8BC2047
:10B4E0001AB1988880B2904711E09B88D4F8AC20BC
:10B4F000D4F8A410DBB28B54D4F8AC20D4F89C3030
:10B500000132B2FBF3F103FB1123C4F8AC302B067C
:10B510001DD5D4F8B820D4F8B4100D4B8A4210D001
:10B52000D3F8A800D3F8E010805C0132C0B2888064
:10B53000D3F8A010B2FBF1F001FB1022C3F8B82041
:10B5400038BDD3F8E030DA6822F08002DA6038BD26
:10B55000881800200F4BD3F834211188090618D51C
:10B56000D3F80C11D3F8080181420ED0D3F8FC00B7
:10B57000405C0131C0B29080D3F8F420B1FBF2F00E
:10B5800002FB1011C3F80C117047D36823F080033D
:10B59000D3607047881800200C480D4B4FF40052C0
:10B5A0005A60D0F818214FF6FE7311680B401360F3
:10B5B000D0F80821D0F80C319A4202D0E430F9F7E3
:10B5C00097BC012380F82831704700BF88180020FD
:10B5D00000000240084A13689B020BD5074B00216C
:10B5E000197007494FF6FE73086803400B604FF46B
:10B5F00000135360704700BF000002406A21002022
:10B600006C00024010B50C4B1A78510713D50B4C47
:10B6100022F004021A70A3685B050CD5FEF7ACFC9F
:10B6200004200121FBF75EFF28B104F59670BDE808
:10B630001040FEF7C5BB10BD6C210020C8190020CA
:10B6400070B5FAF7A9FC38B3144C237A0BB9A38070
:10B6500070BD134D2E78C6F38000FAF7AFFC90B1A1
:10B66000104B46F002061A680F4B51892E70198054
:10B670005189598052899A800C4A12685288DA801E
:10B68000E3880133E380FAF773FC10B92B785B078A
:10B6900002D4BDE87040B5E770BD00BF4C08002083
:10B6A0006C2100204808002062050020C0190020FD
:10B6B0000F4B1A6842F001021A6059680D4A0A409D
:10B6C0005A601A6822F0847222F480321A601A6872
:10B6D00022F480221A605A6822F4FE025A604FF463
:10B6E0001F029A60044B4FF000629A60704700BFDF
:10B6F000001002400000FFF800ED00E0024B1A6865
:10B7000001321A60704700BFC419002008B5084B09
:10B71000B3F8D80093F87C270023D9B2914204D221
:10B72000044921F813000133F7E7FBF708F9FEE7B6
:10B73000C41900204221002081F0004102E000BF36
:10B7400083F0004330B54FEA41044FEA430594EAE1
:10B75000050F08BF90EA020F1FBF54EA000C55EA1C
:10B76000020C7FEA645C7FEA655C00F0E2804FEAED
:10B770005454D4EB5555B8BF6D420CDD2C4480EACF
:10B78000020281EA030382EA000083EA010180EAFF
:10B79000020281EA0303362D88BF30BD11F0004F4D
:10B7A0004FEA01314FF4801C4CEA113102D0404283
:10B7B00061EB410113F0004F4FEA03334CEA1333BE
:10B7C00002D0524263EB430394EA050F00F0A780D6
:10B7D000A4F10104D5F1200E0DDB02FA0EFC22FAD1
:10B7E00005F2801841F1000103FA0EF2801843FAC5
:10B7F00005F359410EE0A5F120050EF1200E012AB6
:10B8000003FA0EFC28BF4CF0020C43FA05F3C018F3
:10B8100051EBE37101F0004507D54FF0000EDCF16C
:10B82000000C7EEB00006EEB0101B1F5801F1BD315
:10B83000B1F5001F0CD349085FEA30004FEA3C0C19
:10B8400004F101044FEA445212F5800F80F09A800F
:10B85000BCF1004F08BF5FEA500C50F1000041EB13
:10B86000045141EA050130BD5FEA4C0C404141EB17
:10B87000010111F4801FA4F10104E9D191F0000F3E
:10B8800004BF01460020B1FA81F308BF2033A3F1C1
:10B890000B03B3F120020CDA0C3208DD02F1140CB8
:10B8A000C2F10C0201FA0CF021FA02F10CE002F1F3
:10B8B0001402D8BFC2F1200C01FA02F120FA0CFCEC
:10B8C000DCBF41EA0C019040E41AA2BF01EB045135
:10B8D000294330BD6FEA04041F3C1CDA0C340EDC33
:10B8E00004F11404C4F1200220FA04F001FA02F376
:10B8F00040EA030021FA04F345EA030130BDC4F134
:10B900000C04C4F1200220FA02F001FA04F340EA28
:10B910000300294630BD21FA04F0294630BD94F0D9
:10B92000000F83F4801306BF81F480110134013DC0
:10B930004EE77FEA645C18BF7FEA655C29D094EA31
:10B94000050F08BF90EA020F05D054EA000C04BFAF
:10B950001946104630BD91EA030F1EBF002100209A
:10B9600030BD5FEA545C05D14000494128BF41F039
:10B97000004130BD14F580043CBF01F5801130BD9D
:10B9800001F0004545F0FE4141F470014FF0000028
:10B9900030BD7FEA645C1ABF194610467FEA655CD9
:10B9A0001CBF0B46024650EA013406BF52EA03357B
:10B9B00091EA030F41F4002130BD00BF90F0000F69
:10B9C00004BF0021704730B54FF4806404F13204A5
:10B9D0004FF000054FF0000150E700BF90F0000F5E
:10B9E00004BF0021704730B54FF4806404F1320485
:10B9F00010F0004548BF40424FF000013EE700BF55
:10BA000042004FEAE2014FEA31014FEA02701FBFE4
:10BA100012F07F4393F07F4F81F06051704792F0B6
:10BA2000000F14BF93F07F4F704730B54FF4607430
:10BA300001F0004521F0004120E700BF50EA01027B
:10BA400008BF704730B54FF000050AE050EA010228
:10BA500008BF704730B511F0004502D5404261EB98
:10BA600041014FF4806404F132045FEA915C3FF4D9
:10BA7000DCAE4FF003025FEADC0C18BF03325FEA72
:10BA8000DC0C18BF033202EBDC02C2F1200300FA27
:10BA900003FC20FA02F001FA03FE40EA0E0021FA4C
:10BAA00002F11444C1E600BF70B54FF0FF0C4CF436
:10BAB000E06C1CEA11541DBF1CEA135594EA0C0FEC
:10BAC00095EA0C0F00F0DEF82C4481EA030621EA27
:10BAD0004C5123EA4C5350EA013518BF52EA033562
:10BAE00041F4801143F4801338D0A0FB02CE4FF014
:10BAF0000005E1FB02E506F00042E0FB03E54FF044
:10BB00000006E1FB03569CF0000F18BF4EF0010E3B
:10BB1000A4F1FF04B6F5007F64F5407404D25FEA37
:10BB20004E0E6D4146EB060642EAC62141EA5551EA
:10BB30004FEAC52040EA5E504FEACE2EB4F1FD0C2C
:10BB400088BFBCF5E06F1ED8BEF1004F08BF5FEAAA
:10BB5000500E50F1000041EB045170BD06F000465C
:10BB600046EA010140EA020081EA0301B4EB5C0409
:10BB7000C2BFD4EB0C0541EA045170BD41F4801101
:10BB80004FF0000E013C00F3AB8014F1360FDEBF26
:10BB9000002001F0004170BDC4F10004203C35DA02
:10BBA0000C341BDC04F11404C4F1200500FA05F385
:10BBB00020FA04F001FA05F240EA020001F0004226
:10BBC00021F0004110EBD37021FA04F642EB06019C
:10BBD0005EEA430E08BF20EAD37070BDC4F10C04C6
:10BBE000C4F1200500FA04F320FA05F001FA04F28A
:10BBF00040EA020001F0004110EBD37041F1000176
:10BC00005EEA430E08BF20EAD37070BDC4F1200580
:10BC100000FA05F24EEA020E20FA04F301FA05F2E8
:10BC200043EA020321FA04F001F0004121FA04F290
:10BC300020EA020000EBD3705EEA430E08BF20EA60
:10BC4000D37070BD94F0000F0FD101F0004640009A
:10BC500041EB010111F4801F08BF013CF7D041EA1C
:10BC6000060195F0000F18BF704703F00046520020
:10BC700043EB030313F4801F08BF013DF7D043EAF1
:10BC80000603704794EA0C0F0CEA135518BF95EAA7
:10BC90000C0F0CD050EA410618BF52EA4306D1D12E
:10BCA00081EA030101F000414FF0000070BD50EA4D
:10BCB000410606BF1046194652EA430619D094EAD7
:10BCC0000C0F02D150EA013613D195EA0C0F05D1C1
:10BCD00052EA03361CBF104619460AD181EA030115
:10BCE00001F0004141F0FE4141F470014FF00000CD
:10BCF00070BD41F0FE4141F4780170BD70B54FF068
:10BD0000FF0C4CF4E06C1CEA11541DBF1CEA1355E7
:10BD100094EA0C0F95EA0C0F00F0A7F8A4EB0504C9
:10BD200081EA030E52EA03354FEA013100F08880C0
:10BD30004FEA03334FF0805545EA131343EA126389
:10BD40004FEA022245EA111545EA10654FEA00263E
:10BD50000EF000419D4208BF964244F1FD0404F5F7
:10BD6000407402D25B084FEA3202B61A65EB030553
:10BD70005B084FEA32024FF480104FF4002CB6EB10
:10BD8000020E75EB030E22BFB61A754640EA0C0090
:10BD90005B084FEA3202B6EB020E75EB030E22BFD0
:10BDA000B61A754640EA5C005B084FEA3202B6EB11
:10BDB000020E75EB030E22BFB61A754640EA9C00D0
:10BDC0005B084FEA3202B6EB020E75EB030E22BFA0
:10BDD000B61A754640EADC0055EA060E18D04FEA5E
:10BDE000051545EA16754FEA06164FEAC30343EAFE
:10BDF00052734FEAC2025FEA1C1CC0D111F4801FCB
:10BE00000BD141EA00014FF000004FF0004CB6E7C3
:10BE100011F4801F04BF01430020B4F1FD0C88BF62
:10BE2000BCF5E06F3FF6AFAEB5EB030C04BFB6EB6D
:10BE3000020C5FEA500C50F1000041EB045170BD60
:10BE40000EF0004E4EEA113114EB5C04C2BFD4EB8D
:10BE50000C0541EA045170BD41F480114FF0000E11
:10BE6000013C90E645EA060E8DE60CEA135594EA8D
:10BE70000C0F08BF95EA0C0F3FF43BAF94EA0C0F90
:10BE80000AD150EA01347FF434AF95EA0C0F7FF405
:10BE900025AF104619462CE795EA0C0F06D152EA59
:10BEA00003353FF4FDAE1046194622E750EA41063D
:10BEB00018BF52EA43067FF4C5AE50EA41047FF44E
:10BEC0000DAF52EA43057FF4EBAE12E74FEA4102B1
:10BED00012F5001215D211D56FF47873B3EB6252DC
:10BEE00012D94FEAC12343F0004343EA505311F003
:10BEF000004F23FA02F018BF404270474FF0000095
:10BF0000704750EA013005D111F0004008BF6FF0D2
:10BF1000004070474FF00000704700BF4A0011D248
:10BF200012F5001211D20DD56FF47873B3EB625293
:10BF30000ED44FEAC12343F0004343EA505323FA9F
:10BF400002F070474FF00000704750EA013002D114
:10BF50004FF0FF3070474FF0000070474FEA41024A
:10BF6000B2F1E04324BFB3F5001CDCF1FE5C0DD957
:10BF700001F0004C4FEAC0024CEA5070B2F1004FA1
:10BF800040EB830008BF20F00100704711F0804FA4
:10BF900021D113F13872BCBF01F00040704741F469
:10BFA00080114FEA5252C2F11802C2F1200C10FA6D
:10BFB0000CF320FA02F018BF40F001004FEAC12351
:10BFC0004FEAD32303FA0CFC40EA0C0023FA02F3F5
:10BFD0004FEA4303CCE77FEA625307D150EA0133CB
:10BFE0001EBF4FF0FE4040F44000704701F000409B
:10BFF00040F0FE4040F40000704700BF80F0004079
:10C0000002E000BF81F0004142001FBF5FEA410330
:10C0100092EA030F7FEA226C7FEA236C6AD04FEA30
:10C020001262D2EB1363C1BFD21841404840414075
:10C03000B8BF5B42192B88BF704710F0004F40F427
:10C04000000020F07F4018BF404211F0004F41F443
:10C05000000121F07F4118BF494292EA030F3FD00F
:10C06000A2F1010241FA03FC10EB0C00C3F1200322
:10C0700001FA03F100F0004302D5494260EB4000B1
:10C08000B0F5000F13D3B0F1807F06D340084FEA1C
:10C09000310102F10102FE2A51D2B1F1004F40EB11
:10C0A000C25008BF20F0010040EA03007047490079
:10C0B00040EB000010F4000FA2F10102EDD1B0FA44
:10C0C00080FCACF1080CB2EB0C0200FA0CF0AABF39
:10C0D00000EBC25052421843BCBFD04018437047D7
:10C0E00092F0000F81F4000106BF80F400000132DD
:10C0F000013BB5E74FEA41037FEA226C18BF7FEAB4
:10C10000236C21D092EA030F04D092F0000F08BFF5
:10C110000846704790EA010F1CBF0020704712F0DC
:10C120007F4F04D1400028BF40F00040704712F11B
:10C1300000723CBF00F50000704700F0004343F080
:10C14000FE4040F4000070477FEA226216BF0846B6
:10C150007FEA23630146420206BF5FEA412390EA79
:10C16000010F40F4800070474FF0000304E000BF6F
:10C1700010F0004348BF40425FEA000C08BF704720
:10C1800043F0964301464FF000001CE050EA0102E4
:10C1900008BF70474FF000030AE000BF50EA0102F9
:10C1A00008BF704711F0004302D5404261EB4101E6
:10C1B0005FEA010C02BF84460146002043F0B6430B
:10C1C00008BFA3F18053A3F50003BCFA8CF2083A30
:10C1D000A3EBC25310DB01FA02FC634400FA02FC39
:10C1E000C2F12002BCF1004F20FA02F243EB020040
:10C1F00008BF20F00100704702F1200201FA02FCA2
:10C20000C2F1200250EA4C0021FA02F243EB020094
:10C2100008BF20EADC7070474FF0FF0C1CEAD052D8
:10C220001EBF1CEAD15392EA0C0F93EA0C0F6FD099
:10C230001A4480EA010C400218BF5FEA41211ED077
:10C240004FF0006343EA501043EA5111A0FB013163
:10C250000CF00040B1F5000F3EBF490041EAD37138
:10C260005B0040EA010062F17F02FD2A1DD8B3F1B4
:10C27000004F40EBC25008BF20F00100704790F023
:10C28000000F0CF0004C08BF49024CEA502040EA75
:10C2900051207F3AC2BFD2F1FF0340EAC25070473B
:10C2A00040F400004FF00003013A5DDC12F1190F79
:10C2B000DCBF00F000407047C2F10002410021FAEB
:10C2C00002F1C2F1200200FA02FC5FEA310040F103
:10C2D000000053EA4C0308BF20EADC70704792F07C
:10C2E000000F00F0004C02BF400010F4000F013AB4
:10C2F000F9D040EA0C0093F0000F01F0004C02BFAF
:10C30000490011F4000F013BF9D041EA0C018FE71D
:10C310000CEAD15392EA0C0F18BF93EA0C0F0AD023
:10C3200030F0004C18BF31F0004CD8D180EA010049
:10C3300000F00040704790F0000F17BF90F0004FE2
:10C34000084691F0000F91F0004F14D092EA0C0FC4
:10C3500001D142020FD193EA0C0F03D14B0218BF57
:10C36000084608D180EA010000F0004040F0FE409D
:10C3700040F40000704740F0FE4040F44000704739
:10C380004FF0FF0C1CEAD0521EBF1CEAD15392EAB8
:10C390000C0F93EA0C0F69D0A2EB030280EA010CA8
:10C3A00049024FEA402037D04FF0805343EA111141
:10C3B00043EA10130CF000408B4238BF5B0042F19F
:10C3C0007D024FF4000C8B4224BF5B1A40EA0C0044
:10C3D000B3EB510F24BFA3EB510340EA5C00B3EB76
:10C3E000910F24BFA3EB910340EA9C00B3EBD10F64
:10C3F00024BFA3EBD10340EADC001B0118BF5FEAB6
:10C400001C1CE0D1FD2A3FF650AF8B4240EBC250DE
:10C4100008BF20F0010070470CF0004C4CEA50209F
:10C420007F32C2BFD2F1FF0340EAC250704740F4EE
:10C4300000004FF00003013A37E792F0000F00F0E0
:10C44000004C02BF400010F4000F013AF9D040EA5E
:10C450000C0093F0000F01F0004C02BF490011F4F2
:10C46000000F013BF9D041EA0C0195E70CEAD153EA
:10C4700092EA0C0F08D142027FF47DAF93EA0C0FD1
:10C480007FF470AF084676E793EA0C0F04D14B02B5
:10C490003FF44CAF08466EE730F0004C18BF31F067
:10C4A000004CCAD130F000427FF45CAF31F0004361
:10C4B0007FF43CAF5FE700BF4FF0FF3C06E000BFFA
:10C4C0004FF0010C02E000BF4FF0010C4DF804CD1D
:10C4D0004FEA40024FEA41037FEA226C18BF7FEA2D
:10C4E000236C11D001B052EA530C18BF90EA010F2F
:10C4F00058BFB2EB030088BFC81738BF6FEAE170BE
:10C5000018BF40F0010070477FEA226C02D15FEA59
:10C51000402C05D17FEA236CE4D15FEA412CE1D0C5
:10C520005DF8040B704700BF844608466146FFE78C
:10C530000FB5FFF7C9FF002848BF10F1000F0FBD6E
:10C540004DF808EDFFF7F4FF0CBF012000205DF867
:10C5500008FB00BF4DF808EDFFF7EAFF34BF0120EC
:10C5600000205DF808FB00BF4DF808EDFFF7E0FF85
:10C5700094BF012000205DF808FB00BF4DF808EDD6
:10C58000FFF7D2FF94BF012000205DF808FB00BF39
:10C590004DF808EDFFF7C8FF34BF012000205DF81B
:10C5A00008FB00BF4FEA4002B2F1FE4F0FD34FF03D
:10C5B0009E03B3EB12620DD94FEA002343F0004310
:10C5C00010F0004F23FA02F018BF404270474FF0BE
:10C5D0000000704712F1610F01D1420205D110F045
:10C5E000004008BF6FF0004070474FF000007047F8
:10C5F00042000ED2B2F1FE4F0BD34FF09E03B3EBCD
:10C60000126209D44FEA002343F0004323FA02F0F8
:10C6100070474FF00000704712F1610F01D14202E4
:10C6200002D14FF0FF3070474FF00000704700BF5D
:10C6300073B96AB9002908BF0028BCBF00204FF0B9
:10C640000041C4BF6FF000414FF0FF3000F03CB834
:10C6500082B0EC462DE9005000F006F8DDF804E069
:10C6600002B00CBC704700BF2DE9704F089E144605
:10C670001D468046894600F029F804FB01F3A4FB1F
:10C6800000AB00FB05329344B8EB0A0869EB0B09D9
:10C69000C6E90089BDE8708F2DE9704F089E1446E9
:10C6A0001D468046894600F061F900FB05F5A0FBB8
:10C6B00004AB04FB0154A344B8EB0A0869EB0B0973
:10C6C000C6E90089BDE8708F704700BF00292DE9D9
:10C6D000F00FC0F2A1800024002BC0F29880154614
:10C6E00006460F46002B3FD18A4258D9B2FA82F350
:10C6F0004BB1C3F1200201FA03F720FA02F29D4088
:10C7000000FA03F61743290CB7FBF1F201FB12778D
:10C71000A8B200FB02F34FEA164C4CEA0747BB42B3
:10C7200009D97F1902F1FF3C80F00581BB4240F23C
:10C730000281023A2F44FF1AB7FBF1F301FB137198
:10C7400000FB03F0B6B246EA0141884208D9491914
:10C7500003F1FF3780F0F180884240F2EE80023B27
:10C7600043EA0242002303E08B420AD900231A461F
:10C770001046194614B1404261EB4101BDE8F00F8B
:10C780007047B3FA83F8B8F1000F40F088808B420D
:10C7900002D3824200F2E28000230122E8E712B9CC
:10C7A0000123B3FBF2F5B5FA85F2002A3AD17F1BDB
:10C7B000280C1FFA85FC0123B7FBF0F100FB117771
:10C7C0000CFB01F24FEA164848EA0747BA4207D97C
:10C7D0007F1901F1FF3802D2BA4200F2C48041460B
:10C7E000BF1AB7FBF0F200FB12700CFB02FCB6B2F2
:10C7F00046EA0040844507D9401902F1FF3702D2CA
:10C80000844500F2AE803A4642EA0142B0E7E44392
:10C81000524263EB430362E7404261EB41014FF058
:10C82000FF3459E79540C2F1200927FA09F126FAA9
:10C8300009F99740280CB1FBF0F800FB18111FFA1A
:10C8400085FC0CFB08F349EA07094FEA194747EA58
:10C8500001418B4206FA02F608D9491908F1FF3264
:10C860007AD28B4278D9A8F102082944C91AB1FBBF
:10C87000F0F300FB13170CFB03F21FFA89F949EAE6
:10C880000747BA4207D97F1903F1FF3160D2BA4294
:10C890005ED9023B2F44BF1A43EA08438CE7C8F134
:10C8A000200225FA02F103FA08FC27FA02F320FA23
:10C8B00002F207FA08F741EA0C0C4FEA1C49B3FBF5
:10C8C000F9F109FB11331FFA8CFA0AFB01FB17433C
:10C8D0003A0C42EA03439B4505FA08F008D913EBEA
:10C8E0000C0301F1FF3235D29B4533D90239634441
:10C8F000CBEB0303B3FBF9F209FB12330AFB02FA99
:10C90000BFB247EA0347BA4508D917EB0C0702F153
:10C91000FF331BD2BA4519D9023A674442EA0145AE
:10C92000A5FB0001CAEB07078F424FF000030AD3B3
:10C9300005D02A461CE76246FDE63B4610E706FAAC
:10C9400008F68642F5D26A1E002311E71A46E5E78B
:10C950000B46A0E71146CBE7904687E743464246A1
:10C9600006E7023A50E702392F4439E72DE9F00F84
:10C97000144605460E46002B43D18A4253D9B2FADB
:10C9800082F757B1C7F1200620FA06F601FA07F33D
:10C9900002FA07F400FA07F51E43210CB6FBF1F288
:10C9A00001FB1266A0B200FB02F32F0C47EA064619
:10C9B000B34209D9361902F1FF3780F0FD80B34246
:10C9C00040F2FA80023A2644F61AB6FBF1F301FB74
:10C9D000136100FB03F0ADB245EA0141884208D97A
:10C9E000091903F1FF3680F0E980884240F2E680C1
:10C9F000023B43EA0242002310461946BDE8F00F0D
:10CA000070478B424CD8B3FA83F6002E4FD18B423D
:10CA100002D3824200F2DD80BDE8F00F0023012244
:10CA200010461946704712B90124B4FBF2F4B4FA67
:10CA300084F2002A40F08280091B260CA7B2012351
:10CA4000B1FBF6F006FB101107FB00F24FEA154CA4
:10CA50004CEA01418A4207D9091900F1FF3C02D290
:10CA60008A4200F2C8806046891AB1FBF6F206FBE2
:10CA7000121107FB02F7ADB245EA0145AF4208D9F2
:10CA80002C1902F1FF3180F09B80A74240F2988080
:10CA9000023A42EA004210461946BDE8F00F7047DC
:10CAA00000231A4610461946BDE8F00F7047C6F13C
:10CAB000200522FA05F703FA06F421FA05F301FA34
:10CAC00006FB20FA05F53C434FEA1448B3FBF8FC9B
:10CAD00008FB1C331FFA84F909FB0CFA45EA0B0B1F
:10CAE0004FEA1B4545EA03439A4502FA06F204D988
:10CAF0001B190CF1FF356FD3AC46CAEB0303B3FB34
:10CB0000F8F508FB153309FB05F91FFA8BFB4BEA17
:10CB10000347B94504D93F1905F1FF3362D31D46D8
:10CB200045EA0C4CACFB0223C9EB07079F424FF0D0
:10CB300000054AD346D062462B465DE79440C2F1D9
:10CB4000200921FA09FC914020FA09F9260CBCFBC6
:10CB5000F6F806FB18CCA7B207FB08F349EA01096F
:10CB60004FEA194141EA0C4C634500FA02F509D934
:10CB70001CEB040C08F1FF323BD2634539D9A8F114
:10CB80000208A444C3EB0C0CBCFBF6F306FB13C178
:10CB900007FB03F21FFA89F949EA01418A4207D9E2
:10CBA000091903F1FF3022D28A4220D9023B2144E5
:10CBB000891A43EA084343E73A4605E7334618E74C
:10CBC0000A4666E7B0409042B5D20CF1FF3200232E
:10CBD00012E7334632460FE79A458DD9ACF1020C85
:10CBE00023448AE7B9459AD9023D274498E703468A
:10CBF000DEE79046C6E70238214435E71C481D4968
:10CC0000026800608A4200F01D80002100F004B834
:10CC1000194B5B58435004311848194B42189A423B
:10CC2000FFF4F6AF174A00F003B8002342F8043BC4
:10CC3000154B9A42FFF4F9AFFEF73AFD00F038F8D1
:10CC4000FFF7FEBF114E124830601248016821F014
:10CC500070610160410201600F4C182020600F4993
:10CC60000F4808600F48D0F800D040680047000027
:10CC7000F04F0020EFBEADDEA0360108000000201E
:10CC8000FC00002000010020882100201810024034
:10CC90000900000004000140140C0140000C014098
:10CCA0004434434400F0FF1FFFF7FEBF00000000C4
:10CCB0002DE9804893B0F3F72BFADFF850928E4CB1
:10CCC000D9F8086000232370330740F1E7806368D8
:10CCD0001B7A042B00F2E080DFE803F00303058AEF
:10CCE000B100237AD9E0627A834B002A00F0D48025
:10CCF00000225A7293F82020170700F1CD80D97ACC
:10CD00009A7A01F0070042EA00225A621A7B02F086
:10CD10003F00400140EAD1019962597B890041EA14
:10CD200092119A7B02F0010041EA8021D962D97BFD
:10CD300001F00F00C00140EA52021A631A7C02F0AF
:10CD40007F00000140EA11115963597C490041EA12
:10CD5000D212997C01F0030042EA40229A63DA7C05
:10CD600002F01F00800140EA9101D963197DC900DA
:10CD700041EA5212997D1A645A7D01F0070042EA95
:10CD800000225A64DA7D02F03F00400140EAD101FE
:10CD90009964197E890041EA92115A7E02F00100DD
:10CDA00041EA8021D964997E01F00F00C00140EA78
:10CDB00052021A65DA7E02F07F00000140EA11118A
:10CDC0005965197F490041EAD212597F01F00300E9
:10CDD00042EA40229A659A7F02F01F00800140EAF1
:10CDE0009101D965D97FC90041EA52121A6651E012
:10CDF00094F86420404B002A4ED0002283F864202F
:10CE000093F86620012A47D193F88A20102A84BF1C
:10CE1000102283F88A2094F88A10384A0023D8B266
:10CE2000884202F1020235D212F8010C12F8025CBB
:10CE300040EA0525324840F823500133EFE794F8E3
:10CE4000CC202D4B42B3002283F8CC2093F8CD2088
:10CE5000A82A21D193F8E050F5B9274901EB450301
:10CE600093F8D00093F8D13003EB0020FEF7A6FD35
:10CE70001DA3D3E90023FEF741FF1DA3D3E900233F
:10CE8000FEF75EFCFFF74AF81E4B43F8250001351C
:10CE9000082DE2D1012300E000232370750408D59A
:10CEA00094F8043123B1144B002283F804210123A8
:10CEB000237023783BB1F00505D50F4BD3F808312B
:10CEC0001B681B689847104D23782A6833B90A4BB2
:10CED000D3F80C31D31ADB43DB0F00E00123BBB1E5
:10CEE000F4F77CFB28E000BF9A9999999999194029
:10CEF0000000000000707740000100206801002061
:10CF00008C010020E40100205C210020C8190020D1
:10CF1000D4F810315A1CC4F810212BB9D9F80830B4
:10CF2000190601D5F5F74AFFD4F81031012B03DDBE
:10CF3000A44B0022C3F81021F9F7ACFAB9F80C3071
:10CF400028602BB1D4F81421821A002AC0F2378647
:10CF500018449C4D99F80530C4F81401059305F563
:10CF60009670D4F82031D4F81861984705F596707A
:10CF7000014694F83221F9F701F9934B1B88002BF5
:10CF800000F09880D5F834314FF000081B7805F593
:10CF90009C75049347468C4BB3F800A08B4BBAF5B5
:10CFA0007A7F03D1002243F808202A61884AD05FA3
:10CFB00053F80820024443F80820FFF7D9F82A69FB
:10CFC0000132012A2A6104D1002368602860AB6025
:10CFD0002AE0D5F800C002926146CDF80CC001905D
:10CFE000FFF710F8029A83461046FFF7C1F8014692
:10CFF0005846FFF7C5F9DDF80CC001466046FFF75B
:10D0000003F8019B02461146686018460292FEF73B
:10D01000F9FF01465846FFF7FFF8A968FEF7F4FF4D
:10D02000029AE8602A60A860694A002302F1540B62
:10D03000BAF1010FBB5227F80B30DFF88CA12CD1CD
:10D040002869012807DD0138FFF792F80146E868F2
:10D05000FFF796F900E0002002F066F80346049816
:10D0600058B10193FFF784F8019B01461846FFF77A
:10D070008FFA10B14FF47A731AE0544B4FF47A726E
:10D0800058F803300A2003F5FA7393FBF2F32BF8F8
:10D0900007300F210122F9F7E7FA0237062F08F1CE
:10D0A000040805F114057FF476AFBAF80030013BAF
:10D0B000AAF800300023434D05F5967205F5C071BE
:10D0C000985A595A411A99520233062BF3D1D5F87E
:10D0D000883113F0020300F0F282D5F8903105F5A3
:10D0E000CC70984705F5CC70014695F89E21F9F76C
:10D0F00045F8B5F8A03105F5CC77002B44D00022D7
:10D10000D5F8A40113462F4D37F902C0B5F8A01188
:10D1100005F5D47EB1F5C87F04BF00214EF8031099
:10D120005EF80310274D61444EF8031004330021CC
:10D130000C2BB952815202F10202E4D1B5F8A031B0
:10D14000012B1CD1D5F8A8314FF4C872C83393FB1A
:10D15000F2F30380D5F8AC31C83393FBF2F343808C
:10D16000D5F8B031C83393FBF2F21A4B1B88D21AB0
:10D170008280A6F85410A6F85610FAF799FDB4F874
:10D18000A031013BA4F8A031D9F808305A0740F18A
:10D190008680B4F8B4210B4B322A1DD1D3F8A421D8
:10D1A0001188A3F8B61151889288A3F8B811A3F892
:10D1B000BA21B6F85420A3F8BC21B6F85620A3F83B
:10D1C000BE210BE000010020682100207402002035
:10D1D0002C02002000000020002A3ED00021D4F8BC
:10D1E000A4510A46C14837F901C0B0F8B43100F57E
:10D1F000E07E322B04BF00234EF802305EF80200BE
:10D20000BA4B60444EF80200043200200C2A7852D7
:10D21000685201F10201E5D1B3F8B421012A17D116
:10D2200083F8CD21052283F8CE21B3F8B62183F807
:10D23000CC012A80B3F8B8216A80B3F8BA21AA8059
:10D24000B3F8BC21B3F8BE31A6F85420A6F8563086
:10D25000B4F8B431013BA4F8B43194F8CF21A34B16
:10D26000EAB1D3F8C001D3F8A4113225002290FB13
:10D27000F5F083F8CF210880D3F8C40190FBF5F0D6
:10D280004880D3F8C83193FBF5F5994B1B88ED1A0C
:10D290008D80A6F85420A6F85620FAF709FDD4F898
:10D2A000A431B4F898111A8800268A1AA4F8982193
:10D2B000B4F89A115A88B3468A1AA4F89A219B881E
:10D2C000B4F89C21D31AA4F89C31F9F7E3F8D4F808
:10D2D000D0310546C31A18460493FEF745FFD4F82B
:10D2E000D4110690FEF798FFD4F8D881C4F8D05135
:10D2F00098F80090079035467E4F785FFEF738FF2C
:10D300000799FEF789FF09A98851B9F1000F2BD0C1
:10D310004846FEF72DFF01464FF07E50FFF730F8EC
:10D320000346194607F1B00A4FF07E500193FEF70D
:10D3300069FE56F80A10FEF76FFF07F16C0102460E
:10D34000485F0292FEF714FF019BBC371946FEF7B7
:10D3500063FF029A01461046FEF756FE4AF80600A1
:10D36000FFF720F9785304E007F1BC036C37EA5B60
:10D37000EA52614F0436EB5F0235062D03FB03BB17
:10D38000BAD15B4D642303FB0BFB2B8807F108002C
:10D390005B439BFBF3FBABF1490B09A91FFA8BFB2A
:10D3A000F9F720FBBBF13B0FD8F8046010D9B4F9B2
:10D3B000FC01FEF7DDFED4F8F86101463046FFF7C8
:10D3C000E7F84A4F94F8FE3160B343F008032BE0CE
:10D3D0004FF07E513046FEF717FE01464FF07E506B
:10D3E000FEF7CEFF4FF0000A8146DFF818B1304655
:10D3F0005BF81A10FEF710FF034637F90A00019395
:10D40000FEF7B6FE019B01461846FEF7FDFD4946B4
:10D41000FEF702FF4BF81A000AF1020ABAF1060FF2
:10D42000E3D1C4E723F008033146D4F8F40187F8C8
:10D43000FE3101F077FE0746C4F80002D4F8F0018F
:10D44000D4F8F8A100F10046D4F8F4010146FEF743
:10D45000E3FE514681465046FEF7DEFE0146484651
:10D46000FEF7D2FD01F060FE0146304601F05AFEA3
:10D4700022490646C4F804023846FEF7CDFE01F004
:10D4800085FD1E49A4F808023046FEF7C5FE01F0EE
:10D490007DFDD4F88831A4F80A021B0736D5184858
:10D4A00009A9F9F79FFAD8F808504FF07E5128469D
:10D4B000FEF7AAFD01464FF07E50FEF761FFDFF850
:10D4C00048A081460AF10C0BDAF804102846FEF752
:10D4D000A3FE0021FEF798FD4946FEF79DFE4AF89F
:10D4E000040FDA45F0D106484DE000BF00010020EE
:10D4F000000000202C020020E80200204C3D0F44D8
:10D500000C030020F002002008030020DFF8B09395
:10D5100009A909F10400F9F765FA6868D5F808A0C7
:10D520000146FEF779FE514683465046FEF774FEEB
:10D5300001465846FEF768FDED68824629462846B2
:10D54000FEF76AFE01465046FEF75EFD01F0ECFD77
:10D5500000210546FEF7F4FFA0B9D9F804002946DA
:10D56000FEF70EFF2946C9F80400D9F80800FEF7B7
:10D5700007FF2946C9F80800D9F80C00FEF700FF9C
:10D58000C9F80C00C948F9F7E5FAC949A4F8180226
:10D590000698FEF741FE06F10046054607F10047F2
:10D5A000B4F918020D960C97FEF7E2FDC14900F19F
:10D5B0000040FEF731FE0E90B4F9E801FEF7D8FD09
:10D5C0000F90B4F9EA01FEF7D3FD1090B4F9EC0125
:10D5D000FEF7CEFD0CA911900FA8F9F703FA98F801
:10D5E0000130B54E012B18D1B44B1B785F070ED418
:10D5F000D6F81C32402093FBF0F0181AFEF7B8FD65
:10D600001199FEF701FDFEF7CDFFC6F81C02D4F814
:10D610001C32402093FBF0F001E0A94B1888FEF784
:10D62000A7FD01461198FEF7EDFCD4F824121190E5
:10D630002846FEF7E9FC01462846FEF7A1FED4F88D
:10D640002062054631461198FEF7DCFC014628466B
:10D65000FEF7E2FD01463046FEF7D6FC0646C4F86A
:10D6600020020F98D4F8287201F090FCD4F83452BC
:10D670002978FCF701F93844C4F828021098D4F846
:10D680002C7201F083FC2978FCF7F6F83844C4F8D2
:10D690002C023046D4F8307201F078FC6978FCF73F
:10D6A000EBF8884B049D1A6838442A441A60D4F871
:10D6B0003832C4F830020133C4F8383205E0A5F836
:10D6C0009831A5F89A31A5F89C31B4F82C21059E23
:10D6D000A4F83C22B4F82E21012E774BA4F83E2268
:10D6E0000ED1B3F94212B3F9302102EB410203210A
:10D6F00092FBF1F292B2A3F84022A3F8422203E097
:10D70000B3F83021A3F84022F8F7C4FE6E4B6A4DFF
:10D710001860D4F84832C4F84802C31AA4F8443256
:10D72000F4F756FCD4F84C3213F4801300F08D80DB
:10D73000B5F85032180600F1ED80604B1B785907A0
:10D7400070D595F852225E4B12B195F853223AB13A
:10D750000022C4F8542201221A74002284F85322B1
:10D760001B7CD4F81851032B95F80080524E05F11C
:10D77000040784F8523206D1384606F516714C2259
:10D7800001F096F944E0012B07D106F516703946F1
:10D790004C2201F08DF9002302E0022B02D101237B
:10D7A00086F8A432012384F8A53284F8A632002337
:10D7B000C4F8A832C4F8AC32444A94F8A432C4F88D
:10D7C000B07213441B7C424A1D4484F8B532C4F83D
:10D7D0005422287984F8B482FEF7CAFC3D49FEF74A
:10D7E000CFFDC4F8B802A87BFEF7C2FC3A49FEF7A9
:10D7F000C7FDC4F8BC02287EFEF7BAFC3749FEF725
:10D800000BFDC4F8C002FEF7F3FE00232876AB73CD
:10D81000B4F8503243F08003A4F85032012384F866
:10D82000C43277E00026D5F854023146FEF788FE70
:10D83000074600286ED1FAF73BFA214B0122C5F8C2
:10D84000546285F852721A7464E0B5F8509219F077
:10D85000800F54D095F85222194F511E012941D8FA
:10D860001D49D5F8BC02FEF7D7FCFEF7C1FED5F87E
:10D87000B06295F8B5821A49B04488F80A00D5F824
:10D88000C002FEF7C9FCFEF7B3FE88F8140030783A
:10D89000FEF76EFC0146FEF7B7FBFEF7A9FEB37A72
:10D8A000B0703373337DB37522E000BF04000020F5
:10D8B000BD37863535FA8E3C000100206C210020F2
:10D8C00000000020642100205C210020F8050108F0
:10D8D0000000A0410000204100007A445555553F0A
:10D8E0009A99993F032A03D185F85232012301E026
:10D8F0003B7C013329F080093B74A4F85092A24B81
:10D900001B785A0706D494F8C4321BB19F4B0122EE
:10D9100083F85322D4F818819C4D98F86471002F35
:10D920004FD0B5F850329B074BD0D5F8F001D5F861
:10D93000F4B10146FEF770FC594682465846FEF7A0
:10D940006BFC01465046FEF75FFBD5F8F861824656
:10D9500031463046FEF760FC01465046FEF754FB68
:10D96000B5F8CC9201F0E0FB01463046FEF708FD29
:10D9700087490646FEF7F8FDF8B9304601F082FB0C
:10D98000D5F8D012FEF748FC01F000FBB0F5617F3E
:10D99000A8BF4FF46170FEF7EBFB7E49FEF7F0FC89
:10D9A00001F032FB05463846FEF7E2FB2946FEF75A
:10D9B00033FC01F0EBFA80B200E000204844A4F808
:10D9C000CC02D4F88831714D9F0640F18380B5F8C0
:10D9D000503203F03003002B7CD095F8FE31DE0787
:10D9E00078D5B5F91802FEF7C3FB6B49FEF714FCB6
:10D9F000064601F009FB8146304601F091FAD5F860
:10DA0000D432074693F803A0B5F9DE02634EBAF1AB
:10DA1000000F31D0B5F8DA32CAF100051FFA83FBE6
:10DA20001BB2C01AFCF7B0F8A84203DB5045A8BFF0
:10DA3000504600E02846B4F8D8328344B4F9DC02FA
:10DA40009AB21BB21FFA8BFBC01AA4F8DAB2029288
:10DA5000FCF79AF8A842029A03DB5045B4BF05468A
:10DA600055461544ADB2A4F8D8520FFA8BF0FEF724
:10DA70007FFB824628B204E0FEF77AFB8246B5F9C6
:10DA8000DC02FEF775FB394605465046FEF7C4FB3F
:10DA9000494683462846FEF7BFFB01465846FEF737
:10DAA000B1FA3F49FEF76CFCFEF77CFD4946308039
:10DAB0005046FEF7B1FB394681462846FEF7ACFBDF
:10DAC00001464846FEF7A0FA3549FEF759FCFEF735
:10DAD00069FD7080334B344D1E6808F1040008F175
:10DAE0005403D4F8E012B5F8F620B047F7F758FE23
:10DAF000D4F8E432002B60D0244B93F8E832013B99
:10DB0000142B55D8DFE803F00B5454275754541FF7
:10DB100054545454542F5454545454272F00D4F86C
:10DB2000EC325B782BB1214B00205989FCF79DF832
:10DB300043E0154B1B7803F0040303F0FF00002BB8
:10DB4000F1D10146F2E7194D0020E988FCF78DF884
:10DB500001202989EAE7154D00202989FCF785F87D
:10DB600001206989E2E7114D0020E988FCF77DF882
:10DB700001202989FCF779F802206989FCF775F8FA
:10DB80000320A989D2E700BF6C21002000010020FA
:10DB90008FC2753CEFB6B04435FA8E3C6021002050
:10DBA000000020417C000020C81900206C000020EB
:10DBB000AB68980601D5F8F707FFF8F7C0FEC64B2B
:10DBC0001B78002B40F0F484C44FBB68590540F12A
:10DBD000EF8494F8F032C24D002B00F0E984FBF79B
:10DBE00063FE002800F0E48495F8F132002B00F089
:10DBF000DF84D5F8F4321B78002B40F03282D5F860
:10DC0000F802F8F787FD002840F02B82DFF8F08259
:10DC1000D5F8FC22D8F800309A1A7C2A40F22182EA
:10DC2000C5F8FC3295F80033013385F8003305461A
:10DC300005F12400AA4EC0B2F8F74AFE06F5F473C7
:10DC400033F91500FEF794FAA64B81461888FEF7C3
:10DC50008FFA01464846FEF793FBA349FEF7DCFA2C
:10DC6000FEF7A0FC013500B2F8F75EFE032DDFD110
:10DC70003020F8F72DFE0020F8F756FEF8F736FEB4
:10DC800096F8005315F0030520D1D6F8FC2241F296
:10DC900088339A420BD91020F8F71AFE2846F8F775
:10DCA00043FE2120F8F714FE2846F8F73DFE142025
:10DCB000F8F70EFEB4F91802F8F736FE1C20F8F754
:10DCC00007FE0020F8F730FEF8F710FE94F8003356
:10DCD000834D5A0740F09F810220F8F7F9FDB5F90E
:10DCE00002030A2390FBF3F0F8F71EFE0320F8F777
:10DCF000EFFD7E4B1B7813F0040F4FF0050304D0AB
:10DD0000B5F9CC0290FBF3F005E0D5F80423528975
:10DD1000B2FBF3F000B2F8F707FEBB689B077FD5B4
:10DD2000734D94F808232B7840F63401B2FBF3F2DC
:10DD30004A432A21B2FBF1F2B4F80A13062091FB00
:10DD4000F3F703FB17173F01BFB247EA0227BFB241
:10DD5000C2F303221743F8F7BBFD38B2F8F7E4FD2E
:10DD6000B4F80A232B78013292B292FBF3F103FB51
:10DD70001123A4F80A3394F808336E255D43152364
:10DD800095FBF3F53A204FF06409F8F7A1FDB5FBD8
:10DD9000F9F73846F8F7C8FD3B20F8F799FD09FB7D
:10DDA000175080B20A27053090FBF7F000B2F8F761
:10DDB000BBFD2820F8F78CFDD4F80C03484E90FBEF
:10DDC000F7F000B2F8F7B0FD0420F8F781FDD4F8C1
:10DDD0000433D6F810035D894FF6FF739842A8BF4D
:10DDE000184620EAE070C5B1281AFDF7F7FD0022B9
:10DDF000404BFDF759FE064628460F46FDF7EEFD5F
:10DE000002460B4630463946FDF778FFFEF75EF8CE
:10DE10004845A8BF484620EAE07000B2F8F784FD04
:10DE2000D4F888312E4D9F0640F1898095F8FE3157
:10DE30009E071AD51120F8F74BFDB5F81403FDF72E
:10DE4000CDFD23A3D3E90023FDF72EFE00222A4BAC
:10DE5000FDF778FCFEF73AF800B2F8F765FD1920F7
:10DE6000F8F736FD0020F8F75FFD94F8FE31B4F8BE
:10DE7000165313F0020F08BF00250120F8F728FD04
:10DE800028B2F8F751FD0920F8F722FD0020F8F735
:10DE90004BFD1A4B94F818531B88B3F5967F0BD99A
:10DEA0000F4A92F8002302F00F02072A04D842F228
:10DEB0000F75AB42B8BF1D460520F8F709FDD4F831
:10DEC0001C335B7BF3B928B237E000BFAFF30080AF
:10DED0007B14AE47E17A843F6B210020C8190020F3
:10DEE000000100200000002000007A446C21002086
:10DEF00080000020000059400000E03F8200002028
:10DF0000C4190020A5F12000FDF768FDD0A3D3E9D6
:10DF10000023FDF7F3FEFEF721F800210546FEF78A
:10DF200019FB10B14FF03F4101E04FF07C51284602
:10DF3000FEF76AF8FEF736FB00B2F8F7F5FCD4F806
:10DF4000883198060ED4C44B0021D3F81C5368685E
:10DF5000FEF7F6FA00285CD1A8680021FEF7F0FA77
:10DF6000002856D194F8FE21BB4B910703D493F8B7
:10DF70002023012A07D10123D4F82463D4F828539D
:10DF800084F820330FE0D3F81C53B4496868FEF7D7
:10DF900043F9FEF707FBB1490646A868FEF73CF9CE
:10DFA000FEF700FB05460FA93046FBF7A5FC132042
:10DFB000F8F78EFCBDF93C00F8F7B6FC1B20F8F72B
:10DFC00087FCBDF93E00F8F7AFFC2320F8F780FC92
:10DFD000002EACBF4E205320F8F7A6FC0FA9284610
:10DFE000FBF78AFC1220F8F773FCBDF93C00F8F748
:10DFF0009BFC1A20F8F76CFCBDF93E00F8F794FC86
:10E000002220F8F765FC002DACBF45205720F8F71B
:10E010008BFCF8F76BFC94F80033282B21D18E4B46
:10E020000022D8F8007083F800234FF47A73B7FB0E
:10E03000F3F73C251720F8F74BFCB7FBF5F6B6FBDA
:10E04000F5F005FB1060000200B2F8F76DFC182037
:10E05000F8F73EFC05FB167000B2F8F765FCF8F720
:10E0600045FCD4F8F4327C4D1B78012B40F0248120
:10E07000F8F710FAD5F82C33794AC31A93420646BA
:10E0800040F2A98095F80823002385F84E2385F8EF
:10E090004423D5F80C2385F8323385F8343385F8DA
:10E0A0004F3385F845330A2392FBF3F285F84C236E
:10E0B000121285F84D23D5F8102392FBF3F385F85F
:10E0C000503395F8FE211B1285F8513395F818331B
:10E0D000920785F8763303D42D2385F8773378E0DB
:10E0E000042B8CBF3323322385F877335D48D4F873
:10E0F0002453DFF878C195FBF0F70CFB07584FF07D
:10E10000060E0EFB08F8584B07EB870798FBF3F950
:10E1100003FB198807EB87074FFA89F9D4F828130E
:10E1200009EB8707BFB291FBF0F084F866733F0AF2
:10E1300084F867730CFB00170EFB07F7ED0F84F8EC
:10E14000655397FBF3F503FB1573642293FBF2F31E
:10E1500084F86D331B12C90F84F86E33B4F814338E
:10E1600084F86A1324214B4398FBF2F893FBF2F2F4
:10E17000B4F8883384F86323C2F3072284F8642355
:10E1800084F86F33B4F816231B0A84F870330A231B
:10E19000B2FBF3F300EB800003F5FA739BB26DB2B0
:10E1A00000EB800005EB800084F871331B0A80B21D
:10E1B00084F87233B4F88A3384F8688384F86B0384
:10E1C0004FEA2828000A84F8698384F86C0384F8ED
:10E1D0007833C4F82C6394F88C331F4D5BB9D5F8B1
:10E1E0009003F8F797FA95F89D34002B40F02B84B4
:10E1F000012800F23084D4F89823174D002A5BD010
:10E2000095F88C733FB1D5F89C3340F6B731F31ACB
:10E210008B420BD850E00123D5F89003022185F8FA
:10E220008C33F8F763FA85F8A07343E095F8A133CF
:10E23000F3B9D5F890030121C5F8983385F88C33EC
:10E24000F8F754FAF8F76BFA34E000BFAFF3008048
:10E25000CDCCCCCCCCCCFC3F000100208096184B20
:10E260003F0D03008096980040420F00806967FFD1
:10E27000013BDBB285F8A13395F8A01395F8A20312
:10E2800043B901304B1C85F8A20385F8A033D5F8BB
:10E2900090030DE0134613F8012B0130114485F86B
:10E2A000A203D5F8900385F8A013C5F8983311465A
:10E2B000F8F742FAC4F89C63D4F8F432AE4D1B78F8
:10E2C000022B1BD1D5F8A433C3B1C5F8A8331B6802
:10E2D000AA4AC5F8AC33D5F8B0331344987CF9F7A3
:10E2E000F3FCD5F8A8339879F8F72BFAD5F8B033C2
:10E2F0000133092B88BF0023C5F8B033FBF726FB99
:10E30000002800F0558194F8B433013B012B00F252
:10E310004F81994D9A4ED5F8B803F8F7FBF9E8B15B
:10E32000D5F8B803F8F7F1F995F8BC2333687E2ADD
:10E3300010D102221B2885F8B423C5F8C03305D0BC
:10E340000D2803D0342801D0672803D18A4901233E
:10E3500081F8C433884A82F8BC03DAE73368D5F819
:10E36000C02341F658319A1A8A4203D9032385F80B
:10E37000B4331DE1D5F8C8239B1A042B40F2188151
:10E3800095F8C433002B00F0138195F8CC237D4B16
:10E3900033F8120018B985F8CC034FF4036094F8F1
:10E3A000CC33B0F5C06F03F10103DBB2724D84F8DA
:10E3B000CC334AD019D8B0F5007F43D006D8B0F599
:10E3C000807F6AD0B0F5887F67D0F1E0B0F5806FCC
:10E3D00072D0B0F5826F00F0B180B0F5047F40F0EC
:10E3E000E78095F808335321DCE0B0F5006F2FD0BB
:10E3F0000CD8B0F5E26F56D0B0F5E46F59D0B0F557
:10E40000E06F40F0D580B5F9E8114EE0B0F5036F4C
:10E4100007D0B0F5046F42D0B0F5026F40F0C8806D
:10E42000B4E0D5F888319F0640F1C28095F8FE31FE
:10E430009E0740F1BD80B5F814332421594364236D
:10E44000123133E0D5F80C13ADE0D5F81013AAE083
:10E45000D5F88821910640F1AB8095F8FE2192070E
:10E4600040F1A680DB0709D5D5F828130029BCBFE9
:10E47000494241F0804141F0004106E0D5F82413C3
:10E480000029BCBF494241F080414FF40060FCF7D5
:10E490004BFC002384F8C4338AE0002183E0B5F903
:10E4A000183264217EE0B5F9EA112C2391FBF3F1D7
:10E4B00079E0B5F9EC11F8E795F8CD3342F2107137
:10E4C0000133DBB2032B85F8CD3384BF012385F8FC
:10E4D000CD3394F8CD3359432B4B1B78DF0748BF1E
:10E4E00001319E0748BF02315807B5F8503248BF86
:10E4F0000431DA0748BF0A319F0748BF14311E06AE
:10E5000048BF2831D80548BF28315A0748BF643171
:10E510001F0748BFC8319E0548BF01F5C87198065E
:10E5200048BF01F57A71DA0648BF01F5FA615B066A
:10E5300048BF01F57A614FF4806034E0D5F8881166
:10E5400011F0200612D095F8FE3113F0020F0CBF27
:10E5500000214FF47A7113F0010F0CBF00234FF428
:10E56000FA63194495F8183319441CE03146FCF756
:10E57000DBFB85F8C4631BE000010020F8050108FF
:10E58000C41900202C1D01086C210020D5F8883109
:10E590009F060DD595F8FE319E0709D5B5F81633BF
:10E5A0004FF47A715943FCF7BFFB002385F8C4335D
:10E5B000DFF8E8B2DBF80830DD037EF57EAB94F8D7
:10E5C000CE33A84E002B3EF478ABA74B1B78002B24
:10E5D0007EF473ABF7F75EFFD6F8D033D6F8D87376
:10E5E000C31A6FEA0309D6F8D433C71BC31AFF4313
:10E5F0006FEA030AFF0F05464FEAD9794FEADA7A44
:10E6000037B9BAF1000F03D1B9F1000F3EF455ABA1
:10E610004FF00008DFF84CC25FFA88F6604690F8C9
:10E6200060349E423BD29149DCF8DC33B200096889
:10E6300013446244C2F8E0135988C8050BD48B0513
:10E640002AD58B4B1B785E0754BF8A4B8A4B1B68BD
:10E65000C2F8E03320E01946884A30460193CDF8ED
:10E660000CC0F6F7BDFADDF80CC0019BBCF85022D7
:10E6700012F0400F03D030461946814A0AE0900755
:10E6800003D5304619467F4A04E0D10704D57E4AB7
:10E6900030461946F6F7A4FA08F10108BAE79E00D9
:10E6A0000023B3421FD06F49D1F8DC231A445288AB
:10E6B000520516D501F57872D0580890B1F9680462
:10E6C0007821A0F57A7048434FF47A7190FBF1F00D
:10E6D00000F22B1040F2671190FBF1FE01FB1E01CE
:10E6E00099520433DDE767B305F5C333A033C4F8AB
:10E6F000D83394F886345B4E1BBB86F88734DBF83E
:10E7000008309B0705D5F7F7F1FD10B1012386F816
:10E710008734D4F88834534E1B689B68984728B1D7
:10E7200096F8873443F0020386F88734504B1B7801
:10E7300013F0050F05D194F8873443F0040384F8EF
:10E74000873494F8872422B9464B93F88634002BFB
:10E750004DD094F8861411F0010FA1F10C001AD1DC
:10E76000032906D8414B434E12F0040F18BF33461D
:10E7700000E03E4B0439072904D8444912F0010F48
:10E7800018BF0B46C0B2032810D8414912F0020F3F
:10E7900018BF0B460AE0C0B2032806D8334B3649EF
:10E7A00012F0020F18BF0B4600E0304B0021DFF8DB
:10E7B000B4E0764696F86004CEB2B0420CD9DEF8EA
:10E7C000DC03B60030444088000603D51868764460
:10E7D000C6F8E0030131EAE78FB14AB194F8862424
:10E7E000204B0132D2B2142A07D1002205E037B102
:10E7F00094F88634002BF1D101E083F88624BAF135
:10E80000000F23D0B4F9C832B4F9C6223221002A4D
:10E81000B8BF5242002BB8BF5B4293FBF1F392FBAF
:10E82000F1F1DBB2C9B28B4238BF0B46194A0BB1CA
:10E8300092FBF3F22A44C4F8D42394F88C24094BB5
:10E840000AB9012200E0002283F88C2494F88C2479
:10E85000044B22B9104AC3F89024002028E0034A50
:10E86000F9E700BF000100206A210020281D0108EF
:10E870006C210020F80501080406010814060108AF
:10E880001A0601082006010826060108FC050108F1
:10E8900000060108400D03002C060108C8190020DD
:10E8A000D3F8DC1394000E197688760607D401306D
:10E8B0007C4BC2B293F860149142F1D89FE0B3F957
:10E8C000C662192E21DD11F8227093F894E407F046
:10E8D0000F0CF445D3F8906408DC93F895E4BEEB94
:10E8E000171F03DC23443468C3F8E0436D4B11F871
:10E8F000224093F896C404F00F0EE6452DDB93F802
:10E900009574B7EB141F28DC22E0193625DA11F8CC
:10E91000227093F894E407F00F0CF445D3F8906458
:10E9200008DC93F897E4BEEB171F03DB234434683D
:10E93000C3F8E0435B4B11F8224093F896C404F00F
:10E940000F0EE64509DB93F89774B7EB141F04DB51
:10E95000346803EB8203C3F8E043524BB3F9C84277
:10E96000192C21DD11F8227093F8946407F00F0E32
:10E97000B645D3F8904409DC93F895E4BEEB171F35
:10E9800004DC276803EB8203C3F8E07311F822303C
:10E9900003F00F01B1428ADC424F97F89714B1EBB4
:10E9A000131F84DB3B4624E0193480DA11F822700F
:10E9B00093F8966407F00F0EB645D3F8904409DB40
:10E9C00093F895E4BEEB171F04DC276803EB820382
:10E9D000C3F8E07311F8223003F00F01B142FFF6E3
:10E9E00066AF304E96F89714B1EB131FFFF65FAF8A
:10E9F000334603EB82022368C2F8E03357E7B9F1EC
:10EA0000000F1CD093F8992493F8981405F543450A
:10EA10008818013890FBF2F402FB140083F89B1471
:10EA2000013183F89A0491FBF2F002FB1012503589
:10EA3000D2B2C3F8D05383F89C2483F89824F6F715
:10EA400070FAFEF73AB900283FF4D5ABD5F8900339
:10EA5000F7F75BFE22E00228134F03D0F7F75FFEC3
:10EA6000012303E07A7C22B1C5F894637B74FFF73D
:10EA7000C2BBD5F89433F31AB3F57A6FFFF4BBAB8E
:10EA80000123D5F890037B74F7F73FFE0746D5F8CE
:10EA90009003F7F73AFE802F7FF4ADABFBF75CFDF8
:10EAA000FFF7A9BB0001002000000020AFF30080A9
:10EAB00010B50023934203D0CC5CC4540133F9E772
:10EAC00010BD02440346934202D003F8011BFAE74B
:10EAD000704700000D4B70B51D680022845C2B1937
:10EAE0005B7803F00303012B8B5C08BF2034EE1826
:10EAF000767806F00306012E08BF2033E41A02D10F
:10EB00000132002BEAD1204670BD00BF90000020EA
:10EB100010B50446224613780134002BFAD1CC5CA0
:10EB2000D4540133002CFAD110BDC9B2024610F8FA
:10EB3000013B1BB18B42F9D1104670470029FBD035
:10EB400018467047034613F8012B002AFBD1181A08
:10EB5000013870470F4BF0B51E680023934215D063
:10EB6000C55C7419647804F00304012CCC5C08BF04
:10EB7000203537197F7807F00307012F08BF2034AD
:10EB80002D1B04D10133002CE8D100E000252846DC
:10EB9000F0BD00BF9000002010B5034632B111F85F
:10EBA000014B013A03F8014B002CF7D11A44934270
:10EBB00003D0002103F8011BF9E710BD30B503783D
:10EBC0000BB1044604E00B78002B18BF002030BDC9
:10EBD00022461078013438B10023C85C28B1D55CD6
:10EBE0008542F5D10133F8E730BD104630BD002134
:10EBF0000A2200F001B92DE9F04E82468B461F46ED
:10EC0000144612B90020BDE8F08E002BFAD0002681
:10EC1000A642F7D2A5196D0807FB05B9504649462B
:10EC2000089B9847002802DB03D06E1C25462C4623
:10EC3000EEE74846BDE8F08E174B2DE9F0411D6820
:10EC40000646AC6D0F46FCB9502000F0E3F8A8650D
:10EC50008460AB6D046044601C61DC60AB6D9C61E2
:10EC60005C61AB6DDC629C62AB6D5C631C63AB6D25
:10EC7000DC639C63AB6D5C641C64AB6DDC649C64A6
:10EC8000AB6D1C77AB6D5C6230463946AA6D0123D3
:10EC9000BDE8F04100F002B8F4000020F0B508B97A
:10ECA000106828B3044614F8015B0F4617F8016B8F
:10ECB0003EB1B542FAD10BB12046F3E714600370C0
:10ECC000F0BD4DB915602846F0BD17F8016BAE4296
:10ECD00007D0002EF9D11C46234613F8015B0F46DE
:10ECE000F3E715B10021217000E02B461360F0BD61
:10ECF000F0BD000084463F482DE9F04FD0F8008079
:10ED00000E46344614F8015B08EB0500407800F02D
:10ED1000080000F0FF0708B12646F2E72D2D03D1C9
:10ED2000B41C7578012703E02B2D04BF7578B41C43
:10ED300033F010000DD1302D08D1207800F0DF0025
:10ED4000582851D165781023023402E0002B08BF07
:10ED50000A23002F0CBF6FF0004A4FF0004ABAFBA5
:10ED6000F3F903FB19AA0026304608EB050B9BF8C4
:10ED700001B01BF0040F01D0303D0BE01BF0030B82
:10ED80001BD0BBF1010F14BF4FF0570B4FF0370BE7
:10ED9000CBEB05059D4210DAB6F1FF3F0AD048459E
:10EDA00006D801D1554503DC03FB0050012601E0E4
:10EDB0004FF0FF3614F8015BD7E7731C0CD1002F1E
:10EDC0004FF022030CBF6FF000404FF00040CCF832
:10EDD00000302AB9BDE8F08F07B1404242B106B118
:10EDE000611E1160BDE8F08F002B08BF0823B0E75B
:10EDF000BDE8F08F9000002030B51346044A054668
:10EE00000C46106829462246BDE83040FFF772BF25
:10EE1000F4000020024B0146186800F003B800BF60
:10EE2000F400002070B5CD1C25F0030508350C2D2D
:10EE300038BF0C25002D06463FDB8D423DD3214BCC
:10EE40001C6818462146A1B10B685B1B0ED40B2B26
:10EE500003D90B60CC18CD501FE08C4202D1626800
:10EE600002601AE04B6863600C4616E00C46496885
:10EE7000E9E7154C23681BB9304600F027F82060FD
:10EE80002946304600F022F8431C014615D0C41C28
:10EE900024F0030484420AD1256004F10B00231DF1
:10EEA00020F00700C31A0BD05A42E25070BD304622
:10EEB000611A00F00BF80130EED10C233360002012
:10EEC00070BD00BF7C2100207821002038B5064CA1
:10EED000002305460846236000F008F8431C02D1D1
:10EEE000236803B12B6038BD84210020094A1368D0
:10EEF00063B118446946884202D8106018467047CA
:10EF0000054B0C221A604FF0FF307047034B136023
:10EF1000EFE700BF8021002084210020882100200D
:10EF200000B5194A20F00043934283B0014617DD33
:10EF3000B3F1FF4F04DBFDF765F803B05DF804FBA8
:10EF4000694600F037FB00F00302012A009801999E
:10EF500011D0022A0AD09AB1012201F0EFF8ECE7B1
:10EF6000002100F0EFFC03B05DF804FB00F0EAFCC8
:10EF700000F10040E1E701F0E1F800F10040DCE7DA
:10EF800000F0E0FCD9E700BFD80F493F30B5C0F32F
:10EF9000C754A4F17F031E2B83B0014620DC581C0C
:10EFA0001BDB162B4FEAD17509DDC1F3160040F4C7
:10EFB0000000963CA04005B1404203B030BD114B6B
:10EFC00053F825402046FDF71FF80190019821468F
:10EFD000FDF718F820F0004333B9002003B030BD2E
:10EFE000FDF7E0FA03B030BDC0F31604C0F3C7501C
:10EFF00044F40004C0F1960024FA00F0002DDCD0A7
:10F00000DAE700BF8C32010800B51D4A20F000434A
:10F01000934283B0014618DDB3F1FF4F04DBFCF7E8
:10F02000F1FF03B05DF804FB694600F0C3FA00F09D
:10F030000300012818D002280ED0D0B10098019901
:10F0400000F080FC00F10040EBE70021002201F01D
:10F0500075F803B05DF804FB00980199012201F0F6
:10F060006DF800F10040DCE70098019900F06AFCBF
:10F07000D7E700980199012201F060F8D1E700BFBD
:10F08000D80F493F70B58AB0054600F09BF8224C76
:10F09000064694F90030013303D0284601F02CFADB
:10F0A00010B930460AB070BD284601F0DBF94FF0C8
:10F0B0007E51FDF76DFA0028F3D018490122002394
:10F0C0002846009208930191FCF79AFC02460B46F1
:10F0D0001348CDE90423CDE9022301F0A7F894F900
:10F0E0000030CDE90601022B0BD0684601F09CF8F8
:10F0F00038B1089B53B9DDE90601FCF72FFF0AB0D0
:10F1000070BD01F073FA21230360F2E701F06EFA9B
:10F11000089B0360EFE700BFF8000020943201086D
:10F120009C32010800F0B6B970B58AB0054600F00F
:10F13000B5FB224C064694F90030013308D028462E
:10F1400001F0DAF920B128460021FDF703FA10B9E1
:10F1500030460AB070BD1A490122002328460191A9
:10F1600000920893FCF74CFC2478CDE90401CDE92A
:10F1700002017CB900220023CDE90623684601F094
:10F1800053F888B1089BA3B9DDE90601FCF7E6FE58
:10F190000AB070BD0020002102460B46FCF7AEFD10
:10F1A000022CCDE90601E9D101F020FA2123036008
:10F1B000E8E701F01BFA089B0360E5E7F800002090
:10F1C000A0320108F8B520F00043B3F17E5F044699
:10F1D00010D008DCB3F17C5F11DAB3F10C5F00F3FF
:10F1E00084809D48F8BD0146FCF70CFF0146FDF701
:10F1F000C7F8F8BD002840F3CD800020F8BD0028F6
:10F20000C0F2CA8001464FF07E50FCF7FBFE4FF083
:10F210007C51FDF701F8044600F040FB8F4906469B
:10F220002046FCF7F9FF8E49FCF7EEFE2146FCF77D
:10F23000F3FF8C49FCF7E6FE2146FCF7EDFF8A4917
:10F24000FCF7E2FE2146FCF7E7FF8849FCF7DAFE0F
:10F250002146FCF7E1FF8649FCF7D6FE2146FCF784
:10F26000DBFF844905462046FCF7D6FF8249FCF7C0
:10F27000C9FE2146FCF7D0FF8049FCF7C5FE2146B8
:10F28000FCF7CAFF7E49FCF7BDFE2146FCF7C4FF30
:10F290004FF07E51FCF7B8FE01462846FDF770F8A6
:10F2A0003146FCF7B9FF26F47F6525F00F050746C8
:10F2B00029462846FCF7B0FF01462046FCF7A2FE8F
:10F2C000294604463046FCF79FFE01462046FDF7DE
:10F2D00057F801463846FCF797FE01462846FCF7EA
:10F2E00093FE0146FCF790FEF8BD0146FCF794FF43
:10F2F0005A490546FCF790FF5949FCF785FE294617
:10F30000FCF78AFF5749FCF77DFE2946FCF784FF8E
:10F310005549FCF779FE2946FCF77EFF5349FCF777
:10F3200071FE2946FCF778FF5149FCF76DFE29462E
:10F33000FCF772FF4F4906462846FCF76DFF4E4921
:10F34000FCF760FE2946FCF767FF4C49FCF75CFEC2
:10F350002946FCF761FF4A49FCF754FE2946FCF7B1
:10F360005BFF4FF07E51FCF74FFE01463046FDF744
:10F3700007F801462046FCF74FFF01464148FCF7DD
:10F3800041FE01462046FCF73DFE01463E48FCF7A3
:10F3900039FEF8BD3D48F8BD4FF07E51FCF734FE14
:10F3A0004FF07C51FCF738FF2C490446FCF734FF42
:10F3B0002B49FCF729FE2146FCF72EFF2949FCF7D3
:10F3C00021FE2146FCF728FF2749FCF71DFE2146B8
:10F3D000FCF722FF2549FCF715FE2146FCF71CFF30
:10F3E0002349FCF711FE2146FCF716FF064620468E
:10F3F00000F054FA1F4905462046FCF70DFF1E4950
:10F40000FCF700FE2146FCF707FF1C49FCF7FCFD5A
:10F410002146FCF701FF1A49FCF7F4FD2146FCF7F1
:10F42000FBFE4FF07E51FCF7EFFD01463046FCF746
:10F43000A7FF2946FCF7F0FE1249FCF7E3FD014661
:10F440002846FCF7E1FD0146FCF7DEFD01461048C9
:10F45000FCF7D8FDF8BD00BFDB0FC93F08EF11383E
:10F46000047F4F3A4611243DA80A4E3E90B0A63E76
:10F47000ABAA2A3E2EC69D3D6133303F2D57014039
:10F4800039D119406821A233DA0FC93FDB0F494057
:10F49000DA0F494021F00042B2F1FF4FF8B50446BF
:10F4A00014DC20F00045B5F1FF4F06460EDCB1F14B
:10F4B0007E5F3AD08F1707F0020747EAD07755B939
:10F4C000022F2FD0032F2FD13148F8BD08462146F7
:10F4D000FCF79AFDF8BDFAB1B2F1FF4F29D0B5F1B2
:10F4E000FF4F19D0AA1AD2153C2A19DC002938DBA3
:10F4F0002046FCF745FF00F0B5FF00F09DFE012F10
:10F500002CD0022F22D0002F2FD02249FCF77CFDD7
:10F510002149FCF777FDF8BD002E15DB1F48F8BD2B
:10F520001E48ECE71C48F8BDF8BDBDE8F84000F007
:10F5300083BEB5F1FF4F19D0022FF3D0032FC3D0F4
:10F54000012F1BD00020F8BD1548F8BD1149FCF76C
:10F550005BFD01461048FCF755FDF8BD00F1004089
:10F56000F8BD3C32C4DA0020C9E7F8BD022F0CD048
:10F57000032F08D0012F04D00A48F8BD4FF00040F7
:10F58000F8BD0948F8BD0948F8BD0948F8BD00BFF5
:10F59000DB0F49C02EBDBB33DB0F4940DB0FC93F3A
:10F5A000DB0FC9BFDB0F493FDB0F49BFE4CB16C000
:10F5B000E4CB16402DE9F04FAB4A20F000449442D2
:10F5C00089B006460D4664DDA84A94421CDC00283A
:10F5D000A74940F3EC80FCF715FDA64B24F00F047F
:10F5E0009C42064664D0A449FCF70CFD0146286005
:10F5F0003046FCF707FDA049FCF704FD01236860D5
:10F60000184609B0BDE8F08F9C4A944262DDB4F11F
:10F61000FF4F46DAE715863FA4EBC7542046FCF7B8
:10F62000C1FFFCF7A5FD0346014620460593FCF704
:10F63000E9FC4FF08741FCF7EFFD8046FCF7B2FF95
:10F64000FCF796FD0146044640460694FCF7DAFCBA
:10F650004FF08741FCF7E0FD00210790FCF770FFB9
:10F66000002800F0C58020460021FCF769FF002833
:10F6700014BF0123022382480221019000913A46DF
:10F6800005A8294600F022FA002EC0F2A780034602
:10F6900003E00022286000234A60184609B0BDE854
:10F6A000F08F0146FCF7AEFC002368602860F4E7A9
:10F6B0007449FCF7A7FC74490446FCF7A3FC014617
:10F6C00028602046FCF79EFC6F49FCF79BFC012359
:10F6D0006860E2E700F0C6FE6C490746FCF79CFD57
:10F6E0004FF07C51FCF790FCFCF75CFF8246FCF786
:10F6F0003FFD5F498346FCF78FFD01463846FCF726
:10F7000081FC5D4980465846FCF786FDBAF11F0F23
:10F7100081464946404618DC5D4B0AF1FF3253F8FA
:10F72000223024F0FF029A420FD0FCF76BFC074610
:10F730002F6039464046FCF765FC4946FCF762FC01
:10F74000002E686056DB5346A7E7FCF75BFCE31529
:10F75000C0F3C7529A1A082A0746E9DD49495846B4
:10F760000393FCF759FD074639464046FCF74AFC2F
:10F77000044621464046FCF745FC3946FCF742FC6E
:10F78000414907465846FCF747FD3946FCF73AFC25
:10F79000814649462046FCF735FC039BC0F3C7521F
:10F7A0009B1A192B074641DC2860A046C1E7FCF7ED
:10F7B0002BFC304B24F00F049C42064623D02E49EC
:10F7C000FCF722FC014628603046FCF71BFC2A4966
:10F7D000FCF71AFC4FF0FF3368605EE795E80C0019
:10F7E00003F1004102F1004243422A60696054E79C
:10F7F000032340E707F1004700F100402F606860F5
:10F80000CAF1000349E71F49FCF7FEFB1E49044605
:10F81000FCF7FAFB014628602046FCF7F3FB1A4987
:10F82000FCF7F2FB4FF0FF33686036E719495846A2
:10F83000FCF7F2FC074639462046FCF7E3FB80461E
:10F8400041462046FCF7DEFB3946FCF7DBFB12495C
:10F8500004465846FCF7E0FC2146FCF7D3FB814602
:10F860004946404661E700BFD80F493FE3CB164009
:10F87000800FC93FD00FC93F43443537800F4943FC
:10F88000283301080044353708A3852E84F9223F28
:10F89000A832010800A3852E32318D2420F00042C9
:10F8A000B2F1FF4FF8B5044603462DD25AB30028F3
:10F8B0003DDBB2F5000F4FEAE0502CD37F38C3F3A5
:10F8C0001603C20743F4000348BF5B000027401043
:10F8D0005B003E4619244FF08072B5189D4202DC51
:10F8E0005B1BAE181744013C4FEA43034FEA520238
:10F8F000F3D113B107F001031F447F1007F17C57C8
:10F9000007EBC050F8BDF8BD0146FCF785FC214669
:10F91000FCF77AFBF8BD14F400020FD15B0019026A
:10F9200002F10102FAD5C2F101021044C6E7014614
:10F93000FCF768FB0146FCF723FDF8BD01221044EB
:10F94000BCE700BF2DE9F84320F00046B6F1485F60
:10F9500005460F4649DAFCF725FE002800F09D8099
:10F9600029462846FCF758FC4E490446FCF754FC4F
:10F970004D49FCF749FB2146FCF74EFC4B49FCF78F
:10F9800041FB2146FCF748FC4949FCF73DFB214679
:10F99000FCF742FC4749FCF735FB2146FCF73CFCF1
:10F9A0004549FCF731FB2146FCF736FC80462046F2
:10F9B0004FF07C51FCF730FC414606462046FCF7F0
:10F9C0002BFC394604462846FCF726FC0146204617
:10F9D000FCF718FB01463046FCF714FB01464FF0DC
:10F9E0007E50FCF70FFBBDE8F8830146FCF714FCE2
:10F9F0002C490446FCF710FC2B49FCF705FB21467B
:10FA0000FCF70AFC2949FCF7FDFA2146FCF704FC47
:10FA10002749FCF7F9FA2146FCF7FEFB2549FCF7DC
:10FA2000F1FA2146FCF7F8FB2349FCF7EDFA2146F1
:10FA3000FCF7F2FB214B80469E42B8DD204B9E42F4
:10FA400027DC06F17F4631464FF07E50FCF7DAFAAC
:10FA5000814620464FF07C51FCF7DEFB3146FCF737
:10FA6000D1FA414606462046FCF7D6FB3946044605
:10FA70002846FCF7D1FB01462046FCF7C3FA0146B5
:10FA80003046FCF7BFFA01464846FCF7BBFABDE832
:10FA9000F883DFF834900B4EDBE74FF07E50BDE883
:10FAA000F88300BF4ED747ADF6740F317CF2933424
:10FAB000010DD037610BB63AABAA2A3D9999993E10
:10FAC0000000483F0000903E0000383F2DE9F04F15
:10FAD000DFB00B93013B0293D31E48BF131DB84CFC
:10FAE00006466898DB1054F8204023EAE3730C9331
:10FAF000DB4302EBC30308940693089C029B0C9A19
:10FB00001D190991C3EB02071DD4699C3D4404EB08
:10FB1000870901354FF0000822AC0AE059F80800C7
:10FB2000FCF726FB0137AF4244F8080008F104084F
:10FB300009D0002FF2DA01370020AF4244F8080064
:10FB400008F10408F5D1089A002AC0F2DF82089A69
:10FB50000B9B02F101089C0022AF4FEA8808274462
:10FB60000025029A002AC0F2F28105EB070B4FF044
:10FB700000094FF0000A56F809005BF8041DFCF775
:10FB80004BFB01465046FCF73FFA09F10409A14539
:10FB90008246F0D14AA840F805A004354545E0D199
:10FBA000089A0EAB03EB82030D9391464FEA89034B
:10FBB0000793079A5EAB1344B9F1000F53F850ACAA
:10FBC00023DD0DF134084AAF174490440DAD4FF0DA
:10FBD0006E515046FCF720FBFCF7E4FCFCF7C8FA3A
:10FBE0004FF087418346FCF717FB01465046FCF770
:10FBF00009FAFCF7D7FC594645F8040F57F8040DED
:10FC0000FCF702FA45458246E1D15046069900F0DC
:10FC10008DFC4FF078510546FCF7FEFA00F026FC0B
:10FC20004FF08241FCF7F8FA01462846FCF7EAF962
:10FC30000546FCF7B7FC8246FCF79AFA01462846CF
:10FC4000FCF7E0F9069A8046002A40F3678109F143
:10FC5000FF310EA850F82130C2F1080043FA00F23B
:10FC600002FA00F01B1A06989244C0F1070743FA03
:10FC700007F70EA840F82130002F32DDB9F1000F50
:10FC80000AF1010A40F375810EAB079A1946114437
:10FC9000002507E0C2F5807012B143F8040C01257D
:10FCA0008B420BD053F8042B002DF3D0C2F1FF028E
:10FCB0008B4243F8042C4FF00105F3D1069B002B37
:10FCC0000DDD012B00F03281022B08D109F1FF3349
:10FCD0000EA951F8232002F03F0241F82320022F01
:10FCE00070D040460021FCF72BFC002800F08380F8
:10FCF000089A09F1FF35AA420DDC079A0EAB0D9860
:10FD00001344002253F8041D834242EA0102F9D150
:10FD1000002A40F0E481089B0EA85A1E50F82230B9
:10FD2000002B40F0F18100EB8202012352F8041D08
:10FD300001330029FAD04B4499450A933DDADDF8A6
:10FD40002CA022AACA44DDF8308002EB8A02C84403
:10FD5000C9EB0309131D03920593699A079B4FEAA8
:10FD600089094AAF02EB8808CDF810901F4400259E
:10FD700058F8040FFCF7FCF9029B039A002B505132
:10FD80004FF0000B13DBDDF814A04FF00009AA447C
:10FD900056F809005AF8041DFCF73EFA0146584689
:10FDA000FCF732F909F10409A1458346F0D1049A20
:10FDB0000435954247F804BFDAD1DDF82890F5E61E
:10FDC0004036010841464FF07E50FCF71BF9804653
:10FDD000002D86D006994FF07E5000F0A7FB01461B
:10FDE0004046FCF70FF9804640460021FCF7A8FB8F
:10FDF00000287FF47DAF069B40465942CDF808A00D
:10FE000000F094FB4FF087410446FCF7B7FB002855
:10FE100000F07F814FF06E512046FCF7FDF9FCF7B2
:10FE2000C1FBFCF7A5F94FF087410546FCF7F4F953
:10FE300001462046FCF7E6F8FCF7B4FB0EAB43F8AE
:10FE400029002846FCF7AEFB069C09F101050834A1
:10FE50000EA9069441F8250006994FF07E5000F057
:10FE600065FB002D04464FDB6E1C4FEA8508C6EB90
:10FE7000867A0DF138094AABC1444FEA8A0A9844A0
:10FE80004FF0000B59F80B00FCF772F92146FCF714
:10FE9000C3F94FF06E5148F80B002046FCF7BCF94F
:10FEA000ABF1040BD3450446ECD1DFF88C92DDF8BE
:10FEB00020A00024B34603950497BAF1000FB8BF01
:10FEC000002515DB00263746002501E0A7420FDCA0
:10FED00058F8061059F80600FCF79EF90146284626
:10FEE000FCF792F80137BA45054606F10406EDDA4B
:10FEF0005EA800EB84030134A345A8F1040843F88D
:10FF0000A05CDAD1039D049F689C032C00F29880CA
:10FF1000DFE814F0CB009C009C00310010D109F107
:10FF2000FF330EA951F823703F12A5E609F1FF3304
:10FF30000EA850F8232002F07F0240F82320CEE6DE
:10FF40004FF07C51FCF71AFB58B90746C9E64FF051
:10FF5000000A4AA840F805A0043545457FF401AEE3
:10FF60001EE6B9F1000F4FF002070AF1010A3FF750
:10FF70008BAE0025A2E6002D40F3DC804FEA850B16
:10FF80005EAB36AE05F1FF3A5B4406EB8A0A53F8E6
:10FF9000A08C54465B4635AABB462F4600E0C846B7
:10FFA00054F804594146284601920093FCF72CF876
:10FFB000814649462846FCF725F84146FCF724F8D7
:10FFC000019AC4F804909442A060009BE7D13D469A
:10FFD000012D5F469B4640F3AD805EAB9B445BF8D2
:10FFE000A04C00E044465AF8049921464846FCF7E4
:10FFF0000BF8804641464846FCF704F82146FCF7DA
:020000040801F1
:1000000003F85645CAF80480CAF80800EAD16C1C07
:1000100006EB84040020083654F8041DFBF7F4FFB7
:10002000B442F9D1002F7ED0369A379B099C00F15B
:10003000004002F1004203F10043A06022606360CF
:10004000029A02F007005FB0BDE8F08F002DB8BF44
:1000500000200ADB36AE6C1C002006EB840454F84A
:10006000041DFBF7D1FFB442F9D1002F35D000F1C8
:100070000043099C014623603698FBF7C3FF002D1F
:1000800008DD36AC04EB850554F8041FFBF7BCFF14
:10009000AC42F9D10FB100F10040099A5060029AC8
:1000A00002F007005FB0BDE8F08F002D39DB6C1C5B
:1000B00036AE002006EB840454F8041DFBF7A4FFC1
:1000C000B442F9D10FB100F10040099A1060029AD0
:1000D00002F007005FB0BDE8F08F0346C9E7069A5B
:1000E0000EAC54F82530083ACDF808A00692002B43
:1000F0007FF4B2AE04EB850353F8041D013D083ACA
:100100000029F9D00692A7E6012314E60B9B9C0078
:1001100046E52046FCF746FA0EAA4D4642F829006D
:100120009AE60020CEE7099C369A379BA0602260B1
:10013000636085E7002075E74C3601082DE9F84338
:1001400020F00043B3F1485F04460F46904603DABF
:10015000FCF728FA002857D021462046FCF75CF827
:1001600021460546FCF758F8294906462846FCF77B
:1001700053F82849FBF746FF2946FCF74DF8264976
:10018000FBF742FF2946FCF747F82449FBF73AFF03
:100190002946FCF741F82249FBF736FF8146B8F1C2
:1001A000000F22D038464FF07C51FCF735F8494615
:1001B00080463046FCF730F801464046FBF722FF08
:1001C0002946FCF729F83946FBF71CFF1549054677
:1001D0003046FCF721F801462846FBF715FF01469B
:1001E0002046FBF70FFFBDE8F88349462846FCF799
:1001F00013F80C49FBF706FF3146FCF70DF82146D2
:10020000FBF702FFBDE8F8832046BDE8F88300BF96
:10021000D3C92E2F342FD7321BEF3836010D50396A
:100220008988083CABAA2A3E00207047002001497B
:10023000704700BF0000F87F2DE9F04120F0004535
:10024000B5F1A14F0446064608DBB5F1FF4F6FDC60
:10025000002840F3A0806F48BDE8F0816E4B9D42BE
:1002600077DCB5F1445F68DB4FF0FF37214620466D
:10027000FBF7D2FF01468046FBF7CEFF67490546F4
:10028000FBF7CAFF6649FBF7BFFE2946FBF7C4FF31
:100290006449FBF7B9FE2946FBF7BEFF6249FBF74D
:1002A000B3FE2946FBF7B8FF6049FBF7ADFE2946D0
:1002B000FBF7B2FF5E49FBF7A7FE4146FBF7ACFF39
:1002C0005C4980462846FBF7A7FF5B49FBF79AFE8F
:1002D0002946FBF7A1FF5949FBF794FE2946FBF796
:1002E0009BFF5749FBF78EFE2946FBF795FF5549C3
:1002F000FBF788FE2946FBF78FFF7B1C0146404633
:100300004CD0FBF781FE2146FBF786FF4E4B4F4D4D
:1003100053F82710FBF776FE2146FBF773FE0146E4
:1003200055F82700FBF76EFE002E30DBBDE8F081AC
:100330000146FBF769FEBDE8F0814549FBF764FE25
:100340004FF07E51FCF724F900288DD02046BDE8FF
:10035000F08100F087F83F4B04469D4229DCA3F56D
:10036000D0039D4244DC0146FBF74EFE4FF07E5128
:10037000FBF748FE4FF0804105462046FBF744FE60
:1003800001462846FBF7FCFF002704466EE700F114
:100390000040BDE8F0813048BDE8F081FBF734FE55
:1003A0002146FBF739FF01462046FBF72BFEBDE84F
:1003B000F0812A4B9D4214DC4FF07F51FBF722FE67
:1003C0004FF07F5105462046FBF726FF4FF07E5148
:1003D000FBF71AFE01462846FBF7D2FF0227044628
:1003E00044E701461E48FBF7CBFF032704463DE7E1
:1003F0004FF07E51FBF706FE4FF07E51054620463A
:10040000FBF702FE01462846FBF7BAFF0127044628
:100410002CE700BFDB0FC93FFFFFDF3ED769853CFC
:1004200059DA4B3D356B883D6E2EBA3D2549123E5B
:10043000ABAAAA3E21A215BD6BF16E3D95879D3DED
:10044000388EE33DCDCC4C3E783601088836010825
:10045000CAF24971FFFF973FDB0FC9BFFFFF1B4087
:10046000000080BF20F00040704700BF2DE9F04140
:1004700020F00047FD0D7F3D162D064613DC002DB4
:1004800080461BDB194F2F41074214D01849FBF758
:10049000BBFD0021FCF77CF868B1002E1BDB28EACD
:1004A0000700BDE8F081B7F1FF4F04D30146FBF729
:1004B000ABFDBDE8F0813046BDE8F0810C49FBF7AB
:1004C000A3FD0021FCF764F80028F4D0002E08DB1F
:1004D0000020BDE8F0814FF4000343FA05F5A8447D
:1004E000DDE7002FE7D00348BDE8F081FFFF7F0084
:1004F000CAF24971000080BF30F0004001D10220F3
:100500007047A0F50003B3F1FE4F01D204207047FD
:10051000054B421E9A4201D803207047B0F1FF43B9
:1005200058425841704700BFFEFF7F0038B530F099
:100530000044024603460D4614D0B4F1FF4F0DD2DD
:10054000B4F5000F0FD3E40D2C44FE2C2EDC002C50
:100550001DDD23F0FF4343EAC45038BD0146FBF7DD
:1005600053FD38BD38BD4FF09841FBF755FE194B90
:1005700002469D4207DBC0F3C7540346193CE3E73C
:10058000154800F02DF81449FBF746FE38BD14F16C
:10059000160F13DA4CF250339D421146F0DD0F482E
:1005A00000F01EF80D49FBF737FE38BD11460B4829
:1005B00000F016F80949FBF72FFE38BD04F11900C9
:1005C00023F0FF4343EAC0504FF04C51FBF724FEA9
:1005D00038BD00BFB03CFFFF6042A20DCAF24971B6
:1005E00001F0004120F0004008437047014B1868BB
:1005F000704700BFF4000020780000FF000000FFFB
:100600003C0000FFF00000FF0001746564666D6A45
:1006100069736C67010B020D0A03050B030D0A03D6
:100620000A0B040D0A03080B040D0A031E0000FF49
:100630004A0100FF2C0100FF0E0100FFD20000FF65
:10064000B40000FF960000FF5A0000FF0000FFFF0B
:10065000281D01084C060108FC0501082C060108AC
:100660000006010848060108F805010844060108CB
:10067000400601083C060108040601083806010886
:10068000340601083006010800000000000C01409B
:1006900008001002000C01400400140200000000D9
:1006A0000000000003010000840C010804000000A9
:1006B000440C010804000000040C010802010000C1
:1006C000E40B01080001000000000000060000002B
:1006D000840B010806000000240B01080101000042
:1006E0000000000004000000E40A01080600000009
:1006F000840A010808000000040A0108080000003C
:100700008409010808000000040901080101000033
:1007100000000000000100000000000000010000D7
:100720000000000004000000C408010806000000EA
:100730006408010800010000000000000201000040
:100740004408010801010000000000000000000052
:10075000000000002A08010810080108F607010837
:10076000DC07010801600008BD5F0008995F000810
:10077000715F0008615F000841B60008ED5F000886
:10078000095F0008E15F0008D35F00080000000077
:1007900000C201000C1E01082F1E0108010000000C
:1007A00000E10000441E0108661E0108020000006E
:1007B000009600007A1E01089C1E0108030000003C
:1007C000004B0000B01E0108D21E0108040000000A
:1007D0008025000077240108772401080001060322
:1007E0000703080409040A040B04010402040304B7
:1007F00004040504FFFF00020102020203020402D6
:10080000050206030703080409040A040B04FFFF9A
:10081000000106030703080309030A030B0301038E
:100820000203030304030503FFFF000201020202A7
:1008300003020402050206030703080309030A036F
:100840000B03FFFF0000803F0000000000000000DD
:10085000000080BF0000803F00000000000000009A
:100860000000803F0000803F000080BF0000803F0C
:10087000000080BF0000803F000080BF000080BFFC
:100880000000803F0000803F0000803F0000803F6C
:100890000000803F0000803F0000803F000080BFDC
:1008A000000080BF0000803F00000000000000004A
:1008B000000000000000803F000000000000000079
:1008C000000000000000803F000000000000803FAA
:1008D0000000803F0000803F000080BF000080BF1C
:1008E000000000000000803F000000000000803F8A
:1008F000000080BF0000803F0000803F000080BFFC
:10090000000000800000803F0000803F000000BF2A
:100910000000803F0000803F000000BF000080BF5B
:100920000000803F0000803F000080BF0000003FCB
:100930000000803F0000803F0000003F0000803F3B
:100940000000803F0000803F0000003F000080BFAB
:10095000000080BF0000803F000080BF000000BF9B
:10096000000080BF0000803F000000BF0000803F0B
:10097000000080BF0000803F0000803F0000003F7B
:10098000000080BF0000803FF704353FF70435BF0B
:100990000000803F0000803FF70435BFF70435BFFB
:1009A0000000803F0000803FF70435BFF704353F6B
:1009B0000000803F0000803FF704353FF704353FDB
:1009C0000000803F0000803F00000000000080BF6A
:1009D000000080BF0000803F000080BF00000000DA
:1009E000000080BF0000803F000000000000803F4A
:1009F000000080BF0000803F0000803F000000003A
:100A0000000080BF0000803F000080BF0000803FEA
:100A1000000080BF0000803F000080BF000080BF5A
:100A20000000803F0000803F0000803F0000803FCA
:100A30000000803F0000803F0000803F000080BF3A
:100A4000000080BF0000803F000080BF0000803FAA
:100A50000000803F0000803F000080BF000080BF9A
:100A6000000080BF0000803F0000803F0000803F0A
:100A7000000080BF0000803F0000803F000080BF7A
:100A80000000803F0000803F000000BFD0B35D3F0A
:100A90000000803F0000803F000000BFD0B35DBF7A
:100AA0000000803F0000803F0000003FD0B35D3F6A
:100AB000000080BF0000803F0000003FD0B35DBF5A
:100AC000000080BF0000803F000080BF00000000E9
:100AD000000080BF0000803F0000803F0000000059
:100AE0000000803F0000803F000000000000803FC9
:100AF000000080BF0000803F000080BF000080BF7A
:100B0000000000000000803F000000000000803F67
:100B10000000803F0000803F0000803F000080BF59
:100B2000000000000000803FD0B35DBF0000003F28
:100B30000000803F0000803FD0B35DBF000000BFD9
:100B4000000080BF0000803FD0B35D3F0000003F49
:100B50000000803F0000803FD0B35D3F000000BF39
:100B6000000080BF0000803F00000000000080BF48
:100B70000000803F0000803F000000000000803F38
:100B8000000080BF0000803F00000000A8AAAA3F2C
:100B90000000803F0000803F000080BFB0AA2ABF55
:100BA000000080BF0000803F0000803FB0AA2ABF45
:100BB000000080BF0000803F00000000A8AAAA3FFC
:100BC000000080BF0000803F000080BFB0AA2ABFA5
:100BD0000000803F0000803F0000803FB0AA2ABF95
:100BE0000000803F0000803F0000803F00000000C8
:100BF000000000000000803F000080BF00000000F7
:100C0000000000000000803F000080BF0000803F27
:100C1000000080BF0000803F000080BF000080BF58
:100C20000000803F0000803F0000803F0000803FC8
:100C30000000803F0000803F0000803F000080BF38
:100C4000000080BF0000803F000000000000803FE7
:100C5000000080BF0000803F000080BF0000000057
:100C60000000803F0000803F0000803F0000000047
:100C70000000803F0000803F00000000000080BFB7
:100C8000000080BF0000803F00000000A8AAAA3F2B
:100C9000000000000000803F000080BFB0AA2ABF13
:100CA000000000000000803F0000803FB0AA2ABF83
:100CB0000000000001000102000103000104000126
:100CC0000500010600010700010800010900010AF2
:100CD00000010B00010C010300000000E61E0108EA
:100CE0000000000001000000EB1E010801000000F0
:100CF00002000000F21E01080200000003000000D4
:100D0000FB1E01080300000004000000011F010891
:100D10000500000005000000061F01080600000095
:100D200006000000101F0108070000000700000077
:100D3000191F01080800000008000000221F010818
:100D400009000000090000002B1F01080A00000034
:100D50000A000000351F01080B0000000B00000016
:100D60003F1F01080C0000000C000000491F010893
:100D70000D0000000D000000511F01080E000000D2
:100D80000E000000591F01080F0000000F000000B6
:100D9000611F010810000000100000006A1F010818
:100DA0001100000011000000711F01081200000076
:100DB000120000007B1F0108130000001300000058
:100DC000831F010814000000140000008E1F01089A
:100DD0001500000015000000981F01081600000013
:100DE0001600000000000000FF000000B5620601D0
:100DF0000300F00500FF19B56206010300F00300CF
:100E0000FD15B56206010300F00100FB11B5620695
:100E1000010300F00000FA0FB56206010300F002C2
:100E200000FC13B56206010300F00400FE17B56272
:100E3000060103000102010E47B56206010300012D
:100E400003010F49B56206010300010601124FB507
:100E500062060103000112011E67B5620608060062
:100E6000C80001000100DE6A00B562061608000332
:100E70000703000000000031E501B5620616080016
:100E800003070300510800008A4102B562061608F4
:100E9000000307030004E00400199D03B562061671
:100EA0000800030703000002020035EF04B56206E4
:100EB0001608000307030080010000B2E8004000AC
:100EC0008000000100020004495746415401020419
:100ED0000810204E45535755442C3A3A0000000064
:100EE000000000008025000000C201000600000094
:100EF000010000008025000000C201000700000082
:100F00000200000080250000004B000009000000E6
:100F10001E1E64646464646422004602210082012F
:100F20002000430210000101000049020100880175
:100F300002004C0212008401110090011100900186
:100F40001100A0011100A0016B9400088994000811
:100F5000A5940008A9760008D1940008DD94000843
:100F600095A200083994000807940008214E000853
:100F7000559400081D4E000811230108182301088C
:100F80001D2301082E2301083823010843230108EB
:100F90004E230108592301085D2301086623010837
:100FA0006C230108762301088422010884230108A8
:100FB000942301089B230108A4230108AE23010800
:100FC00000000000524F4C4C3B50495443483B59A1
:100FD00041573B414C543B506F733B506F73523BF6
:100FE0004E6176523B4C4556454C3B4D41473B5636
:100FF000454C3B00E6210108DD210108D121010813
:1010000000010000C3240108CC24010825A8000821
:10101000F0240108F424010859A900080A25010850
:101020000F25010819410008232501082925010879
:10103000D93E0008CF2301083A250108B98A0008E3
:10104000572501085C250108E5B100088B2501083A
:1010500077240108D58A0008902501089825010801
:10106000A5790008AC250108B025010841AA0008AF
:10107000C3250108D2250108059D0008EC250108BB
:1010800077240108454A0008F1250108F5250108E3
:10109000114800080426010808260108714A0008C2
:1010A0001D250108242601089D3D0008372601085A
:1010B0003D260108393E00083B2F0108582601084B
:1010C00099B1000867260108582601084D6C0008F0
:1010D0007326010878260108018B00083A210108CF
:1010E000882601089DAA0008B6260108AA2601083C
:1010F000D5A60008012D010877240108B54700088E
:10110000020000008025000000C201000000000075
:10111000200000008025000000C201000100000046
:10112000400000008025000000C201000000000017
:10113000010000008025000000C201000000000046
:10114000100000008025000000C201000003000024
:101150000400000080250000004B0000000000009B
:101160000800000000E1000000E1000000040000B1
:1011700034280108392801083D28010846280108BB
:1011800066230108592301084228010800000000D5
:1011900077240108F0270108F82701080028010832
:1011A000082801080F2801081A2801082228010828
:1011B0002A2801082F280108000000009001C8001B
:1011C000C800C800C800C800C800C800C800640043
:1011D0000000C800C800C800C80032005F2901082C
:1011E00063290108692901086F290108722901088A
:1011F000792901087C290108812901088D29010824
:1012000090290108962901089D290108A7290108AC
:10121000B1290108BA290108C8290108D4290108FF
:10122000DB290108E1290108EE290108F929010853
:10123000062A010800000000222A010844000000DC
:10124000D419002000000000282300002B2A0108E8
:1012500041000000D619002000000000010000003D
:10126000392A010844000000E21A0020B0040000FE
:10127000A4060000402A010844000000E41A0020EF
:1012800000000000D00700004A2A010844000000C6
:10129000E61A002000000000D0070000542A0108D0
:1012A00042000000E81A00200000000012000000C8
:1012B000612A010842000000E91A00200100000034
:1012C000FF0000006C2A010842000000EA1A00201A
:1012D0000000000001000000812A01084400000015
:1012E000981A002000000000D00700008E2A010894
:1012F000440000009A1A002000000000D0070000FF
:101300009B2A0108440000009C1A002000000000F5
:10131000D0070000A72A0108440000009E1A002000
:1013200000000000D0070000B72A010844000000B8
:10133000A01A002000000000D0070000C82A010801
:1013400044000000A21A002000000000D0070000A6
:10135000D32A010844000000A41A00200000000065
:10136000D0070000E82A010844000000A61A002067
:1013700032000000007D0000F72A01084400000050
:10138000A81A002032000000F2010000062B01081C
:1013900041000000EB1A00200000000001000000E6
:1013A000132B010841000000EC1A0020000000008F
:1013B00001000000262B010841000000ED1A00206A
:1013C00000000000B4000000322B010841000000C2
:1013D000EE1A002000000000640000003E2B01080F
:1013E00042000000EF1A0020FFFFFFFF0100000095
:1013F000542B010841000000F41A002000000000F6
:10140000090000006B2B010841000000F51A0020C4
:101410000000000009000000822B010841000000CC
:10142000F61A00200000000009000000992B0108B6
:1014300041000000081B0020300000007E0000007A
:10144000AA2B010850000000F81A0020B004000088
:1014500000C20100B72B010850000000FC1A002058
:10146000B004000000C20100C42B010850000000BD
:10147000001B00200000000000C20100D12B010869
:1014800050000000041B0020B004000000C2010056
:10149000EA2B010841000000F01A002000000000C3
:1014A00001000000F72B010841000000F11A0020A4
:1014B0000000000004000000052C010841000000AD
:1014C000F21A00200000000001000000152C0108A5
:1014D00081000000E41B002000000000C8000000A4
:1014E0001F2C010881000000EE1B002000000000FE
:1014F000C8000000292C010881000000F81B002012
:1015000000000000C8000000332C0108810000002A
:10151000E51B002000000000C80000003E2C010870
:1015200081000000EF1B002000000000C800000048
:10153000492C010881000000F91B00200000000078
:10154000C8000000542C010881000000E61B0020A8
:1015500000000000C80000005E2C010881000000AF
:10156000F01B002000000000C8000000682C0108EB
:1015700081000000FA1B002000000000C8000000ED
:10158000722C0108840000008E1D00200000000065
:10159000D0070000802C010881000000921D00206F
:1015A0000000000001000000952C010884000000EC
:1015B000941D00200A000000D0070000A32C0108A1
:1015C00084000000961D00200A000000D0070000E3
:1015D000B12C010881000000911D002000000000D6
:1015E00064000000BF2C010841000000E01A002048
:1015F0000000000003000000D12C010841000000A1
:101600000C1B00200000000003000000E42C010877
:10161000410000000D1B0020000000000100000040
:10162000F52C0108410000000E1B00200000000006
:1016300001000000092D010860000000101B0020BF
:10164000A6FFFFFF5A000000212D010860000000E6
:10165000141B00204CFFFFFFB4000000392D0108CF
:1016600041000000181B00200000000001000000E5
:10167000522D010841000000191B0020000000004D
:10168000010000005D2D010844000000D61A002072
:1016900000000000204E00006E2D010841000000F7
:1016A000CC1A002000000000FF000000792D010886
:1016B00041000000CD1A00200A00000032000000A6
:1016C0008F2D010841000000CE1A00200A00000002
:1016D00032000000A52D010844000000D01A0020AF
:1016E0000100000010270000B92D0108440000008F
:1016F000D21A00200000000072060000CE2D010862
:1017000041000000D41A0020000000000100000089
:10171000EC2D010841000000AA1A00200000000082
:1017200008000000F72D010841000000AB1A00205E
:101730000000000008000000012E01084100000028
:10174000AC1A002000000000080000000B2E010869
:1017500048000000AE1A00204CFFFFFF68010000A7
:101760001C2E010848000000B01A00204CFFFFFFAB
:10177000680100002E2E010848000000B21A002067
:101780004CFFFFFF680100003E2E010844000000EE
:10179000BE1A00206400000084030000542E0108DB
:1017A00044000000B61A0020000000000001000004
:1017B0005D2E010841000000BC1A0020000000005E
:1017C000800000006D2E010844000000B81A0020BF
:1017D00064000000E80300007E2E010844000000C1
:1017E000BA1A002064000000E8030000902E0108EF
:1017F000810000003B1D002001000000FA000000F5
:10180000A22E0108810000003C1D00200000000005
:1018100001000000992E010881000000391D002000
:101820000000000020000000B72E01088100000029
:101830003A1D00200000000064000000C42E0108D2
:1018400081000000401D0020000000009600000004
:10185000DE2E0108840000003E1D00200100000073
:1018600084030000F82E010842000000B41A002092
:10187000FFFFFFFF010000000E2F010882000000A3
:101880008A1D0020FFFFFFFF010000001C2F010840
:10189000820000008B1D00200000000001000000FD
:1018A0002E2F0108810000002C1C002000000000E9
:1018B00002000000432F0108010100001E2100204A
:1018C00000000000FA0000004B2F01080101000099
:1018D0001F2100200000000064000000532F0108B9
:1018E0000101000020210020000000006400000031
:1018F0005B2F0108010100002121002000000000F1
:1019000064000000642F0108010100002221002072
:101910000000000064000000742F010801010000B5
:101920002321002000000000640000007D2F01083A
:1019300001010000242100200000000064000000DC
:10194000862F01080401000026210020E803000082
:10195000D0070000952F010881000000821D0020A3
:1019600000000000C8000000A42F01088100000052
:10197000831D002000000000C8000000B72F0108F0
:1019800084000000841D0020E8030000D007000050
:10199000C92F010884000000861D0020640000009B
:1019A000D0070000DB2F010884000000881D002004
:1019B00064000000B80B0000ED2F0108810000005A
:1019C0008C1D002000000000FF000000FA2F01081D
:1019D00041000000B51A00200000000009000000CE
:1019E0000730010881000000341C002000000000C6
:1019F000FA00000016300108810000003C1C0020A5
:101A00000000000064000000253001088100000093
:101A10003D1C00200000000064000000333001087D
:101A2000A0000000381C002001000000140000008D
:101A30004330010881000000501C0020000000001D
:101A4000010000005230010888000000321C002014
:101A5000D4FEFFFF2C010000613001088800000067
:101A6000301C0020D4FEFFFF2C0100006F30010865
:101A700081000000401C0020000000003000000039
:101A80007D300108A0000000441C00200000000080
:101A9000010000008C300108A0000000481C00205C
:101AA000000000000100000098300108A0000000C4
:101AB0004C1C00200000000001000000A4300108C0
:101AC000880000002E1C0020B0B9FFFF5046000027
:101AD000B430010881000000DC1B00200000000081
:101AE00002000000C330010881000000E11B00205B
:101AF00000000000C8000000CB3001088100000099
:101B0000EB1B002000000000C8000000262E01088A
:101B100081000000F51B002000000000C80000004C
:101B2000D330010881000000E01B0020000000000D
:101B3000C8000000DA30010881000000EA1B002024
:101B400000000000C8000000152E01088100000000
:101B5000F41B002000000000C8000000E130010874
:101B600081000000E21B002000000000C80000000F
:101B7000E730010881000000EC1B0020000000009D
:101B8000C8000000382E010881000000F61B00206C
:101B900000000000C8000000ED300108A0000000B7
:101BA000041C00200000000064000000F630010862
:101BB000A0000000101C00200000000064000000D5
:101BC000FF300108A00000001C1C002000000000E5
:101BD0006400000008310108A0000000001C002083
:101BE000000000006400000010310108A0000000A7
:101BF0000C1C0020000000006400000018310108E7
